:020000040000FA
:1000000099EF00F01200000080EF01F012001200E2
:10001000FFFFFFFFFFFFFFFFDCEF01F01200060E06
:10002000F66E000EF76E000EF86E04010900F55032
:10003000F96F0900F550FA6F03E1F96701D03DD07F
:100040000900F550F46F0900F550F56F0900F550FF
:10005000F66F09000900F550E96E0900F550EA6EE7
:10006000090009000900F550F76F0900F550F86F15
:1000700009000900F6CFFBF4F7CFFCF4F8CFFDF44C
:10008000F4C4F6FFF5C4F7FFF6C4F8FF0401F75314
:1000900002E1F85307E00900F550EE6EF707F8E2C9
:1000A000F807F9D7FBC4F6FFFCC4F7FFFDC4F8FF5F
:1000B0000401F907000EFA5BBFD71200120110010C
:1000C00002000008D8040A00010000000001090233
:1000D0004300020100C064090400000102020000A4
:1000E0000524001001042402020524060001052451
:1000F0000100010705820308000209040100020A49
:1001000000000007050302400001070583024000CC
:1001100001FF400EF36E00EE00F00F0E01D812004A
:10012000EA6002D0EE6AFCD7F350E9601200EE6A92
:10013000FCD71EEE00F02EEE00F0F86A049C0FECE7
:1001400000F007EC00F075EC02F0FBD71200FFFFA7
:10015000FFFFFFFFFFFFFFFFFFFFFFFFFFFFFFFFAF
:10016000FFFFFFFFFFFFFFFFFFFFFFFFFFFFFFFF9F
:10017000FFFFFFFFFFFFFFFFFFFFFFFFFFFFFFFF8F
:10018000FFFFFFFFFFFFFFFFFFFFFFFFFFFFFFFF7F
:10019000FFFFFFFFFFFFFFFFFFFFFFFFFFFFFFFF6F
:1001A000FFFFFFFFFFFFFFFFFFFFFFFFFFFFFFFF5F
:1001B000FFFFFFFFFFFFFFFFFFFFFFFFFFFFFFFF4F
:1001C000FFFFFFFFFFFFFFFFFFFFFFFFFFFFFFFF3F
:1001D000FFFFFFFFFFFFFFFFFFFFFFFFFFFFFFFF2F
:1001E000FFFFFFFFFFFFFFFFFFFFFFFFFFFFFFFF1F
:1001F000FFFFFFFFFFFFFFFFFFFFFFFFFFFFFFFF0F
:10020000FFFFFFFFFFFFFFFFFFFFFFFFFFFFFFFFFE
:10021000FFFFFFFFFFFFFFFFFFFFFFFFFFFFFFFFEE
:10022000FFFFFFFFFFFFFFFFFFFFFFFFFFFFFFFFDE
:10023000FFFFFFFFFFFFFFFFFFFFFFFFFFFFFFFFCE
:10024000FFFFFFFFFFFFFFFFFFFFFFFFFFFFFFFFBE
:10025000FFFFFFFFFFFFFFFFFFFFFFFFFFFFFFFFAE
:10026000FFFFFFFFFFFFFFFFFFFFFFFFFFFFFFFF9E
:10027000FFFFFFFFFFFFFFFFFFFFFFFFFFFFFFFF8E
:10028000FFFFFFFFFFFFFFFFFFFFFFFFFFFFFFFF7E
:10029000FFFFFFFFFFFFFFFFFFFFFFFFFFFFFFFF6E
:1002A000FFFFFFFFFFFFFFFFFFFFFFFFFFFFFFFF5E
:1002B000FFFFFFFFFFFFFFFFFFFFFFFFFFFFFFFF4E
:1002C000FFFFFFFFFFFFFFFFFFFFFFFFFFFFFFFF3E
:1002D000FFFFFFFFFFFFFFFFFFFFFFFFFFFFFFFF2E
:1002E000FFFFFFFFFFFFFFFFFFFFFFFFFFFFFFFF1E
:1002F000FFFFFFFFFFFFFFFFFFFFFFFFFFFFFFFF0E
:10030000DACFE4FFE2CFDAFFE9CFE4FFEACFE4FFA0
:10031000F6CFE4FFF7CFE4FFF5CFE4FFF3CFE4FF40
:10032000F4CFE4FFFACFE4FF00EE03F0020EE8049E
:1003300003E3EECFE4FFFBD700EE00F0030EE8048A
:1003400003E3EECFE4FFFBD7E6521EEC7AF0A4AA5B
:100350000FD00401EA050BE19CA207D09C98030191
:10036000020EFE6F1AEC0CF09C88D6EC33F0A49AC7
:10037000E55200EE02F0030EE80403E3E5CFEDFFE3
:10038000FBD700EE04F0020EE80403E3E5CFEDFF37
:10039000FBD7E5CFFAFFE5CFF4FFE5CFF3FFE5CFDD
:1003A000F5FFE5CFF7FFE5CFF6FFE5CFEAFFE5CFB5
:1003B000E9FFE5CFDAFF1100D8CFE4FFE0CFE4FF9B
:1003C000E46EDACFE4FFE2CFDAFFE652F250200B20
:1003D00001E182D0F250040B01E17ED0F2940101E0
:1003E000E2070101E25101E077D00101180EE26F4E
:1003F0000F0130B38B780F013DA90AD08B9A0B0106
:10040000782B060E0B01785D03E10B01786B8B8A6C
:100410000F0131A105D08B908B720101EB6B22D0C3
:100420000F0131A913D00F0131B38B820F0131A518
:1004300007D08B808B50010B02E08B8201D08B9216
:100440000F0131B78B800F0131990CD08B908B92BB
:100450000101EB2B080E0101EB5D04E10101EB6BE7
:100460000F0131890F0132A10CD00D01FE2BE60ED8
:100470000D01FE5D06E10D01FE6B0F0132910F01D2
:1004800032830F013CB70ED00F013CA10AD00B0103
:10049000732BE30E0B01735D04E10B01736B0F0112
:1004A0003D810DD00F013BAF0AD00B01762BE30E3F
:1004B0000B01765D04E10B01766B0F013D810F01AD
:1004C0003CAB0AD00B01772BE30E0B01775D04E107
:1004D0000B01776B0F013C9BE552E5CFDAFFE5504E
:1004E000E5CFE0FFE5CFD8FF100024EC10F00C01C1
:1004F000100EF96F22EC0CF077EC10F0F9EC36F0FE
:100500000C01100EF96F22EC0CF04EEC18F0550EA9
:100510000001A05D06E1AA0E0001A15D02E100EC70
:10052000FCF0E5EC17F0CC6A2EEC0CF08A980C018C
:10053000B00EF96F22EC0CF00F013181F28EF28CCB
:1005400085AA0BD00C01200EF96F22EC0CF085AAC5
:1005500004D00F01308F13EC7AF00C01300EF96FDC
:1005600022EC0CF0DFEC4CF00ED00F01316B8A88DE
:100570000C01FA0EF96F22EC0CF08A980C01600E57
:10058000F96F22EC0CF00F01010E316F0C01700EAF
:10059000F96F22EC0CF00301FF6BFE0E0301FF5D0F
:1005A0000BE20301FF51EA6A000FE96E050EEA2231
:1005B000EF6A0301FF2BF1D70F01299F89820C01FC
:1005C0004A0EF96F22EC0CF00301FF6B0E0E0301D3
:1005D000FF5D12E20C01250EF96F22EC0CF085AEE6
:1005E00006D00F0129BF08D00F01298F02D00F01BB
:1005F000299F0301FF2BEAD70C01F40EF96F22ECBF
:100600000CF089920C01FA0EF96F22EC0CF00C013F
:10061000FA0EF96F22EC0CF085AEA7D70F012893E4
:100620009E9A0C01FA6B030E0C01FA5D16E2B7EC10
:100630003FF00301FF6BA00E0301FF5D0BE20F0112
:1006400028B30CD0CC6A2EEC0CF02EEC0CF003018D
:10065000FF2BF1D70C01FA2BE6D787D70C010B0E35
:10066000F96F22EC0CF00F0128930C01FA6B020ECB
:100670000C01FA5D16E2EBEC40F00301FF6BA00EFB
:100680000301FF5D0BE20F0128B30BD0CC6A2EEC07
:100690000CF02EEC0CF00301FF2BF1D70C01FA2B20
:1006A000E6D70601FF6B3FEC4CF0AAEC31F00F01EE
:1006B0003D9B0F013EA108D00F013E91F6EC19F0D1
:1006C0000301FE690301FE690F013EA504D00F017D
:1006D0003E9533EC1AF00C010B0EF96F22EC0CF086
:1006E0000F0128930C01FA6B020E0C01FA5D19E25E
:1006F00054EC41F00301FF6BA00E0301FF5D0EE21D
:100700000F0128B554D00F0128B70CD0CC6A2EECBD
:100710000CF02EEC0CF00301FF2BEED70C01FA2BA2
:10072000E3D727D00C01200EF96F22EC0CF00F015B
:1007300028930F0128950F0128970C01FA6B030EDF
:100740000C01FA5D16E227EC41F00301FF6BA00EED
:100750000301FF5D0BE20F0128B529D0CC6A2EEC16
:100760000CF02EEC0CF00301FF2BF1D70C01FA2B4F
:10077000E6D70F012A9B0F012AB918D0600EE66E4A
:10078000000EE66E5EEC7AF0E552E5521DEC4FF09D
:10079000AAEC31F00F0129AB04D00F01299B0F0106
:1007A0002A890F0130A702D0ADEC18F0DED60C017B
:1007B0000B0EF96F22EC0CF00F0128930C01FA6B71
:1007C000030E0C01FA5D16E205EC40F00301FF6B2D
:1007D000A00E0301FF5D0BE20F0128B30BD0CC6A22
:1007E0002EEC0CF02EEC0CF00301FF2BF1D70C01DA
:1007F000FA2BE6D70C010B0EF96F22EC0CF00F016F
:1008000028930C01FA6B020E0C01FA5D16E2E1EC82
:100810003FF00301FF6BA00E0301FF5D0BE20F0130
:1008200028B30BD0CC6A2EEC0CF02EEC0CF00301AC
:10083000FF2BF1D70C01FA2BE6D70C01200EF96F34
:1008400022EC0CF00F0128930F0128950F01289737
:100850000C01FA6B020E0C01FA5D16E205EC42F097
:100860000301FF6BA00E0301FF5D0BE20F0128B334
:100870000BD0CC6A2EEC0CF02EEC0CF00301FF2B0D
:10088000F1D70C01FA2BE6D70C01200EF96F22EC00
:100890000CF00F0128930C01FA6B020E0C01FA5DAB
:1008A00016E2DBEC41F00301FF6BA00E0301FF5DDC
:1008B0000BE20F0128B30BD0CC6A2EEC0CF02EEC1F
:1008C0000CF00301FF2BF1D70C01FA2BE6D70C013A
:1008D000200EF96F22EC0CF00F0128930C01FA6B3B
:1008E000020E0C01FA5D16E21FEC45F00301FF6BEE
:1008F000A00E0301FF5D0BE20F0128B30BD0CC6A01
:100900002EEC0CF02EEC0CF00301FF2BF1D70C01B8
:10091000FA2BE6D70C01200EF96F22EC0CF00F0138
:1009200028930C01FA6B020E0C01FA5D16E24CECF6
:1009300045F00301FF6BA00E0301FF5D0BE20F0109
:1009400028B30BD0CC6A2EEC0CF02EEC0CF003018B
:10095000FF2BF1D70C01FA2BE6D70C01200EF96F13
:1009600022EC0CF00F0128930C01FA6B020E0C0123
:10097000FA5D16E273EC45F00301FF6BA00E030174
:10098000FF5D0BE20F0128B30BD0CC6A2EEC0CF00C
:100990002EEC0CF00301FF2BF1D70C01FA2BE6D75C
:1009A0000C01200EF96F22EC0CF00F0128930C01C2
:1009B000FA6B020E0C01FA5D16E29DEC45F00301A4
:1009C000FF6BA00E0301FF5D0BE20F0128B30BD0FC
:1009D000CC6A2EEC0CF02EEC0CF00301FF2BF1D7BF
:1009E0000C01FA2BE6D70F0139A123D00C01200E00
:1009F000F96F22EC0CF00F0128930C01FA6B020E38
:100A00000C01FA5D16E25EEC47F00301FF6BA00EED
:100A10000301FF5D0BE20F0128B30BD0CC6A2EEC73
:100A20000CF02EEC0CF00301FF2BF1D70C01FA2B8C
:100A3000E6D70C01200EF96F22EC0CF00F01289381
:100A40000C01FA6B020E0C01FA5D16E2FFEC45F0A8
:100A50000301FF6BA00E0301FF5D0BE20F0128B342
:100A60000BD0CC6A2EEC0CF02EEC0CF00301FF2B1B
:100A7000F1D70C01FA2BE6D70C010B0EF96F22EC23
:100A80000CF00F0129930C01FA6B100E0C01FA5DAA
:100A900016E2B1EC41F00301FF6BF00E0301FF5DC4
:100AA0000BE20F0129B30CD0CC6A2EEC0CF02EEC2B
:100AB0000CF00301FF2BF1D70C01FA2BE6D763D51D
:100AC0000F012A990F0128930F012ABB1BD0600E3A
:100AD000E66E000EE66E5EEC7AF0E552E55230EC22
:100AE00050F00F012A8BAAEC31F00F0130A702D091
:100AF000ADEC18F00F0129BB05D00101010E3B6FD1
:100B000005EC2EF00F01299B0F012B6B0301FC6BF1
:100B10000301FD6BFC0E0301FD5D0BE20301FD51C2
:100B2000EA6A000FE96E030EEA22EF6A0301FD2B69
:100B3000F1D70F0128930101E6510101E85D1EE0A4
:100B4000C0EC2EF0FDEC5AF0AAEC31F00F0130A70A
:100B500002D0ADEC18F00F0129AB10D00F01299B8A
:100B60000101E82B400E0101E85D02E10101E86BA3
:100B70000C01160EF96F22EC0CF0DDD70F012A9153
:100B80000F012A930101756B020E0101755D01E3EE
:100B900076D075EC41F00101766BF00E0101765DC7
:100BA0006BE20F012AA14CD00101772B0101786B78
:100BB0000101792B0A0E0101775D0EE10101776BCE
:100BC0000F012AB509D00F012A970101020E3B6FD0
:100BD00005EC2EF00F012A850F0E0101795D2FE142
:100BE0000101776B0101796B0F013DA710D00F0157
:100BF0003D830B01AE6B3BEC3BF00C01FA0EF96F41
:100C000022EC0CF00C01FA0EF96F22EC0CF00F0143
:100C10003DA510D00F013D830B01AD6B16EC3CF0F0
:100C20000C01FA0EF96F22EC0CF00C01FA0EF96FC0
:100C300022EC0CF00F013C6B0F013D6B96D452D0AF
:100C40000F012AA313D00101776B0101786B010119
:100C5000796B0F012AB709D00F012A950101030E04
:100C60003B6F05EC2EF00F012A873CD0CC6A2EECAE
:100C70000CF00101762B91D70101752B85D701016D
:100C8000782B020E0101785D2DE10101786B0F01D7
:100C90003DA710D00F013D830B01AE6B3BEC3BF049
:100CA0000C01FA0EF96F22EC0CF00C01FA0EF96F40
:100CB00022EC0CF00F013DA510D00F013D830B017C
:100CC000AD6B16EC3CF00C01FA0EF96F22EC0CF057
:100CD0000C01FA0EF96F22EC0CF00F013C6B0F01C6
:100CE0003D6B43D496EC41F00C01600EF96F22ECA1
:100CF0000CF0EFEC47F00C01600EF96F22EC0CF0F9
:100D00000D01005101E1DBD00F012AA3D8D00F0162
:100D100028930F012DA715D02BEC40F00301FF6B9A
:100D2000A00E0301FF5D0BE2CC6A2EEC0CF02EEC62
:100D30000CF00F0128B319D00301FF2BF1D7BFD05E
:100D400014D005EC40F00301FF6BA00E0301FF5D22
:100D50000BE2CC6A2EEC0CF02EEC0CF00F0128B359
:100D600004D00301FF2BF1D7AAD00C01200EF96F9C
:100D700022EC0CF00F012DB703D023EC42F002D08F
:100D800098EC42F00F012C930F012C970301FF6B9D
:100D9000FF0E0301FF5D1BE2CC6A2EEC0CF02EEC83
:100DA0000CF00F012CA310D00F012C93CC6A2EEC69
:100DB0000CF02EEC0CF00F012DB703D006EC43F035
:100DC00002D080EC43F029D00301FF2BE1D716ECD1
:100DD00045F0CC6A2EEC0CF00101E32B030E01016F
:100DE000E35D1AE10101E36B0F01299D0101F36B42
:100DF000FE0E0101F35D0BE20101F351EA6A000FFF
:100E0000E96E0D0EEA22EF6A0101F32BF1D7010121
:100E1000090E3B6F05EC2EF052D00301FF6BFF0E65
:100E20000301FF5D2CE2CC6A2EEC0CF02EEC0CF0F2
:100E30002EEC0CF02EEC0CF00F012CA71DD00F01A6
:100E40002C970101E36B0F01299D0101F36BFE0E4D
:100E50000101F35D0BE20101F351EA6A000FE96E53
:100E60000D0EEA22EF6A0101F32BF1D70101080E02
:100E70003B6F05EC2EF023D00301FF2BD0D70101EF
:100E8000E32B030E0101E35D1AE10101E36B0F01A6
:100E9000299D0101F36BFE0E0101F35D0BE20101DF
:100EA000F351EA6A000FE96E0D0EEA22EF6A0101C2
:100EB000F32BF1D70101090E3B6F05EC2EF00F016A
:100EC00029A50BD0DFEC4CF00F0129950F013D9DBA
:100ED0000C01300EF96F22EC0CF00F0138A90BD089
:100EE0002BEC4DF00F0138990F013D9D0C01300E98
:100EF000F96F22EC0CF00F0138A126D018EC5AF053
:100F00000F0138AD08D06CEC4EF00F01389D0F0189
:100F10003D9D0F0138910F0138AB08D0D5EC4EF054
:100F20000F01389B0F013D9D0F0138910F0138A132
:100F300006D0A9EC4DF00F013D9D0F0138910C0139
:100F4000100EF96F22EC0CF00F0138A50DD0CFEC8C
:100F500059F0E2EC4DF00F0138950F013D9D0C0169
:100F6000100EF96F22EC0CF00F0138AF0BD021EC12
:100F70004EF00F01389F0F013D9D0C01100EF96FCF
:100F800022EC0CF00C01200EF96F22EC0CF00101A8
:100F90002B5102E0F7EC30F00F012B6B0F0130B555
:100FA000B3D10F0128930F012AAF19D005EC40F0FF
:100FB0000301FF6BA00E0301FF5D11E2CC6A2EEC72
:100FC0000CF02EEC0CF00F0128A306D00C01200E23
:100FD000F96F22EC0CF003D00301FF2BEBD751EC9F
:100FE00040F00301FF6BD00E0301FF5D13E2CC6AFA
:100FF0002EEC0CF02EEC0CF00F012BA108D04CECD9
:101000002EF001017A6B01017B6B0F012B91030123
:10101000FF2BE9D701017C5101E176D17CC17AF146
:101020007DC17BF101017B5102E00F012B830F0198
:10103000289381EC40F00301FF6BA00E0301FF5DDC
:101040000BE2CC6A2EEC0CF02EEC0CF00F0128B366
:1010500003D00301FF2BF1D70F012BB70BD00101F8
:10106000CD2B020E0101CD5D01E2E1D70101CD6B77
:101070000F012A8D0F012B978B840F012893B2EC5F
:1010800040F00301FF6BA00E0301FF5D09E2CC6A93
:101090002EEC0CF00F0128B303D00301FF2BF3D784
:1010A00079EC2EF00101CD6B0101F56B0101F66BBE
:1010B0000F012BA9B4D00F012B990F012EA118D02D
:1010C0003AEC30F00101E62B400E0101E65D02E151
:1010D0000101E66B0101E8510101E65D08E1010152
:1010E000E82B400E0101E85D02E10101E86B11D03F
:1010F0000101E56B100E0101E55D0BE20101E55117
:10110000EA6A100FE96E010EEA22EF6A0101E52B8F
:10111000F1D77DEC2FF00101E62B400E0101E65DD9
:1011200002E10101E66B0101E8510101E65D08E120
:101130000101E82B400E0101E85D02E10101E86BCD
:1011400001016E5126E00F012EB30AD00101F551C5
:10115000EA6A460FE96E010EEA22EFCF06F109D0E6
:101160000101F551EA6A460FE96E010EEA22EFCF5E
:1011700009F10101F52B0101F551EA6A460FE96E0B
:10118000010EEA22EFCF0AF10101F52B01016E07F2
:10119000C0D70C01F05142E00101F651EA6A000F9C
:1011A000E96E0C0EEA22EFCF08F10101F629EA6A96
:1011B000000FE96E0C0EEA22EFCF09F1020E0101D9
:1011C000F625EA6A000FE96E0C0EEA22EFCF0AF16B
:1011D000030E0101F625EA6A000FE96E0C0EEA2201
:1011E000EFCF0BF1040E0101F625EA6A000FE96E5C
:1011F0000C0EEA22EFCF0CF1050E0101F625EA6A8A
:10120000000FE96E0C0EEA22EFCF0DF1060E010180
:10121000F6250101F66F0C01F0077BD771D00F01A5
:101220002ABD6ED00F012EA129D0FDEC5AF001018C
:10123000E56B100E0101E55D0BE20101E551EA6A83
:10124000000FE96E010EEA22EF6A0101E52BF1D7EA
:101250000F010F013C51800B05E00F010F013D51C3
:10126000400B0BE0AAEC31F00F01299B0F0130A7D6
:1012700002D0ADEC18F00F013D9D11D00101E56BDE
:10128000100E0101E55D0BE20101E551EA6A000F74
:10129000E96E010EEA22EF6A0101E52BF1D71FEC9E
:1012A00052F00F010F013C51800B05E00F010F01BF
:1012B0003D51400B0BE0AAEC31F00F01299B0F01CF
:1012C00030A702D0ADEC18F00F013D9D0F012EA705
:1012D00017D076EC52F00F010F013C51800B05E066
:1012E0000F010F013D51400B0BE0AAEC31F00F0153
:1012F000299B0F0130A702D0ADEC18F00F013D9DE6
:101300000F012A9D8B9486D60F0139AF33D00F0180
:1013100039BD20D00F01289300EC41F00301FF6B91
:10132000600E0301FF5D08E20F0128B305D0CC6A0F
:1013300095DA0301FF2BF4D70F01399F0F01399D77
:1013400012EC41F0CC6A0C01FA0EF96F7BDAB4ECC6
:1013500056F010D00F01399F0F01399D12EC41F06A
:1013600001010F0E3B6F05EC2EF0CC6A0C01A00EB4
:10137000F96F68DA0F0130AB32D00F01309B0501F5
:10138000FF2B050E0501FF5D2AE10501FF6B0F0133
:101390003DA70ED00F013D830B01AE6B3BEC3BF044
:1013A0000C01FA0EF96F4EDA0C01FA0EF96F4ADAF7
:1013B0000F013DA50ED00F013D830B01AD6B16EC67
:1013C0003CF00C01FA0EF96F3DDA0C01FA0EF96FE0
:1013D00039DA0F013C6B0F013D6BB5EF02F00101F3
:1013E000E6510101E85D4EE00101E1510101E05DDE
:1013F0002AE00101E02BC0EC2EF0FDEC5AF00F01C9
:101400000F013C51800B05E00F010F013D51400BD6
:1014100019E0AAEC31F00F013D9D0F0130A702D079
:10142000ADEC18F00F0129AB0DD00F01299B010184
:10143000E06B0101E82B400E0101E85D02E10101D2
:10144000E86BCDD71FD00F012DBF1CD00F012D8F02
:101450008A860C012D0EF96FF5D98A960C012D0E96
:10146000F96FF0D98A860C012D0EF96FEBD98A96A7
:101470000C012D0EF96FE6D98A860C015A0EF96F10
:10148000E1D98A960401F25108E13FEC4CF00F01DA
:101490003D8BAAEC31F00F013D9B0F0130A702D02C
:1014A000ADEC18F00F013EA104D00F013E91F6EC17
:1014B00019F00F013EA504D00F013E9533EC1AF050
:1014C0000F0129AB41D00F01299B0F013B990B0163
:1014D000726B0B01756B0D01FF6B0F012D9F0F01DF
:1014E0003CAF2AD00F0139AB16D00F013DA706D073
:1014F0000F013D830B01AE6B3BEC3BF00F013C9FBA
:101500000B01AE6B0F013AAD05D001010C0E3B6F24
:1015100005EC2EF002D00F013A8D0F013ABB0CD032
:101520000F013C9F0B01AE6B0F013BAB05D00101DE
:101530000D0E3B6F05EC2EF00101E1510101E05D64
:1015400002E10101E06B47D00F013BB944D00B0130
:10155000722B070E0B01725D1EE10B01726B0F0106
:101560003C8F0F013B890F013A9D0F013DA706D02B
:101570000F013D830B01AE6B3BEC3BF00F013DA532
:1015800006D00F013D830B01AD6B16EC3CF00B0157
:10159000AD6B0B01AE6B0F0130AF1DD00D01FF2BFA
:1015A000070E0D01FF5D17E10D01FF6B0F01309F6D
:1015B0001BEC7AF00C01F00EF96F44D90C01F00E1F
:1015C000F96F40D90C01F00EF96F3CD90C01F00E07
:1015D000F96F38D928D10F0139AF33D00F0139BD98
:1015E00020D00F01289300EC41F00301FF6B600E47
:1015F0000301FF5D08E20F0128B305D0CC6A2ED9A4
:101600000301FF2BF4D70F01399F0F01399D12EC15
:1016100041F0CC6A0C01FA0EF96F14D9B4EC56F013
:1016200010D00F01399F0F01399D12EC41F00101DB
:101630000F0E3B6F05EC2EF0CC6A0C01A00EF96F7B
:1016400001D90F013CAF77D00F013AB128D036EC69
:101650003AF097EC4CF00F013DAD1FD0AAEC31F001
:101660000F013D9D0F0129AB0ED00F01299B0F01EA
:101670002D9F0B01756B0101E1510101E05D02E15C
:101680000101E06B0AD00B01752B030E0B01755D98
:1016900004E10B01756B0F013D833BEC3BF00F0147
:1016A0003AAD48D00F013AB113D00B01AF2B280E41
:1016B0000B01AF5D0CE10B01AF6B0F013D830B0123
:1016C000AE6B3BEC3BF00B01AE6B0F013A8132D0BD
:1016D0000F0139B31FD00F0139A517D00F01399170
:1016E0000F0128939DEC45F00301FF6BA00E030151
:1016F000FF5D09E20F0128B306D0CC6AAFD8AED89F
:101700000301FF2BF3D70F013981CFEC3BF016EC2F
:101710003CF010D00F013A910B01AD6B0F0139B9BC
:1017200009D00F0139890F01399B01010B0E3B6F65
:1017300005EC2EF050D00F013AB310D00F013DB799
:101740000AD00B01B02B070E0B01B05D04E10B01B9
:10175000B06B36EC3AF03BEC3BF03DD00F0139B3C7
:101760002AD00F0139A517D00F0139910F01289305
:101770009DEC45F00301FF6BA00E0301FF5D09E244
:101780000F0128B306D0CC6A69D868D80301FF2BB3
:10179000F3D70F0139810F013DB50AD00B01AC2BF6
:1017A000070E0B01AC5D04E10B01AC6BCFEC3BF021
:1017B00016EC3CF010D00F013A930B01AD6B0F010A
:1017C00039B909D00F0139890F01399B01010B0E7D
:1017D0003B6F05EC2EF00F0130BF19D085AA16D053
:1017E0000C01200EF96F2ED885AA10D00F01308F72
:1017F00013EC7AF00C01500EF96F24D8600EE66EEF
:10180000000EE66E5EEC7AF0E552E5520CD085BA39
:101810000AD00C01200EF96F15D885BA04D00F013B
:10182000309F1BEC7AF00301FE690301FE69BEEFF5
:1018300005F012000301FE5103E00301FE07FAD791
:10184000040012000C01F86B0C01F9510C01F85D59
:1018500004E204D80C01F82BF7D712009E920C0179
:10186000FB6B0F0E0C01FB5D2EE29EB228D0030134
:10187000020EFE6FDFDFACA206D0AC980301020EB1
:10188000FE6FD8DFAC889EAA11D0AFCFFEF59E9A2E
:10189000B9EC2DF00A0E0501FE5D02E122EC6EF0BE
:1018A0003E0E0501FE5D02E10F012C839CA206D0D5
:1018B0009C980301020EFE6FBDDF9C88D6D79E92D6
:1018C0000C01FB2BCED70F0130B117D081B212D053
:1018D0000101EF2B100E0101EF5D0BE10101EF6B38
:1018E0000F0130810F0130830101060E3B6F05ECC3
:1018F0002EF002D00101EF6B17D081A213D00101AD
:10190000EF2B100E0101EF5D0CE10101EF6B0F01F8
:1019100030910F0130938B880101070E3B6F05EC6E
:101920002EF002D00101EF6B0F0130B921D081B44C
:1019300013D00101F02B0101F16B100E0101F05DDC
:101940000AE10101F06B0F0130890101040E3B6FC8
:1019500005EC2EF08B960BD00101F06B0101F12B01
:101960000A0E0101F15D03E10101F16B8B8615D0D7
:1019700081A411D00101F02B100E0101F05D0AE1EC
:101980000101F06B0F0130990101050E3B6F05EC71
:101990002EF08B8602D00101F06B12009E920C019A
:1019A000FB6B0F0E0C01FB5D6DE29EB267D0030175
:1019B000020EFE6F3FDFACA206D0AC980301020E10
:1019C000FE6F38DFAC889EAA50D0AFCFFEF5FEC5C3
:1019D000FEF69E9A0F0129B11AD0060E0501FE5D92
:1019E00015E10F0129810101F36BFE0E0101F35D89
:1019F0000BE20101F351EA6A000FE96E060EEA22DA
:101A0000EF6A0101F32BF1D70601FF6B20D0060E20
:101A10000501FE5D02E0DAEC2DF0140E0501FE5D1D
:101A200016E1F9EC11F00F0129890101F36BFE0EAB
:101A30000101F35D0BE20101F351EA6A000FE96E67
:101A4000050EEA22EF6A0101F32BF1D785D0B9EC3C
:101A50002DF00A0E0501FE5D02E122EC6EF03E0E55
:101A60000501FE5D02E10F012C839CA206D09C982B
:101A70000301020EFE6FDEDE9C8897D79E920C015A
:101A8000FB2B8FD70F0130B117D081B212D00101DB
:101A9000EF2B100E0101EF5D0BE10101EF6B0F0168
:101AA00030810F0130830101060E3B6F05EC2EF0F3
:101AB00002D00101EF6B17D081A213D00101EF2BEF
:101AC000100E0101EF5D0CE10101EF6B0F01309190
:101AD0000F0130938B880101070E3B6F05EC2EF050
:101AE00002D00101EF6B0F0130B921D081B413D0C6
:101AF0000101F02B0101F16B100E0101F05D0AE113
:101B00000101F06B0F0130890101040E3B6F05EC00
:101B10002EF08B960BD00101F06B0101F12B0A0E18
:101B20000101F15D03E10101F16B8B8615D081A408
:101B300011D00101F02B100E0101F05D0AE101014D
:101B4000F06B0F0130990101050E3B6F05EC2EF093
:101B50008B8602D00101F06B12009E920C01FB6B90
:101B60000F0E0C01FB5D01E304D29EB2FED1030116
:101B7000020EFE6F5FDEACA206D0AC980301020E2F
:101B8000FE6F58DEAC889EAA11D0AFCFFEF59E9AAC
:101B9000B9EC2DF00A0E0501FE5D02E122EC6EF0BB
:101BA0003E0E0501FE5D02E10F012C830F0130BFE7
:101BB000D9D09CA206D09C980301020EFE6F3ADE9B
:101BC0009C88A4AACED0AACFFEF6A49A0F0129B170
:101BD00020D0060E0601FE5D1BE10F0129810101E7
:101BE000F36BFE0E0101F35D0BE20101F351EA6AB2
:101BF000000FE96E060EEA22EF6A0101F32BF1D71E
:101C00000601FF6B0F013E990F013E9B0F013E9DA8
:101C1000A8D00F013EBB0FD0060E0601FE5D02E00C
:101C2000DAEC2DF0140E0601FE5D04E1E2DB0F019B
:101C3000298909D217D0DAEC2DF00F010F013E519E
:101C4000400B08E0140E0601FE5D04E1D2DB0F013B
:101C50002989F9D10601FE5103E10F013E8D02D021
:101C60000F013E9D0F013EB97AD0230E0601FE5DA5
:101C700076E10F013E890F013E8B0101FE6B110ED3
:101C80000101FE5D31E20101FE51EA6A000FE96ED9
:101C9000060EEA22EF50230824E12A0E0601005D19
:101CA00008E1230E0601015D04E10F013E9B57D0C0
:101CB00018D00101FF6B0101FE510101FF5D10E22F
:101CC0000101FF51EA6A000FE96E060EEA22EF50A9
:101CD0003A0803E10F013E9B42D00101FF2BEBD7F5
:101CE00006D00101FE2BCBD70F013E9B38D001015E
:101CF000FE5103E10F013E9B32D00B01B96B2B0E5D
:101D00000601005D09E10B01010EB96F0101FE053D
:101D100003E10F013E9B23D0B9CBFFF10101FE513E
:101D20000101FF5D1CE20101FF51EA6A000FE96E4B
:101D3000060EEA22EFCF00F0300E005C0AE301014C
:101D4000FF51EA6A000FE96E060EEA22EF503908E9
:101D500003E20F013E9B03D00101FF2BDFD70101FE
:101D6000FF6B02D128EC7AF00001A06F0001A051B6
:101D700001E1F8D0600EE66E000EE66E5EEC7AF0E1
:101D8000E552E5520101F96B0001A0510101F95D35
:101D900001E3D7D00101F951EA6A600FE96E000E44
:101DA000EA22EFCFFEF60F0129B120D0060E060180
:101DB000FE5D1BE10F0129810101F36BFE0E0101A4
:101DC000F35D0BE20101F351EA6A000FE96E060EC2
:101DD000EA22EF6A0101F32BF1D70601FF6B0F0135
:101DE0003E990F013E9B0F013E9DA8D00F013EBBC7
:101DF0000FD0060E0601FE5D02E0DAEC2DF0140EA7
:101E00000601FE5D04E1F5DA0F0129891CD117D026
:101E1000DAEC2DF00F010F013E51400B08E0140EDB
:101E20000601FE5D04E1E5DA0F0129890CD1060106
:101E3000FE5103E10F013E8D02D00F013E9D0F01C7
:101E40003EB97AD0230E0601FE5D76E10F013E8990
:101E50000F013E8B0101FE6B110E0101FE5D31E2AF
:101E60000101FE51EA6A000FE96E060EEA22EF5008
:101E7000230824E12A0E0601005D08E1230E060175
:101E8000015D04E10F013E9B57D018D00101FF6BAB
:101E90000101FE510101FF5D10E20101FF51EA6AFB
:101EA000000FE96E060EEA22EF503A0803E10F0137
:101EB0003E9B42D00101FF2BEBD706D00101FE2B48
:101EC000CBD70F013E9B38D00101FE5103E10F013A
:101ED0003E9B32D00B01B96B2B0E0601005D09E170
:101EE0000B01010EB96F0101FE0503E10F013E9BDD
:101EF00023D0B9CBFFF10101FE510101FF5D1CE2CE
:101F00000101FF51EA6A000FE96E060EEA22EFCFE7
:101F100000F0300E005C0AE30101FF51EA6A000F95
:101F2000E96E060EEA22EF50390803E20F013E9BEC
:101F300003D00101FF2BDFD70101FF6B0101F92B5A
:101F400023D70101F96B400E0101F95D0BE201019C
:101F5000F951EA6A600FE96E000EEA22EF6A0101A8
:101F6000F92BF1D70001A06B00D69E920C01FB2B40
:101F7000F7D50F0130B117D081B212D00101EF2B8C
:101F8000100E0101EF5D0BE10101EF6B0F013081DC
:101F90000F0130830101060E3B6F05EC2EF002D0DD
:101FA0000101EF6B17D081A213D00101EF2B100EAE
:101FB0000101EF5D0CE10101EF6B0F0130910F01A9
:101FC00030938B880101070E3B6F05EC2EF002D099
:101FD0000101EF6B0F0130B921D081B413D00101A1
:101FE000F02B0101F16B100E0101F05D0AE101011E
:101FF000F06B0F0130890101040E3B6F05EC2EF0F0
:102000008B960BD00101F06B0101F12B0A0E01013F
:10201000F15D03E10101F16B8B8615D081A411D034
:102020000101F02B100E0101F05D0AE10101F06BDE
:102030000F0130990101050E3B6F05EC2EF08B86E8
:1020400002D00101F06B1200400E9B6E896A0C0EEB
:10205000926E8A6AE60E936E100E8B6E800E946EF0
:102060008C6A956A8D6A966A8E6AB80E976E8F6AC8
:10207000040E986E656A200EF26E800EF16EF06AA4
:102080009D6AA06AA36A100EA26E200EA56ED08E65
:10209000C70ED56ECD6A070ECA6ECB68796A766AAE
:1020A000BB6AB66AB16A736A706AC66A6C6AC088CB
:1020B0009F0EC16EFC0EC26E010ECE6EC098C26A3B
:1020C000C16AD26AD16AA66A0F014B6B0401F26B36
:1020D000220EAD6E900EAC6E220EA86E900E9C6E0F
:1020E0007E6A260EB06E7C6A260EAB6E1200D9CFC9
:1020F000E6FFE1CFD9FFE6520C01A00EF16F0F0110
:10210000286B0F01296B0F01306B0F01316B01013F
:10211000E06B0501FE6B0F012A6B0101E66B01010B
:10212000E86B0101776B0101786B0101796B0101AB
:10213000EF6B0101F06B0101F16B01017A6B0101A1
:102140007B6B0F012B6B0101CD6B0F012C6B010120
:10215000DE6B0101DF6B0101E36B0F012D6B0101F0
:102160006E6B0C01F06B0F012E6B0101180EE26F0C
:102170000101EB6B01013B6B0501FF6B0001A06BE3
:102180000001A16B0D01FE6B0F01326B0F01336B70
:102190000F01346B0D01FF6B0F01386B0F01396BB1
:1021A0000F013A6B0F013B6B0F013C6B0F013D6B55
:1021B0000B01726B0B01756B0B01746B0B01736B75
:1021C0000B01766B0B01776B0B01786B0F013E6B8C
:1021D0000B01AC6B0B01AF6B0B01B06B0B01AD6B6B
:1021E0000B01AE6B0601FF6BDF6AFE0EDF5C09E2DE
:1021F000DF50EA6A000FE96E050EEA22EF6ADF2A75
:10220000F4D7DF6A100EDF5C09E2DF50EA6A000FE4
:10221000E96E010EEA22EF6ADF2AF4D7DF6A100EB8
:10222000DF5C09E2DF50EA6A100FE96E010EEA2274
:10223000EF6ADF2AF4D7DF6A100EDF5C09E2DF50B5
:10224000EA6A180FE96E0F0EEA22EF68DF2AF4D768
:10225000DF6A100EDF5C09E2DF50EA6A790FE96E8F
:102260000B0EEA22EF68DF2AF4D7DF6A100EDF5C7C
:1022700009E2DF50EA6A2B0FE96E010EEA22EF6AEB
:10228000DF2AF4D7DF6A0A0EDF5C09E2DF50EA6A70
:102290003C0FE96E010EEA22EF6ADF2AF4D7DF6A0B
:1022A000100EDF5C09E2DF50EA6ACE0FE96E010E24
:1022B000EA22EF6ADF2AF4D7DF6A100EDF5C09E258
:1022C000DF50EA6A020FE96E0F0EEA22EF6ADF2A98
:1022D000F4D7DF6AFE0EDF5C09E2DF50EA6A000F26
:1022E000E96E060EEA22EF6ADF2AF4D7DF6A500EA3
:1022F000DF5C09E2DF50EA6A7C0FE96E010EEA2238
:10230000EF6ADF2AF4D7DF6AFE0EDF5C09E2DF50F6
:10231000EA6A000FE96E0D0EEA22EF6ADF2AF4D7AF
:10232000DF6A280EDF5C09E2DF50EA6A460FE96ED9
:10233000010EEA22EF6ADF2AF4D7DF6AF00EDF5CD3
:1023400009E2DF50EA6A000FE96E0C0EEA22EF6A3A
:10235000DF2AF4D7DF6A400EDF5C09E2DF50EA6A69
:10236000600FE96E000EEA22EF6ADF2AF4D7DF6A17
:10237000060EDF5C09E2DF50EA6AB10FE96E0B0E70
:10238000EA22EF6ADF2AF4D7DF6AFF0EDF5C1EE283
:10239000DF50EA6A000FE96E070EEA22EF6ADF50AB
:1023A000EA6A000FE96E080EEA22EF6ADF50EA6A75
:1023B000000FE96E090EEA22EF6ADF50EA6A000FA9
:1023C000E96E0A0EEA22EF6ADF2ADFD70701FF6B08
:1023D0000801FF6B0901FF6B0A01FF6B0101320E5F
:1023E000FA6F0101310EFB6FE552E552E7CFD9FFDD
:1023F00012000F013CBFDBD0730E0601005D2BE124
:10240000660E0601015D27E1690E0601025D23E10A
:10241000720E0601035D1FE16D0E0601045D1BE1F6
:10242000140E0601055D17E10F0130870101F36B02
:10243000FE0E0101F35D0BE20101F351EA6A000FA8
:10244000E96E060EEA22EF6A0101F32BF1D70601CD
:10245000FF6BABEF16F06D0E0601005D2BE16F0E0A
:102460000601015D27E1640E0601025D23E1650EB0
:102470000601035D1FE13F0E0601045D1BE1140E22
:102480000601055D17E10F013E810101F36BFE0EB0
:102490000101F35D0BE20101F351EA6A000FE96EFD
:1024A000060EEA22EF6A0101F32BF1D70601FF6B5A
:1024B000ABEF16F0300E0601005D3BE1300E060179
:1024C000015D37E1300E0601025D33E1300E060199
:1024D000035D2FE13A0E0601045D2BE16C0E06014F
:1024E000055D27E1630E0601065D23E1660E060128
:1024F000075D1FE1670E0601085D1BE1140E060172
:10250000095D17E10F013E830101F36BFE0E01012E
:10251000F35D0BE20101F351EA6A000FE96E060E6A
:10252000EA22EF6A0101F32BF1D70601FF6BABEF53
:1025300016F0300E0601005D3AE1300E0601015D35
:1025400036E1300E0601025D32E1300E0601035D18
:102550002EE13A0E0601045D2AE1730E0601055DC7
:1025600026E1630E0601065D22E1660E0601075DA7
:102570001EE1670E0601085D1AE1140E0601095DF1
:1025800016E10F013E850101F36BFE0E0101F35DC3
:102590000BE20101F351EA6A000FE96E060EEA222E
:1025A000EF6A0101F32BF1D70601FF6BD4D3760E4E
:1025B0000601005D22E1650E0601015D1EE1720E5D
:1025C0000601025D1AE13F0E0601035D16E10F01EF
:1025D00029850101F36BFE0E0101F35D0BE20101A0
:1025E000F351EA6A000FE96E060EEA22EF6A010172
:1025F000F32BF1D70601FF6BAED3630E0601005D2E
:1026000022E1730E0601015D1EE1710E0601025DFD
:102610001AE13F0E0601035D16E10F013889010141
:10262000F36BFE0E0101F35D0BE20101F351EA6A67
:10263000000FE96E060EEA22EF6A0101F32BF1D7D3
:102640000601FF6B88D3630E0601005D2AE16C0E64
:102650000601015D26E1650E0601025D22E1610EC3
:102660000601035D1EE1720E0601045D1AE1140EFF
:102670000601055D16E10F0138850101F36BFE0EC1
:102680000101F35D0BE20101F351EA6A000FE96E0B
:10269000060EEA22EF6A0101F32BF1D70601FF6B68
:1026A0005AD30F013EABF1D00D01005101E0D7D05C
:1026B0000D01010E006F0D01016B0B01B9510101FC
:1026C000FE5D0D01026F0D01910E036F0B01030EF4
:1026D000B76F0F013E9FB9CBFFF10101FE51010120
:1026E000FF5D4FE20101FF51EA6A000FE96E060E3D
:1026F000EA22EF50D00FE66E0101FF51EA6A000FA7
:10270000E96E060EEA22E552E750EF6E0F013E7FBA
:102710000F013EBF33D00B01B72B0101FF51EA6A15
:10272000000FE96E060EEA22EF38F00BE66E0B01A1
:10273000B751EA6A000FE96E0D0EEA22E552E75042
:10274000EF6E0101FF05EA6A000FE96E060EEA224C
:10275000EFCF00F00B01B751EA6A000FE96E0D0EE2
:10276000EA22EF500024E66E0B01B751EA6A000F2F
:10277000E96E0D0EEA22E552E750EF6E0101FF2BE4
:10278000ACD70B01B72B0F013EAF16D00101FF05EF
:10279000EA6A000FE96E060EEA22EF50F00FE66ECD
:1027A0000B01B751EA6A000FE96E0D0EEA22E552FD
:1027B000E750EF6E0B01B72B0B01B751EA6A000F20
:1027C000E96E0D0EEA22EF6A0B01B72B0B01B75130
:1027D000EA6A000FE96E0D0EEA22080EEF6E0B0199
:1027E000B72B030E0601FF5D0601FF6F0101FE51CD
:1027F0000601FF5DE66E0B01B751EA6A000FE96E54
:102800000D0EEA22E552E750EF6E0101FE2B0601A4
:10281000FF2BFEC1FFF10601FF510101FF5D18E230
:102820000B01B72B0101FF51EA6A000FE96E060E9A
:10283000EA22EF50E66E0B01B751EA6A000FE96E2B
:102840000D0EEA22E552E750EF6E0101FF2BE3D7B0
:102850000B01B7290B01B86F0F012D8702D00F01B3
:10286000298D0101F36BFE0E0101F35D0BE2010105
:10287000F351EA6A000FE96E060EEA22EF6A0101DF
:10288000F32BF1D70601FF6B66D20101F26B010158
:10289000F26B110E0101F25D0EE20101F251EA6AE2
:1028A000000FE96E060EEA22EF503A0801E119D056
:1028B0000101F22BEED70101F36BFE0E0101F35D76
:1028C0000BE20101F351EA6A000FE96E060EEA22FB
:1028D000EF6A0101F32BF1D70601FF6B0F012D8584
:1028E0003AD2730E0601005D01E0D0D1650E0601FB
:1028F000015D01E0CBD1740E0601025D01E0C6D19D
:102900003A0E0601035D01E0C1D12C0E0601045D03
:1029100003E10F01388FA6D10101040EF26F01010E
:10292000F36B110E0101F35D2BE20101F251EA6A32
:10293000000FE96E060EEA22EF502C0803E10101B8
:10294000F20721D00101F251EA6A000FE96E060E8A
:10295000EA22EFCF00F0300E005C0AE30101F251F1
:10296000EA6A000FE96E060EEA22EF50390803E228
:102970000F01388F77D10101F22B0101F32BD1D751
:102980000F01388F6FD10101F36B0B0E0101F35D65
:102990000BE20101F351EA6A180FE96E0F0EEA2209
:1029A000EF680101F32BF1D7040E0101F25D03E1A1
:1029B00004C618FF25D00101F46BF2C1F3F1010147
:1029C000F35103081DE20101F351EA6A000FE96EB9
:1029D000060EEA22EF50E66E0101F451EA6A180F82
:1029E000E96E0F0EEA22E552E750EF6E0101F42B7B
:1029F0000B0E0101F45D01E103D00101F307DFD704
:102A0000020E0101F2250101F26F01010B0EF46FBC
:102A10000101F36B040E0101F35D01E38AD00101B2
:102A2000F251EA6A000FE96E060EEA22EF502F0813
:102A30000CE20101F251EA6A000FE96E060EEA2289
:102A4000EFCF00F03A0E005C2CE30101F251EA6A8C
:102A5000000FE96E060EEA22EF5040080CE2010179
:102A6000F251EA6A000FE96E060EEA22EFCF01F09A
:102A7000470E015C16E30101F251EA6A000FE96EAC
:102A8000060EEA22EF5060084CE20101F251EA6AB8
:102A9000000FE96E060EEA22EFCF02F0670E025C2D
:102AA00040E20101F251EA6A000FE96E060EEA22E5
:102AB000EF50600820E20101F251EA6A000FE96E6E
:102AC000060EEA22EFCF00F0670E005C14E201016F
:102AD000F251EA6A000FE96E060EEA22EF50E00FAB
:102AE000E66E0101F251EA6A000FE96E060EEA2273
:102AF000E552E750EF6E0101F251EA6A000FE96E0C
:102B0000060EEA22EF50E66E0101F451EA6A180F50
:102B1000E96E0F0EEA22E552E750EF6E0101F42B49
:102B200003D00F01388F9ED00101F22B0101F32B4E
:102B300071D70101F251EA6A000FE96E060EEA222E
:102B4000EF502C0803E00F01388F8CD00101F22BDD
:102B50000101F251EA6A000FE96E060EEA22EF5017
:102B600030080CE20101F251EA6A000FE96E060E2C
:102B7000EA22EFCF00F03A0E005C2CE30101F251A3
:102B8000EA6A000FE96E060EEA22EF5040080CE2F6
:102B90000101F251EA6A000FE96E060EEA22EFCF58
:102BA00001F0470E015C16E30101F251EA6A000FE1
:102BB000E96E060EEA22EF50600840E20101F25190
:102BC000EA6A000FE96E060EEA22EFCF02F0670E06
:102BD000025C34E20101F251EA6A000FE96E060E6E
:102BE000EA22EF50600820E20101F251EA6A000F88
:102BF000E96E060EEA22EFCF00F0670E005C14E2E9
:102C00000101F251EA6A000FE96E060EEA22EF5066
:102C1000E00FE66E0101F251EA6A000FE96E060E5E
:102C2000EA22E552E750EF6E0101F251EA6A000F25
:102C3000E96E060EEA22EFCF27FF03D00F01388F8F
:102C400011D00101F22B0101F251EA6A000FE96E85
:102C5000060EEA22EF50140803E00F01388F02D06D
:102C60000F0138810101F36BFE0E0101F35D0BE2F0
:102C70000101F351EA6A000FE96E060EEA22EF6ADB
:102C80000101F32BF1D70601FF6B65D02A0E060177
:102C9000005D18E1230E0601015D14E1300E06010E
:102CA000025D10E12A0E0601035D0CE13A0E0601F9
:102CB000045D08E10601FF050101746F0F012D811C
:102CC0004AD049D00101F46B2B0E0601005D03E1EF
:102CD0000101010EF46FF4C1F3F10101F2510101A0
:102CE000F35D1CE20101F351EA6A000FE96E060E82
:102CF000EA22EFCF00F0300E005C0AE30101F3514D
:102D0000EA6A000FE96E060EEA22EF50390803E284
:102D10000F012D850DD00101F32BDFD70D010051DF
:102D200005E19FEC2EF00F012D9702D00F01298DA8
:102D30000101F36BFE0E0101F35D0BE20101F351A2
:102D4000EA6A000FE96E060EEA22EF6A0101F32B30
:102D5000F1D70601FF6B1200966A0001A26B000119
:102D6000A36B8F980F01309D8F960301FE69A2C05F
:102D70008DFF0301FE698F80A3C08CFF0F010F013F
:102D80003051400B02E08E8C01D08E9C8F9003015D
:102D9000FE698D680301FE698F880301FE690301E6
:102DA000FE690301FE698F980001A22B0001A25168
:102DB00012E10001A32B0001A3510DE10F0130BD71
:102DC00003D00F01308D07D00001A26B0001A36B6F
:102DD0000F01309D01D0C9D712008F980301FE6901
:102DE0008F960301FE69A2C08DFF966A0301FE69FA
:102DF0008F80A3C08CFF0F010F013051400B02E008
:102E00008E8C01D08E9C0301FE698F900301FE69B8
:102E1000A4C08DFF0301FE698F880301FE690301D1
:102E2000FE690301FE698F980301FE691200D9CF84
:102E3000E6FFE1CFD9FFE6520001080EA26F0001C4
:102E4000A36B0F01309D8F86DF6AA2C08DFF966A4B
:102E50000301FE698F80A3C08CFF0F010F01305169
:102E6000400B02E08E8C01D08E9C0301FE698F9096
:102E70008F8896680301FE69DF50EA6A000FE96EE9
:102E8000070EEA2284CFEFFF8F98DF2A040EDF5C63
:102E900003E20001A22BD9D7800E0701005D0BE1F0
:102EA000EF0E0701015D07E10701020504E1F00EE5
:102EB0000701035D02E00F0134870301FE6903018E
:102EC000FE69E552E552E7CFD9FF1200D9CFE6FF00
:102ED000E1CFD9FFE6520001850EA26F0001A36B7E
:102EE0008F86DF6AA2C08DFF966A0301FE698F801C
:102EF000A3C08CFF8E9C0301FE698F908F8896681B
:102F00000301FE69DF50EA6A790FE96E0B0EEA22CF
:102F100084CFEFFF8F98DF2A040EDF5C03E200010D
:102F2000A22BE0D7340E0B01795D14E1310E0B01B9
:102F30007A5D10E1300E0B017B5D0CE30B017B51E0
:102F4000390808E3300E0B017C5D04E30B017C5172
:102F5000390802E20F0134870301FE690301FE69AB
:102F6000E552E552E7CFD9FF1200D9CFE6FFE1CF16
:102F7000D9FFE6528F86DF6AA2C08DFF966A0301F1
:102F8000FE698F80A3C08CFF8E9C0301FE698F9029
:102F90008F8896680301FE69DF50EA6A790FE96E4F
:102FA0000B0EEA2284CFEFFF8F98DF2A100EDF5C32
:102FB00003E20001A22BE0D70301FE690301FE69D1
:102FC000E552E552E7CFD9FF12008F980001A26BBE
:102FD0000001A36B0F01309D8F960301FE69A2C013
:102FE0008DFF966A0301FE698F80A3C08CFF0F01DD
:102FF0000F013051400B02E08E8C01D08E9C0301FA
:10300000FE698F900301FE69A2C08DFF8F880301C6
:10301000FE690301FE690301FE698F980301FE69E1
:103020008F860301FE698F80A3C08CFF0F010F0103
:103030003051400B02E08E8C01D08E9C8F900001AD
:10304000A06B8F8896680301FE6984CFA0F08F98EB
:103050000301FE690001A2510001A05D0EE08B8A10
:103060000C01200EF96F22EC0CF08B9A0C01200E53
:10307000F96F22EC0CF0F3D710D00F0130BD0DD05A
:103080000001A22B0001A25107E10001A32B0001C6
:10309000A35102E10F01308D9FD712008F860301EB
:1030A000FE69FE0E8D6E966A0301FE698F808C6844
:1030B0008E8C0301FE698F908F8896680301FE69EC
:1030C00084CFA0F08F980301FE698D68966A030192
:1030D000FE698F808C688E8C0301FE698F908F88CB
:1030E00096680301FE6984CFA1F08F980301FE6901
:1030F00012008F960301FE69FE0E8D6E966A030123
:10310000FE698F808C688E8C0301FE698F900301AD
:10311000FE69550E8D6E8F880301FE690301FE69FD
:103120000301FE698F980301FE698D680301FE6942
:103130008F808C688E8C0301FE698F900301FE697D
:10314000AA0E8D6E8F880301FE690301FE690301DB
:10315000FE698F980301FE691200CAEC20F0FCDDC5
:10316000CAEC20F0CAEC20F0CAEC20F0CAEC20F047
:10317000CAEC20F06BEC4AF00F01309D0F01328158
:103180000D01FE6B0001AC6B0001AD6B0001AE6B7D
:103190000001AF6B0F01006B0F01016B0F01336B6F
:1031A0000F01346B0F01356BDEEC20F00F0134ADF5
:1031B00040D0CAEC20F0B1EC4AF0CAEC20F0CAECE6
:1031C00020F0CAEC20F00F0130AF0CD01BEC7AF0ED
:1031D000CAEC20F0CAEC20F0CAEC20F0CAEC20F0D7
:1031E000CAEC20F00F013DA710D00F013D830B0169
:1031F000AE6B3BEC3BF0CAEC20F0CAEC20F0CAEC22
:1032000020F0CAEC20F0CAEC20F00F013DA510D050
:103210000F013D830B01AD6B16EC3CF0CAEC20F0C6
:10322000CAEC20F0CAEC20F0CAEC20F0CAEC20F086
:10323000FF000F0134A540D0CAEC20F0DFEC4AF0CB
:10324000CAEC20F0CAEC20F0CAEC20F00F0130AF3D
:103250000CD01BEC7AF0CAEC20F0CAEC20F0CAECDF
:1032600020F0CAEC20F0CAEC20F00F013DA710D0EE
:103270000F013D830B01AE6B3BEC3BF0CAEC20F041
:10328000CAEC20F0CAEC20F0CAEC20F0CAEC20F026
:103290000F013DA510D00F013D830B01AD6B16EC66
:1032A0003CF0CAEC20F0CAEC20F0CAEC20F0CAECEA
:1032B00020F0CAEC20F0FF000F0134A95CD0CAEC6A
:1032C00020F0B5DD0F0134A705D0CAEC20F01FECCB
:1032D0004BF011D0CAEC20F0B7EC4BF0CAEC20F068
:1032E000CAEC20F006DFCAEC20F0CAEC20F0CAECF1
:1032F00020F050EC4BF0CAEC20F0CAEC20F0CAEC05
:1033000020F00F0130AF0CD01BEC7AF0CAEC20F0AB
:10331000CAEC20F0CAEC20F0CAEC20F0CAEC20F095
:103320000F013DA710D00F013D830B01AE6B3BECAD
:103330003BF0CAEC20F0CAEC20F0CAEC20F0CAEC5A
:1033400020F0CAEC20F00F013DA510D00F013D8305
:103350000B01AD6B16EC3CF0CAEC20F0CAEC20F08F
:10336000CAEC20F0CAEC20F0CAEC20F00301FE69A0
:103370000301FE69FF000F0132A336D00F0130AF09
:103380000CD01BEC7AF0CAEC20F0CAEC20F0CAECAE
:1033900020F0CAEC20F0CAEC20F00F013DA710D0BD
:1033A0000F013D830B01AE6B3BEC3BF0CAEC20F010
:1033B000CAEC20F0CAEC20F0CAEC20F0CAEC20F0F5
:1033C0000F013DA510D00F013D830B01AD6B16EC35
:1033D0003CF0CAEC20F0CAEC20F0CAEC20F0CAECB9
:1033E00020F0CAEC20F0FF00DFD61200CAEC20F07B
:1033F000D3EC4BF00301FF6B0A0E0301FF5D05E206
:10340000CAEC20F00301FF2BF7D73FEC4CF0010191
:10341000FC6B0B0E0101FC5D11E20301FF6BF00E72
:103420000301FF5D08E2ADEC0DF00F013EB30CD0DF
:103430000301FF2BF4D70101FC2BEBD70F0129A1CE
:1034400002D054EC56F00ED00F013E93CAEC20F09F
:10345000CAEC20F0CAEC20F0E3EC27F0CAEC20F034
:10346000CAEC20F01200CAEC20F076DCCAEC20F0A6
:10347000CAEC20F0CAEC20F0CAEC20F0CAEC20F034
:103480006BEC4AF00F01309D0001AC6B0001AD6B9D
:103490000001AE6B0F01006B0F01016B0F01336B6D
:1034A0000F01346B0F01356B0F01366B0F0130AF1D
:1034B00064D00101FC6B0B0E0101FC5D5DE20301B8
:1034C000FF6BF00E0301FF5D54E2040012DB0F01FD
:1034D00034AD0DD00401EA6BCAEC20F011EC4CF0D5
:1034E000CAEC20F0CAEC20F0CAEC20F02ED10F017B
:1034F00034A93CD0CAEC20F0E9DC0F0134A705D098
:10350000CAEC20F01FEC4BF02AD0CAEC20F0B7EC4C
:103510004BF0CAEC20F0CAEC20F00001100EA26FB4
:103520000001A36BA2C0F2FCA3C0F3FC1EDDA9EC5A
:103530003EF01F0E0001A35D0AE1FF0E0001A25D37
:1035400006E10001A26B0001A36B00D9FED00001CF
:10355000A22B0001A25102E10001A32BE3D7CAEC88
:1035600020F0CAEC20F0CAEC20F0EFD00301FF2BD2
:10357000A8D70101FC2B9FD7E8D063EC33F0A39AC6
:103580000401F3A704D00401F397B1EC4AF004015D
:10359000F3A504D00401F3951FEC4BF00401F3A94B
:1035A00004D00401F399DFEC4AF00401F3ABCDD071
:1035B0000401F39B0A0E0401EEAF02D0D89003D0B1
:1035C000ED5D000EEE590BE2300E0401ED25020117
:1035D000036F0201140E046F0101040E736F0A0ED3
:1035E0000401EEAF02D0D89003D0ED5D000EEE598D
:1035F0003CE3640E0401EEAF02D0D89003D0ED5D41
:10360000000EEE5932E20201036B0201046B040169
:10361000EF6BF06B0401F0510401EE19E8AE02D03B
:10362000EE3507D0ED510401EF5D0401EE510401C8
:10363000F0590FE20201032B0A0E0201045D04E1BE
:103640000201046B0201032B0401EF2B000EF02397
:10365000E1D7300E02010327300E020104270201D8
:10366000140E056F0101050E736F640E0401EEAFB9
:1036700002D0D89003D0ED5D000EEE593FE3020179
:10368000036B0201046B0201056B0401EF6BF06B2D
:103690000401F0510401EE19E8AE02D0EE3507D076
:1036A000ED510401EF5D0401EE510401F05917E200
:1036B0000201052B0A0E0201055D04E10201056B02
:1036C0000201042B0A0E0201045D04E10201046BF5
:1036D0000201032B0401EF2B000EF023D9D7300E8B
:1036E00002010327300E02010427300E02010527D4
:1036F0000201140E066F0101060E736F0401ED6BDB
:10370000EE6BB7EC4BF00001100EA26F0001A36B43
:10371000A2C0F2FCA3C0F3FC28DCA9EC3EF01F0E13
:103720000001A35D0AE1FF0E0001A25D06E10001B8
:10373000A26B0001A36B0AD808D00001A22B0001E4
:10374000A25102E10001A32BE3D712000C01F36B9D
:103750000C01100EF26F0101F26B200E0101F25DFF
:1037600013E23CEC3EF0F350E66E0101F251EA6ADE
:10377000000FE96E0B0EEA22E552E750EF6E0C01E6
:10378000F22B0101F22BE9D70101F26B080E0101C6
:10379000F25D13E23CEC3EF0F350E66E0101F251B3
:1037A000EA6A200FE96E0B0EEA22E552E750EF6E4F
:1037B0000C01F22B0101F22BE9D70101F26B080E8B
:1037C0000101F25D13E23CEC3EF0F350E66E0101C4
:1037D000F251EA6A280FE96E0B0EEA22E552E75031
:1037E000EF6E0C01F22B0101F22BE9D70101F26B14
:1037F0000F0E0101F25D13E23CEC3EF0F350E66E79
:103800000101F251EA6A300FE96E0B0EEA22E5522D
:10381000E750EF6E0C01F22B0101F22BE9D7010109
:10382000F26B0F0E0101F25D13E23CEC3EF0F3503F
:10383000E66E0101F251EA6A3F0FE96E0B0EEA22D1
:10384000E552E750EF6E0C01F22B0101F22BE9D7A4
:103850000101F26B200E0101F25D13E23CEC3EF03F
:10386000F350E66E0101F251EA6A4E0FE96E0B0E5B
:10387000EA22E552E750EF6E0C01F22B0101F22B28
:10388000E9D70101F26B040E0101F25D13E23CEC99
:103890003EF0F350E66E0101F251EA6A6E0FE96EF6
:1038A0000B0EEA22E552E750EF6E0C01F22B0101FC
:1038B000F22BE9D70101F26B030E0101F25D13E275
:1038C0003CEC3EF0F350E66E0101F251EA6A140F4F
:1038D000E96E0F0EEA22E552E750EF6E0C01F22B73
:1038E0000101F22BE9D7300E0F01145D0CE30F013B
:1038F0001451390804E2410E0F01145D04E30F0175
:10390000145146080AE20F01310E146F0F01320EF6
:10391000156F0F01300E166F33D0300E0F01155D8D
:103920000CE30F011551390804E2410E0F01155D3A
:1039300004E30F01155146080AE20F01310E146F1E
:103940000F01320E156F0F01300E166F19D0300EA9
:103950000F01165D0CE30F011651390804E2410E08
:103960000F01165D04E30F011651460809E20F012D
:10397000310E146F0F01320E156F0F01300E166FDE
:103980000C01890EF26F0101F26B0F0E0101F25D65
:1039900013E23CEC3EF0F350E66E0101F251EA6AAC
:1039A000990FE96E0B0EEA22E552E750EF6E0C011B
:1039B000F22B0101F22BE9D70101F26B040E010198
:1039C000F25D13E23CEC3EF0F350E66E0101F25181
:1039D000EA6AA80FE96E0B0EEA22E552E750EF6E95
:1039E0000C01F22B0101F22BE9D70F013993FF0EE5
:1039F0000B01995D04E0FF0E0B01A85D02E10F01D0
:103A00003983FF0E0B013F5D02E00F0139810F0189
:103A10003DA70DD00F013D830B01AE6B3BEC3BF09E
:103A20000B01AE6B0C01600EF96F22EC0CF00F0174
:103A30003DA50DD00F013D830B01AD6B16EC3CF0A5
:103A40000B01AD6B0C01600EF96F22EC0CF00C0158
:103A5000200EF96F22EC0CF00F0128939DEC45F03D
:103A60000301FF6BA00E0301FF5D0BE20F0128B302
:103A700008D0CC6A2EEC0CF02EEC0CF00301FF2BDE
:103A8000F1D70F0139A11AD00C01200EF96F22ECE9
:103A90000CF00F0128935EEC47F00301FF6BA00EC2
:103AA0000301FF5D0BE20F0128B308D0CC6A2EECB6
:103AB0000CF02EEC0CF00301FF2BF1D70C01200EC3
:103AC000F96F22EC0CF00F012893FFEC45F0030195
:103AD000FF6BA00E0301FF5D0BE20F0128B308D0BE
:103AE000CC6A2EEC0CF02EEC0CF00301FF2BF1D77E
:103AF00012009E929EB249D30301020EFE6F1AEC91
:103B00000CF00F0130BF0ED0D59E0401010EEA6FFC
:103B10000401EA5106E00301020EFE6F1AEC0CF0FC
:103B2000F7D732D328EC7AF00001A06FA0C073F170
:103B30000001A05101E128D3600EE66E000EE66E92
:103B40005EEC7AF0E552E5520101F96B0001A051FB
:103B50000101F95D01E303D30101F951EA6A600F44
:103B6000E96E000EEA22EFCFFEF60101F951EA6A92
:103B7000600FE96E000EEA22EF50E66E0101F95186
:103B8000EA6A010FE96E020EEA22E552E750EF6E93
:103B90000F0133B11DD03A0E0601FE5D18E10F0191
:103BA000010E336F0F01346B0001AA6B0001AB6B88
:103BB0000001A56B0001A8690001A96B0D01FE6B56
:103BC0000F01002B0F01005102E10F01012BC1D2A7
:103BD0000F0135AF1BD10F0136B10BD00D0E060111
:103BE000FE5D04E00F01348DD1D203D00F01368188
:103BF000B0D20F0136B30BD00A0E0601FE5D04E011
:103C00000F01348DC3D203D00F013683A2D20F012E
:103C100035B107D0430E0601FE5D02E10F0135818B
:103C2000F4D00F0135B30BD02F0E0601FE5D03E17A
:103C30000F01358303D00F01348DA8D2E6D00F01D8
:103C400035BD4CD00D0E0601FE5D03E10F01358D33
:103C500080D20F0135B514D00601FE512F080CE2B9
:103C60003A0E0601FE5D08E2300E0601FE5D00011F
:103C7000AC6F0F01358503D00F01348D87D22DD065
:103C80000F0135B714D00601FE512F080CE23A0E91
:103C90000601FE5D08E2300E0601FE5D0001AD6F1B
:103CA0000F01358703D00F01348D70D216D00F016C
:103CB00035B913D00601FE512F080CE23A0E060169
:103CC000FE5D08E2300E0601FE5D0001AE6F0F01E1
:103CD000358903D00F01348D59D297D00A0E0601D1
:103CE000FE5D01E08FD00001AA6B0001AB6B300ECE
:103CF0000001AC250201036F300E0001AD25020169
:103D0000046F300E0001AE250201056F0F0135A9C9
:103D100043D00001AC51000812E2AAC0A5F0640E25
:103D20000001AA250001AA6F0001AA510001D88054
:103D3000A55502E20001AB2B0001AC07EAD7000158
:103D4000AD51000812E2AAC0A5F00A0E0001AA2592
:103D50000001AA6F0001AA510001D880A55502E216
:103D60000001AB2B0001AD07EAD7AAC0A5F0000106
:103D7000AA510001AE250001AA6F0001AA5100015D
:103D8000D880A55502E20001AB2B0201140E066F8C
:103D90000101060E736F24D00F0135A712D00A0E51
:103DA0000001AC03F3CFAAF00001AA510001AD2538
:103DB0000001AA6F0201140E056F0101050E736F59
:103DC0000FD00F0135A509D0ACC0AAF00201140E26
:103DD000046F0101040E736F03D00F01348DD6D12F
:103DE0000001AA510F01005D09E10001AB510F0173
:103DF000015D04E10F013489C9D103D00F01348D75
:103E0000C5D103D00F01348DC1D1A3D10D0E060150
:103E1000FE5D25E10001A80508E10F010F01345105
:103E2000800B03E00F01348B94D1020E0001A85DDA
:103E300008E10F010F013451800B03E00F01348BB7
:103E400088D10001A85108E10F010F013451800B06
:103E500003E00F01348B7DD10F01348D97D10A0E11
:103E60000601FE5D25E10001A80508E10F010F0133
:103E70003451200B03E00F01358F6BD1020E00018E
:103E8000A85D08E10F010F013451200B03E00F0181
:103E900033915FD10001A85108E10F010F013451A6
:103EA000200B03E00F01339154D10F01348D6ED1FB
:103EB0000F0134BB4BD10F0133B318D03A0E0601BA
:103EC000FE5D06E2300E0601FE5D0001AA6F05D020
:103ED000370E0601FE5D0001AA6F0001AA39F00B42
:103EE0000001AA6F0F01338334D117D03A0E0601B7
:103EF000FE5D06E2300E0601FE5D0001AB6F05D0EF
:103F0000370E0601FE5D0001AB6F0001AA510001F2
:103F1000AB250001AA6F0F0133930F0133B507D012
:103F2000AAC0A5F00F013385A5C0A9F012D10F01D9
:103F300033B70BD0AAC0A6F00F0133870001A951F7
:103F40000001A6250001A96F04D10F0133B90BD0E0
:103F5000AAC0A7F00F0133890001A9510001A725CC
:103F60000001A96FF6D00F0133BB0BD0AAC0A8F097
:103F70000F01338B0001A9510001A8250001A96F91
:103F8000E8D00F0133BD46D00F01338D0001A805E5
:103F90000BE1FF0E0001AA5D04E10F01348FD9D0BF
:103FA00002D00F01348DF2D0020E0001A85D0DE1A8
:103FB0000001AA5103E00F01348DE8D00001A9519E
:103FC0000001AA250001A96FC4D00001A8511FE17A
:103FD0000001A55104E10F01348DD8D017D00001A4
:103FE000A6511F0803E20F01348DD0D00001A95162
:103FF0000001AA250001A96F0001A507A7C0A2F032
:10400000A6C0A3F0AAC0A4F0EDEC16F0A2D00F0158
:10401000348DBCD00F0133BF2FD00F01338F020E70
:104020000001A85D0DE10001AA5103E00F01348DEC
:10403000ADD00001A9510001AA250001A96F89D0C6
:104040000001A85116E10001A55104E10F01348DD2
:104050009DD00ED00001A9510001AA250001A96F31
:104060000001A5070001A22BAAC0A4F0EDEC16F0F8
:1040700070D00F01348D8AD00F0134B33ED00F01C0
:104080003483020E0001A85D10E10001A951000176
:10409000AA250001A96F0001A95104E10F01348F85
:1040A00058D003D00F01348D71D00001A85122E106
:1040B0000001A55110E10001A9510001AA2500014C
:1040C000A96F0001A95103E10F01348F03D00F0143
:1040D000348D5CD00ED00001A9510001AA25000149
:1040E000A96F0001A5070001A22BAAC0A4F0EDEC66
:1040F00016F02FD00F01348D49D00001A85122E1D4
:104100000001A55110E10001A9510001AA250001FB
:10411000A96F0001A95103E10F01348F03D00F01F2
:10412000348D34D00ED00001A9510001AA25000120
:10413000A96F0001A5070001A22BAAC0A4F0EDEC15
:1041400016F007D00F01348D21D003D00F01348D2C
:104150001DD00301020EFE6F0101F92BF7D4D7EC3D
:1041600032F00101F96B400E0101F95D0BE2010132
:10417000F951EA6A600FE96E000EEA22EF6A010166
:10418000F92BF1D70001A06BB5D49E920301020E6A
:10419000FE6F12009E920C01FB6B960E0C01FB5DF4
:1041A0000CE29EB206D00301020EFE6F1AEC0CF078
:1041B000F8D79E920C01FB2BF0D712009E929EB274
:1041C000DCEF27F00301020EFE6F1AEC0CF00F017A
:1041D00030BF66D39CA207D09C980301020EFE6FED
:1041E0001AEC0CF09C88A4AA5AD3AACFFEF6A49A83
:1041F0000F0133B11DD03A0E0601FE5D18E10F012B
:10420000010E336F0F01346B0001AA6B0001AB6B21
:104210000001A56B0001A8690001A96B0D01FE6BEF
:104220000F01002B0F01005102E10F01012B37D3C9
:104230000F0135AF7AD10F0135B107D0430E06011A
:10424000FE5D02E10F0135816ED10F0135B30AD059
:104250002F0E0601FE5D03E10F01358302D00F0131
:10426000348D61D10F0135BD63D00D0E0601FE5DA9
:1042700004E10F01358DDDEF27F00F0135B513D0C7
:104280000601FE512F080CE23A0E0601FE5D08E21F
:10429000300E0601FE5D0001AC6F0F01358502D0C6
:1042A0000F01348D44D00F0135B713D00601FE51F4
:1042B0002F080CE23A0E0601FE5D08E2300E060100
:1042C000FE5D0001AD6F0F01358702D00F01348D07
:1042D0002ED00F0135B913D00601FE512F080CE284
:1042E0003A0E0601FE5D08E2300E0601FE5D000199
:1042F000AE6F0F01358902D00F01348D18D00F0138
:1043000035BB13D00601FE512F080CE23A0E060110
:10431000FE5D08E2300E0601FE5D0001AF6F0F0189
:10432000358B02D00F01348D02D00F01348DFBD0BC
:104330000A0E0601FE5D01E0F4D00001AA6B000147
:10434000AB6B300E0001AC250201036F300E000193
:10435000AD250201046F300E0001AE250201056F8C
:10436000300E0001AF250201066F0F0135AB5ED0A4
:104370000001AC51000817E2AAC0A5F0E80E000148
:10438000AA250001AA6F0001AA510001D880A555F5
:1043900002E20001AB2B030E0001AB250001AB6F65
:1043A0000001AC07E5D70001AD51000812E2AAC038
:1043B000A5F0640E0001AA250001AA6F0001AA5110
:1043C0000001D880A55502E20001AB2B0001AD072A
:1043D000EAD70001AE51000812E2AAC0A5F00A0E09
:1043E0000001AA250001AA6F0001AA510001D8808E
:1043F000A55502E20001AB2B0001AE07EAD7AAC027
:10440000A5F00001AA510001AF250001AA6F00012B
:10441000AA510001D880A55502E20001AB2B020190
:10442000140E076F0101070E736F6BD00F0135A9D2
:1044300043D00001AC51000812E2AAC0A5F0640EFE
:104440000001AA250001AA6F0001AA510001D8802D
:10445000A55502E20001AB2B0001AC07EAD7000131
:10446000AD51000812E2AAC0A5F00A0E0001AA256B
:104470000001AA6F0001AA510001D880A55502E2EF
:104480000001AB2B0001AD07EAD7AAC0A5F00001DF
:10449000AA510001AE250001AA6F0001AA51000136
:1044A000D880A55502E20001AB2B0201140E066F65
:1044B0000101060E736F25D00F0135A712D00A0E29
:1044C0000001AC03F3CFAAF00001AA510001AD2511
:1044D0000001AA6F0201140E056F0101050E736F32
:1044E00010D00F0135A509D0ACC0AAF00201140EFE
:1044F000046F0101040E736F04D00F01348DDDEFE2
:1045000027F00001AA510F01005D08E10001AB5145
:104510000F01015D03E10F01348902D00F01348DD9
:1045200002D00F01348DDDEF27F00D0E0601FE5D88
:1045300029E10001A80509E10F010F013451800BA9
:1045400004E00F01348BDDEF27F0040E0001A85DBD
:1045500009E10F010F013451800B04E00F01348B8E
:10456000DDEF27F00001A85109E10F010F013451DF
:10457000800B04E00F01348BDDEF27F00F01348D49
:10458000DDEF27F00A0E0601FE5D29E10001A80516
:1045900009E10F010F013451200B04E00F01358FA9
:1045A000DDEF27F0040E0001A85D09E10F010F0106
:1045B0003451200B04E00F013391DDEF27F00001AF
:1045C000A85109E10F010F013451200B04E00F0144
:1045D0003391DDEF27F00F01348DDDEF27F00F0170
:1045E00034BB5AD10F0133B319D03A0E0601FE5D28
:1045F00006E2300E0601FE5D0001AA6F05D0370EFF
:104600000601FE5D0001AA6F0001AA39F00B00014E
:10461000AA6F0F013383DDEF27F017D03A0E0601A2
:10462000FE5D06E2300E0601FE5D0001AB6F05D0B7
:10463000370E0601FE5D0001AB6F0001AA510001BB
:10464000AB250001AA6F0F0133930F0133B508D0DA
:10465000AAC0A5F00F013385A5C0A9F0DDEF27F0B2
:104660000F0133B70CD0AAC0A6F00F0133870001A9
:10467000A9510001A6250001A96FDDEF27F00F0168
:1046800033B90CD0AAC0A7F00F0133890001A9519A
:104690000001A7250001A96FDDEF27F00F0133BB53
:1046A0000CD0AAC0A8F00F01338B0001A951000162
:1046B000A8250001A96FDDEF27F00F0133BD4BD016
:1046C0000F01338D0001A8050BE1FF0E0001AA5D6B
:1046D00003E10F01348F02D00F01348DDDEF27F09D
:1046E000040E0001A85D0DE10001AA5102E00F01D6
:1046F000348D0001A9510001AA250001A96FDDEF49
:1047000027F00001A85123E10001A55103E10F01A9
:10471000348D1BD00F0130AD08D00001A651F70831
:1047200004E20F013485DDEF27F00001A9510001FB
:10473000AA250001A96F0001A507A7C0A2F0A6C085
:10474000A3F0AAC0A4F0EDEC16F0DDEF27F00F0106
:10475000348DDDEF27F00F0133BF37D00F01338FDA
:10476000040E0001A85D14E10001AA51010803E252
:104770000F01348D05D00001AA0502E10F01308D33
:104780000001A9510001AA250001A96FDDEF27F062
:104790000001A85116E10001A55103E10F01348D7C
:1047A0000ED00001A9510001AA250001A96F000146
:1047B000A5070001A22BAAC0A4F0EDEC16F0DDEFD6
:1047C00027F00F01348DDDEF27F00F0134B33CD01B
:1047D0000F013483040E0001A85D0FE10001A9510F
:1047E0000001AA250001A96F0001A95103E10F01F1
:1047F000348F02D00F01348DE0D30001A85121E1A4
:104800000001A5510FE10001A9510001AA250001F5
:10481000A96F0001A95103E10F01348F02D00F01EC
:10482000348D0ED00001A9510001AA250001A96F05
:104830000001A5070001A22BAAC0A4F0EDEC16F020
:10484000BCD30F01348DB9D30001A85121E100017F
:10485000A5510FE10001A9510001AA250001A96F8E
:104860000001A95103E10F01348F02D00F01348DF3
:104870000ED00001A9510001AA250001A96F000175
:10488000A5070001A22BAAC0A4F0EDEC16F095D369
:104890000F01348D92D303D00F01348D8ED38AD380
:1048A00028EC7AF00001A06F0001A05101E182D351
:1048B000600EE66E000EE66E5EEC7AF0E552E552B2
:1048C0000101F96B0001A0510101F95D01E35FD322
:1048D0000101F951EA6A600FE96E000EEA22EFCF9A
:1048E000FEF60F0133B11DD03A0E0601FE5D18E150
:1048F0000F01010E336F0F01346B0001AA6B000131
:10490000AB6B0001A56B0001A8690001A96B0D014B
:10491000FE6B0F01002B0F01005102E10F01012B73
:1049200030D30F0135AF80D10F0135B107D0430E21
:104930000601FE5D02E10F01358175D10F0135B32E
:104940000BD02F0E0601FE5D03E10F01358303D06E
:104950000F01348D32D367D10F0135BD67D00D0EF5
:104960000601FE5D03E10F01358D0BD30F0135B557
:1049700014D00601FE512F080CE23A0E0601FE5D2E
:1049800008E2300E0601FE5D0001AC6F0F013585B7
:1049900003D00F01348D11D348D00F0135B714D097
:1049A0000601FE512F080CE23A0E0601FE5D08E2F8
:1049B000300E0601FE5D0001AD6F0F01358703D09B
:1049C0000F01348DFAD231D00F0135B914D0060160
:1049D000FE512F080CE23A0E0601FE5D08E2300E91
:1049E0000601FE5D0001AE6F0F01358903D00F0196
:1049F000348DE3D21AD00F0135BB14D00601FE511D
:104A00002F080CE23A0E0601FE5D08E2300E0601A8
:104A1000FE5D0001AF6F0F01358B03D00F01348DA8
:104A2000CCD203D00F01348DC8D2FDD00A0E0601BE
:104A3000FE5D01E0F5D00001AA6B0001AB6B300E0A
:104A40000001AC250201036F300E0001AD2502010B
:104A5000046F300E0001AE250201056F300E00011B
:104A6000AF250201066F0F0135AB5ED00001AC51DE
:104A7000000817E2AAC0A5F0E80E0001AA2500016F
:104A8000AA6F0001AA510001D880A55502E20001D9
:104A9000AB2B030E0001AB250001AB6F0001AC078F
:104AA000E5D70001AD51000812E2AAC0A5F0640EDE
:104AB0000001AA250001AA6F0001AA510001D880B7
:104AC000A55502E20001AB2B0001AD07EAD70001BA
:104AD000AE51000812E2AAC0A5F00A0E0001AA25F4
:104AE0000001AA6F0001AA510001D880A55502E279
:104AF0000001AB2B0001AE07EAD7AAC0A5F0000168
:104B0000AA510001AF250001AA6F0001AA510001BE
:104B1000D880A55502E20001AB2B0201140E076FED
:104B20000101070E736F6AD00F0135A943D0000150
:104B3000AC51000812E2AAC0A5F0640E0001AA253B
:104B40000001AA6F0001AA510001D880A55502E218
:104B50000001AB2B0001AC07EAD70001AD51000802
:104B600012E2AAC0A5F00A0E0001AA250001AA6F50
:104B70000001AA510001D880A55502E20001AB2B2B
:104B80000001AD07EAD7AAC0A5F00001AA510001B3
:104B9000AE250001AA6F0001AA510001D880A555D9
:104BA00002E20001AB2B0201140E066F0101060E9A
:104BB000736F24D00F0135A712D00A0E0001AC0389
:104BC000F3CFAAF00001AA510001AD250001AA6FA0
:104BD0000201140E056F0101050E736F0FD00F0156
:104BE00035A509D0ACC0AAF00201140E046F010172
:104BF000040E736F03D00F01348DDFD10001AA5171
:104C00000F01005D09E10001AB510F01015D04E1FD
:104C10000F013489D2D103D00F01348DCED103D00E
:104C20000F01348DCAD1ADD10D0E0601FE5D25E117
:104C30000001A80508E10F010F013451800B03E0CA
:104C40000F01348B9ED1040E0001A85D08E10F0115
:104C50000F013451800B03E00F01348B92D100011E
:104C6000A85108E10F010F013451800B03E00F013F
:104C7000348B87D10F01348DA0D10A0E0601FE5D61
:104C800025E10001A80508E10F010F013451200BB7
:104C900003E00F01358F75D1040E0001A85D08E116
:104CA0000F010F013451200B03E00F01339169D143
:104CB0000001A85108E10F010F013451200B03E05E
:104CC0000F0133915ED10F01348D77D10F0134BBC9
:104CD00055D10F0133B318D03A0E0601FE5D06E23E
:104CE000300E0601FE5D0001AA6F05D0370E0601E9
:104CF000FE5D0001AA6F0001AA39F00B0001AA6F46
:104D00000F0133833ED117D03A0E0601FE5D06E255
:104D1000300E0601FE5D0001AB6F05D0370E0601B7
:104D2000FE5D0001AB6F0001AA510001AB2500013F
:104D3000AA6F0F0133930F0133B507D0AAC0A5F0B6
:104D40000F013385A5C0A9F01CD10F0133B70BD0DB
:104D5000AAC0A6F00F0133870001A9510001A625C2
:104D60000001A96F0ED10F0133B90BD0AAC0A7F073
:104D70000F0133890001A9510001A7250001A96F86
:104D800000D10F0133BB0BD0AAC0A8F00F01338BA9
:104D90000001A9510001A8250001A96FF2D00F015F
:104DA00033BD49D00F01338D0001A8050BE1FF0E83
:104DB0000001AA5D04E10F01348FE3D002D00F019E
:104DC000348DFBD0040E0001A85D0DE10001AA5155
:104DD00003E00F01348DF1D00001A9510001AA2593
:104DE0000001A96FCED00001A85122E10001A55118
:104DF00004E10F01348DE1D01AD00F0130AD07D09E
:104E00000001A651F70803E20F013485D6D0000156
:104E1000A9510001AA250001A96F0001A507A7C09B
:104E2000A2F0A6C0A3F0AAC0A4F0EDEC16F0A9D0A1
:104E30000F01348DC2D00F0133BF36D00F01338F35
:104E4000040E0001A85D14E10001AA51010804E26A
:104E50000F01348DB2D005D00001AA0502E10F0187
:104E6000308D0001A9510001AA250001A96F89D048
:104E70000001A85116E10001A55104E10F01348D94
:104E80009CD00ED00001A9510001AA250001A96FF4
:104E90000001A5070001A22BAAC0A4F0EDEC16F0BA
:104EA00070D00F01348D89D00F0134B33ED00F0183
:104EB0003483040E0001A85D10E10001A951000136
:104EC000AA250001A96F0001A95104E10F01348F47
:104ED00058D003D00F01348D70D00001A85122E1C9
:104EE0000001A55110E10001A9510001AA2500010E
:104EF000A96F0001A95103E10F01348F03D00F0105
:104F0000348D5BD00ED00001A9510001AA2500010B
:104F1000A96F0001A5070001A22BAAC0A4F0EDEC27
:104F200016F02FD00F01348D48D00001A85122E196
:104F30000001A55110E10001A9510001AA250001BD
:104F4000A96F0001A95103E10F01348F03D00F01B4
:104F5000348D33D00ED00001A9510001AA250001E3
:104F6000A96F0001A5070001A22BAAC0A4F0EDECD7
:104F700016F007D00F01348D20D003D00F01348DEF
:104F80001CD00301020EFE6F0101F92B9BD401011D
:104F9000F96B400E0101F95D0BE20101F951EA6A7A
:104FA000600FE96E000EEA22EF6A0101F92BF1D7DA
:104FB0000001A06BDFEF20F09E920301020EFE6F56
:104FC0001AEC0CF012000201230E016F0201340EE4
:104FD000026F02013A0E036F0201300E046F0201EC
:104FE000320E056F0201300E066F0201300E076FA0
:104FF0000201300E086F0201300E096F0201300EFF
:105000000A6F0201320E0B6F0201300E0C6F0201AB
:10501000300E0D6F0201300E0E6F0201300E0F6F59
:105020000201460E106F0201430E116F0201140EB1
:10503000126F0101120E736F0F013E970F0130BF07
:1050400003D0D7EC32F024D042EC7AF000090CE126
:1050500073C1E6FF010EE66E020EE66E4AEC7AF0D0
:10506000E552E552E55214D00F013EB70FD00301CF
:10507000FF6B050E0301FF5D05E2CAEC20F00301A2
:10508000FF2BF7D70F013E87DFD702D0B8EF2DF007
:105090000B01010E966F0B01976B0B01986B0C01C6
:1050A000100EF26F0C01F36B3CEC3EF0F3CF79FB8A
:1050B0000C01F22B3CEC3EF0F3CF7AFB0C01F22B0F
:1050C0003CEC3EF0F3CF7BFB0C01F22B3CEC3EF0D2
:1050D000F3CF7CFB0C01F22B3CEC3EF0F3CF7DFBDD
:1050E0000C01F22B3CEC3EF0F3CF7EFB0C01F22BDB
:1050F0003CEC3EF0F3CF7FFB0C01F22B3CEC3EF09E
:10510000F3CF80FB0C01F22B3CEC3EF0F3CF81FBA4
:105110000C01F22B3CEC3EF0F3CF82FB0C01F22BA6
:105120003CEC3EF0F3CF83FB0C01F22B3CEC3EF069
:10513000F3CF84FB0C01F22B3CEC3EF0F3CF85FB6C
:105140000C01F22B3CEC3EF0F3CF86FB0C01F22B72
:105150003CEC3EF0F3CF87FB0C01F22B3CEC3EF035
:10516000F3CF88FB0101F26B100E0101F25D0EE23C
:105170000101F251EA6A790FE96E0B0EEA22EF5053
:10518000FF0801E015D00101F22BEED70C01F22B44
:105190001F0E0C01F35D06E1F00E0C01F25D02E161
:1051A000CFEF2CF00C01F25102E10C01F32B7CD774
:1051B000240E0B01795D12E10101010EF26F100E58
:1051C0000101F25D0BE20101F251EA6A790FE96E29
:1051D0000B0EEA22EF680101F22BF1D70201230E38
:1051E000016F0201340E026F02013A0E036F0201D9
:1051F000310E046F0201300E056FF00E0C01F31535
:105200000B01946F0B0194390F0B0B01946F0A0E75
:105210000B01945D06E2300E0B0194250201066F2E
:1052200005D0370E0B0194250201066F0F0E0C01FD
:10523000F3150B01946F0A0E0B01945D06E2300E1C
:105240000B0194250201076F05D0370E0B01942541
:105250000201076FF00E0C01F2150B01946F0B01A8
:1052600094390F0B0B01946F0A0E0B01945D06E24B
:10527000300E0B0194250201086F05D0370E0B018B
:1052800094250201086F0201300E096F0201300EF1
:105290000A6F0201300E0B6FF00E0B0179150B0136
:1052A000946F0B0194390F0B0B01946F0A0E0B01D5
:1052B000945D06E2300E0B01942502010C6F05D0BF
:1052C000370E0B01942502010C6F0F0E0B0179159F
:1052D0000B01946F0A0E0B01945D06E2300E0B0178
:1052E000942502010D6F05D0370E0B0194250201A4
:1052F0000D6FF00E0B017A150B01946F0B019439B1
:105300000F0B0B01946F0A0E0B01945D06E2300E39
:105310000B01942502010E6F05D0370E0B01942569
:1053200002010E6F0F0E0B017A150B01946F0A0E1E
:105330000B01945D06E2300E0B01942502010F6F04
:1053400005D0370E0B01942502010F6FF00E0B01F3
:105350007B150B01946F0B0194390F0B0B01946FAC
:105360000A0E0B01945D06E2300E0B01942502013A
:10537000106F05D0370E0B0194250201106F0F0E30
:105380000B017B150B01946F0A0E0B01945D06E275
:10539000300E0B0194250201116F05D0370E0B0161
:1053A00094250201116FF00E0B017C150B01946F17
:1053B0000B0194390F0B0B01946F0A0E0B01945DD6
:1053C00006E2300E0B0194250201126F05D0370E54
:1053D0000B0194250201126F0F0E0B017C150B01BE
:1053E000946F0A0E0B01945D06E2300E0B019425BA
:1053F0000201136F05D0370E0B0194250201136FC4
:10540000F00E0B017D150B01946F0B0194390F0BFE
:105410000B01946F0A0E0B01945D06E2300E0B0136
:1054200094250201146F05D0370E0B01942502015B
:10543000146F0F0E0B017D150B01946F0A0E0B01FB
:10544000945D06E2300E0B0194250201156F05D024
:10545000370E0B0194250201156FF00E0B017E151E
:105460000B01946F0B0194390F0B0B01946F0A0E13
:105470000B01945D06E2300E0B0194250201166FBC
:1054800005D0370E0B0194250201166F0F0E0B018C
:105490007E150B01946F0A0E0B01945D06E2300E2F
:1054A0000B0194250201176F05D0370E0B019425CF
:1054B0000201176FF00E0B017F150B01946F0B01AA
:1054C00094390F0B0B01946F0A0E0B01945D06E2E9
:1054D000300E0B0194250201186F05D0370E0B0119
:1054E00094250201186F0F0E0B017F150B01946FAD
:1054F0000A0E0B01945D06E2300E0B0194250201A9
:10550000196F05D0370E0B0194250201196FF00EAB
:105510000B0180150B01946F0B0194390F0B0B01DC
:10552000946F0A0E0B01945D06E2300E0B01942578
:1055300002011A6F05D0370E0B01942502011A6F74
:105540000F0E0B0180150B01946F0A0E0B01945D79
:1055500006E2300E0B01942502011B6F05D0370EB9
:105560000B01942502011B6FF00E0B0181150B013D
:10557000946F0B0194390F0B0B01946F0A0E0B0102
:10558000945D06E2300E0B01942502011C6F05D0DC
:10559000370E0B01942502011C6F0F0E0B018115B4
:1055A0000B01946F0A0E0B01945D06E2300E0B01A5
:1055B000942502011D6F05D0370E0B0194250201C1
:1055C0001D6FF00E0B0182150B01946F0B019439C6
:1055D0000F0B0B01946F0A0E0B01945D06E2300E67
:1055E0000B01942502011E6F05D0370E0B01942587
:1055F00002011E6F0F0E0B0182150B01946F0A0E34
:105600000B01945D06E2300E0B01942502011F6F21
:1056100005D0370E0B01942502011F6FF00E0B0110
:1056200083150B01946F0B0194390F0B0B01946FD1
:105630000A0E0B01945D06E2300E0B019425020167
:10564000206F05D0370E0B0194250201206F0F0E3D
:105650000B0183150B01946F0A0E0B01945D06E29A
:10566000300E0B0194250201216F05D0370E0B017E
:1056700094250201216FF00E0B0184150B01946F2C
:105680000B0194390F0B0B01946F0A0E0B01945D03
:1056900006E2300E0B0194250201226F05D0370E71
:1056A0000B0194250201226F0F0E0B0184150B01D3
:1056B000946F0A0E0B01945D06E2300E0B019425E7
:1056C0000201236F05D0370E0B0194250201236FD1
:1056D000F00E0B0185150B01946F0B0194390F0B24
:1056E0000B01946F0A0E0B01945D06E2300E0B0164
:1056F00094250201246F05D0370E0B019425020179
:10570000246F0F0E0B0185150B01946F0A0E0B0110
:10571000945D06E2300E0B0194250201256F05D041
:10572000370E0B0194250201256FF00E0B01861533
:105730000B01946F0B0194390F0B0B01946F0A0E40
:105740000B01945D06E2300E0B0194250201266FD9
:1057500005D0370E0B0194250201266F0F0E0B01A9
:1057600086150B01946F0A0E0B01945D06E2300E54
:105770000B0194250201276F05D0370E0B019425EC
:105780000201276FF00E0B0187150B01946F0B01BF
:1057900094390F0B0B01946F0A0E0B01945D06E216
:1057A000300E0B0194250201286F05D0370E0B0136
:1057B00094250201286F0F0E0B0187150B01946FC2
:1057C0000A0E0B01945D06E2300E0B0194250201D6
:1057D000296F05D0370E0B0194250201296FF00EB9
:1057E0000B0188150B01946F0B0194390F0B0B0102
:1057F000946F0A0E0B01945D06E2300E0B019425A6
:1058000002012A6F05D0370E0B01942502012A6F81
:105810000F0E0B0188150B01946F0A0E0B01945D9E
:1058200006E2300E0B01942502012B6F05D0370ED6
:105830000B01942502012B6FF00E0C01F2150B01E8
:10584000946F100E0B0194250B01946F0B01945172
:105850000C01F3250B01946F0101F26B100E010195
:10586000F25D0FE20101F251EA6A790FE96E0B0E67
:10587000EA22EF500B0194250B01946F0101F22BEA
:10588000EDD70B019429E86C0B01956F0B01952B5B
:10589000F00E0B0195150B01946F0B0194390F0B52
:1058A0000B01946F0A0E0B01945D06E2300E0B01A2
:1058B000942502012C6F05D0370E0B0194250201AF
:1058C0002C6F0F0E0B0195150B01946F0A0E0B0137
:1058D000945D06E2300E0B01942502012D6F05D078
:1058E000370E0B01942502012D6F0201140E2E6F4D
:1058F00001012E0E736F0F013E970F0130BF03D0D1
:10590000D7EC32F023D042EC7AF000090CE173C1FD
:10591000E6FF010EE66E020EE66E4AEC7AF0E55204
:10592000E552E55213D00F013EB70FD00301FF6BD4
:10593000050E0301FF5D05E2CAEC20F00301FF2B19
:10594000F7D70F013E87DFD701D012D10B01962B7D
:105950000A0E0B01965D0CE10B01966B0B01972B68
:105960000A0E0B01975D04E10B01976B0B01982B5D
:10597000240E0B01795D01E112D00C01F22B1F0EF8
:105980000C01F35D05E1F00E0C01F25D01E107D0C1
:105990000C01F25102E10C01F32B54EF28F003014A
:1059A000FF6B0A0E0301FF5D05E2CAEC20F0030164
:1059B000FF2BF7D70201230E016F0201340E026F95
:1059C00002013A0E036F0201300E046F0201300E25
:1059D000056F0201300E066F0201300E076F0201E3
:1059E000300E086F0201300E096F0201300E0A6F8F
:1059F0000201310E0B6F0201460E0C6F0201460EC2
:105A00000D6F0201140E0E6F01010E0E736F0F0168
:105A10003E970F0130BF03D0D7EC32F023D042ECD9
:105A20007AF000090CE173C1E6FF010EE66E020E8A
:105A3000E66E4AEC7AF0E552E552E55213D00F01DA
:105A40003EB70FD00301FF6B050E0301FF5D05E2BA
:105A5000CAEC20F00301FF2BF7D70F013E87EFD7E9
:105A600001D086D00B01962B0A0E0B01965D0CE13E
:105A70000B01966B0B01972B0A0E0B01975D04E14E
:105A80000B01976B0B01982B0301FF6B0A0E0301AF
:105A9000FF5D05E2CAEC20F00301FF2BF7D70B01F5
:105AA000985116E0300E0B0198250201036F300E5D
:105AB0000B0197250201046F300E0B0196250201A0
:105AC000056F0201140E066F0101060E736F1FD0E1
:105AD0000B01975111E0300E0B0197250201036F66
:105AE000300E0B0196250201046F0201140E056FA2
:105AF0000101050E736F0BD0300E0B0196250201CC
:105B0000036F0201140E046F0101040E736F020192
:105B1000430E016F02012F0E026F0F013E970F011E
:105B200030BF03D0D7EC32F023D042EC7AF000093A
:105B30000CE173C1E6FF010EE66E020EE66E4AEC62
:105B40007AF0E552E552E55213D00F013EB70FD07F
:105B50000301FF6B050E0301FF5D05E2CAEC20F0B7
:105B60000301FF2BF7D70F013E87DFD701D000D00D
:105B70001200D9CFE6FFE1CFD9FFE652DF6AFE0E71
:105B8000DF5C13E2DF50EA6A000FE96E050EEA22DD
:105B9000EF5009E1DF50EA6A000FE96E050EEA22D4
:105BA000FEC5EFFF02D0DF2AEAD7E552E552E7CF84
:105BB000D9FF1200D9CFE6FFE1CFD9FFE652FE0EA2
:105BC0000601FF5D0CE00601FF51EA6A000FE96E75
:105BD000060EEA22FEC6EFFF0601FF2B11D0DF6A98
:105BE000FE0EDF5C09E2DF50EA6A000FE96E060E86
:105BF000EA22EF6ADF2AF4D70F0129870601FF6B3B
:105C0000E552E552E7CFD9FF1200D9CFE6FFE1CF49
:105C1000D9FFE652DF6A100EDF5C13E2DF50EA6A5A
:105C20002B0FE96E010EEA22EF5009E1DF50EA6A1C
:105C30002B0FE96E010EEA223BC1EFFF05D0DF2AF0
:105C4000EAD707D83BC13AF1E552E552E7CFD9FF91
:105C50001200D9CFE6FFE1CFD9FFE652DF6A0F0E7F
:105C6000DF5C13E2DF28EA6A2B0FE96E010EEA22FD
:105C7000EF50E66EDF50EA6A2B0FE96E010EEA2262
:105C8000E552E750EF6EDF2AEAD701013A6BE552A1
:105C9000E552E7CFD9FF1200D9CFE6FFE1CFD9FF18
:105CA000E652DF6A280EDF5C1FE2DF50E824EA6A72
:105CB0007C0FE96E010EEA22EF5014E1DF50E82478
:105CC000EA6A7C0FE96E010EEA227AC1EFFFDF502B
:105CD000E824010FEA6A7C0FE96E010EEA227BC11B
:105CE000EFFF02D0DF2ADED7E552E552E7CFD9FF3A
:105CF0001200D9CFE6FFE1CFD9FFE652DF6A4E0EA0
:105D0000DF5C14E2020EDF24EA6A7C0FE96E010E0A
:105D1000EA22EF50E66EDF50EA6A7C0FE96E010E70
:105D2000EA22E552E750EF6EDF2AE9D70101CA6B9C
:105D30000101CB6BE552E552E7CFD9FF1200D9CF75
:105D4000E6FFE1CFD9FFE652DF6AFE0EDF5C13E229
:105D5000DF50EA6A000FE96E060EEA22EF50E66EA7
:105D6000DF50EA6A000FE96E0D0EEA22E552E750B5
:105D7000EF6EDF2AEAD7E552E552E7CFD9FF1200EE
:105D8000E8C1E7F1100E0101E75D24E2100E010108
:105D9000E703F3CFE4F10101E56B100E0101E55DCE
:105DA00018E20101E4510101E525EA6A000FE96EFC
:105DB000070EEA22EF50E66E0101E551EA6A000F94
:105DC000E96E010EEA22E552E750EF6E0101E52B84
:105DD000E4D792D00101E7510F082DE2200E010116
:105DE000E75D29E2100E0101E75D0101E76F100E8A
:105DF0000101E703F3CFE4F10101E56B100E0101AE
:105E0000E55D18E20101E4510101E525EA6A000FB0
:105E1000E96E080EEA22EF50E66E0101E551EA6AEA
:105E2000000FE96E010EEA22E552E750EF6E010124
:105E3000E52BE4D761D00101E7511F082DE2300EB8
:105E40000101E75D29E2200E0101E75D0101E76F35
:105E5000100E0101E703F3CFE4F10101E56B100E31
:105E60000101E55D18E20101E4510101E525EA6A5D
:105E7000000FE96E090EEA22EF50E66E0101E551CE
:105E8000EA6A000FE96E010EEA22E552E750EF6E72
:105E90000101E52BE4D730D00101E7512F082CE2B6
:105EA000400E0101E75D28E2300E0101E75D0101CE
:105EB000E76F100E0101E703F3CFE4F10101E56B99
:105EC000100E0101E55D18E20101E4510101E52533
:105ED000EA6A000FE96E0A0EEA22EF50E66E01014F
:105EE000E551EA6A000FE96E010EEA22E552E75039
:105EF000EF6E0101E52BE4D71200E6C1E7F1100EC9
:105F00000101E75D24E2100E0101E703F3CFE4F1A4
:105F10000101E56B100E0101E55D18E20101E5519B
:105F2000EA6A000FE96E010EEA22EF50E66E010107
:105F3000E4510101E525EA6A000FE96E070EEA2245
:105F4000E552E750EF6E0101E52BE4D792D0010155
:105F5000E7510F082DE2200E0101E75D29E2100E46
:105F60000101E75D0101E76F100E0101E703F3CFC7
:105F7000E4F10101E56B100E0101E55D18E201019C
:105F8000E551EA6A000FE96E010EEA22EF50E66E73
:105F90000101E4510101E525EA6A000FE96E080EEE
:105FA000EA22E552E750EF6E0101E52BE4D761D01C
:105FB0000101E7511F082DE2300E0101E75D29E2E2
:105FC000200E0101E75D0101E76F100E0101E703FB
:105FD000F3CFE4F10101E56B100E0101E55D18E27C
:105FE0000101E551EA6A000FE96E010EEA22EF5065
:105FF000E66E0101E4510101E525EA6A000FE96E50
:10600000090EEA22E552E750EF6E0101E52BE4D7D5
:1060100030D00101E7512F082CE2400E0101E75D6D
:1060200028E2300E0101E75D0101E76F100E01016A
:10603000E703F3CFE4F10101E56B100E0101E55D2B
:1060400018E20101E551EA6A000FE96E010EEA2249
:10605000EF50E66E0101E4510101E525EA6A000F07
:10606000E96E0A0EEA22E552E750EF6E0101E52BD8
:10607000E4D71200E6C1E7F1100E0101E75D24E26A
:10608000100E0101E703F3CFE4F10101E56B100EFF
:106090000101E55D18E20101E551EA6A100FE96EC0
:1060A000010EEA22EF50E66E0101E4510101E525FF
:1060B000EA6A000FE96E070EEA22E552E750EF6E3A
:1060C0000101E52BE4D792D00101E7510F082DE241
:1060D000200E0101E75D29E2100E0101E75D0101DB
:1060E000E76F100E0101E703F3CFE4F10101E56B67
:1060F000100E0101E55D18E20101E551EA6A100F99
:10610000E96E010EEA22EF50E66E0101E451010151
:10611000E525EA6A000FE96E080EEA22E552E7502B
:10612000EF6E0101E52BE4D761D00101E7511F08B3
:106130002DE2300E0101E75D29E2200E0101E75D4D
:106140000101E76F100E0101E703F3CFE4F1010154
:10615000E56B100E0101E55D18E20101E551EA6A07
:10616000100FE96E010EEA22EF50E66E0101E451D4
:106170000101E525EA6A000FE96E090EEA22E552FF
:10618000E750EF6E0101E52BE4D730D00101E75174
:106190002F082CE2400E0101E75D28E2300E0101DC
:1061A000E75D0101E76F100E0101E703F3CFE4F1B2
:1061B0000101E56B100E0101E55D18E20101E551F9
:1061C000EA6A100FE96E010EEA22EF50E66E010155
:1061D000E4510101E525EA6A000FE96E0A0EEA22A0
:1061E000E552E750EF6E0101E52BE4D71200010103
:1061F0002B0502E130EC50F0020E01012B5D02E1B3
:1062000093EC50F0030E01012B5D02E1F6EC50F02F
:10621000040E01012B5D02E102EC54F0050E0101B8
:106220002B5D02E165EC54F0060E01012B5D02E1ED
:10623000C8EC54F0070E01012B5D02E12BEC55F088
:10624000080E01012B5D02E1D9EC52F0090E0101AB
:106250002B5D02E13CEC53F00A0E01012B5D02E1E3
:106260009FEC53F00F0E01012B5D02E1BCEC51F0ED
:106270000B0E01012B5D10E10F013CBF03D08EEC32
:1062800055F00AD0E6DC0C01100EF96F22EC0CF090
:1062900001012B5101E0ABD70C0E01012B5D10E188
:1062A0000F013CBF03D0F1EC55F00AD0D2DC0C0159
:1062B000100EF96F22EC0CF001012B5101E097D781
:1062C0000D0E01012B5D10E10F013CBF03D080ECEE
:1062D0004FF00AD0BEDC0C01100EF96F22EC0CF06E
:1062E00001012B5101E083D70E0E01012B5D10E15E
:1062F0000F013CBF03D0D8EC4FF00AD0AADC0C0150
:10630000100EF96F22EC0CF001012B5101E06FD758
:106310000F010F013C51800B05E00F010F013D51B2
:10632000400B17E017D80F013D9D0F0130A702D099
:10633000ADEC18F00F0129AB0CD00F01299B89DCC3
:106340000C01100EF96F22EC0CF001012B5101E051
:106350004ED712000F012991A49A0F012D99030124
:10636000FF6BFE0E0301FF5D31E20F010F013C5197
:10637000800B05E00F010F013D51200B03E0ADEC58
:106380000DF002D0CEEC0CF00F0129A105D00F01C9
:10639000298B0F01309565D00F010F013C51800B07
:1063A00005E00F010F013D51200B03E0ADEC0DF0B6
:1063B00002D0CEEC0CF00F0129A105D00F01298BE2
:1063C0000F0130954ED00301FF2BCBD70F010F01EA
:1063D0003C51800B05E00F010F013D51200B01E006
:1063E0001DD00301FF6BFE0E0301FF5D17E2CEEC33
:1063F0000CF00F0129A105D00F01298B0F01309559
:1064000030D0CEEC0CF00F0129A105D00F01298B63
:106410000F01309526D00301FF2BE5D70F012DB3D7
:1064200018D00301FE690301FE690F013DB90BD0CD
:106430008B8A0F0130858A860C01200EF96F22ECC1
:106440000CF08A9605D00C01200EF96F22EC0CF0AE
:1064500007D00F012D930C01200EF96F22EC0CF0E8
:10646000A5D00F010F013D51100B07E10F010F01E6
:106470003D51400B02E00F013D890F013DA98B9A70
:106480000F012D930301FF6B300E0301FF5D15E239
:106490000F010F013C51800B05E00F010F013D5131
:1064A000200B03E0ADEC0DF002D0CEEC0CF00F01B0
:1064B00029B92DD00301FF2BE7D70601005105E1D3
:1064C0000F0129910F01299771D00301FF6BD00EA5
:1064D0000301FF5D15E20F010F013C51800B05E048
:1064E0000F010F013D51200B03E0ADEC0DF002D088
:1064F000CEEC0CF00F0129B90AD00301FF2BE7D72E
:1065000084EC56F00F0129910F0129974FD00F010C
:1065100030B74CD00F0129A704D00F0129970F01E4
:106520002D850F0129910F0129990F0129AD03D064
:106530000F012D953BD00F012DB52FD00F012DA1AF
:1065400004D07CEC3CF00F012D910F010F013E5166
:10655000010B07E10F010F013E51040B02E154EC66
:1065600056F00F012DAD0ED00F012D9D1FEC52F0F6
:106570000F013D9D0F012DB905D00F012D890F0190
:106580002D95EDD60F012DAB07D00F012D9B0101ED
:106590000A0E3B6F05EC2EF007D054EC56F00101CB
:1065A0000A0E3B6F05EC2EF00F012D951200D9CF8E
:1065B000E6FFE1CFD9FFE652DF6A01017351DF5CEC
:1065C00037E2DF50EA6A010FE96E020EEA22EF506D
:1065D000A96E0301080EFE6F1AEC0CF09CA207D006
:1065E0009C980301020EFE6F1AEC0CF09C889EAA88
:1065F0000BD0AFCFFEF59E9AB9EC2DF00A0E050137
:10660000FE5D02E122EC6EF0A8B210D00301FE693B
:106610009EAA0BD0AFCFFEF59E9AB9EC2DF00A0ED4
:106620000501FE5D02E122EC6EF0EED7DF2AC5D750
:10663000E552E552E7CFD9FF1200D9CFE6FFE1CF0F
:10664000D9FFE652DF6A02010051DF5C37E2DF501A
:10665000EA6A010FE96E020EEA22EF50AE6E030104
:10666000080EFE6F1AEC0CF0ACA207D0AC98030138
:10667000020EFE6F1AEC0CF0AC889EAA0BD0AFCFC6
:10668000FEF59E9AB9EC2DF00A0E0501FE5D02E1C1
:1066900022EC6EF0ADB210D00301FE699EAA0BD0C1
:1066A000AFCFFEF59E9AB9EC2DF00A0E0501FE5D06
:1066B00002E122EC6EF0EED7DF2AC5D7E552E552B3
:1066C000E7CFD9FF1200A38A0401010EEA6F04018B
:1066D000EA0502E10400FBD71200D9CFE6FFE1CFC3
:1066E000D9FFE652FE0EDBCF00F02F0EE76E00184A
:1066F000E8AE02D0003403D0E750D880005411E255
:10670000FE0EDBCF01F03A0EE76E0118E8AE02D0C4
:10671000E73402D0E750015C04E2FE0EDB50D00FFC
:10672000DF6EFE0EDBCF00F0400EE76E0018E8AE25
:1067300002D0003403D0E750D880005411E2FE0E9E
:10674000DBCF01F0470EE76E0118E8AE02D0E73468
:1067500002D0E750015C04E2FE0EDB50C90FDF6E91
:10676000FE0EDBCF00F0600EE76E0018E8AE02D040
:10677000003403D0E750D880005411E2FE0EDBCF86
:1067800001F0670EE76E0118E8AE02D0E73402D0E0
:10679000E750015C04E2FE0EDB50A90FDF6EDF5014
:1067A00000D0E552E552E7CFD9FF1200AACFF1F4AD
:1067B0000401E92B2F0E0401F15D0CE10401ED2B26
:1067C000000EEE230401EA6BA39AA49A0401F3914C
:1067D0000401F38B3A0E0401F15D05E10401F3813C
:1067E0000401E96B04D30401F3A101D30401E951CD
:1067F0002A0A01E176D2030A01E168D2010A01E125
:1068000053D20F0A01E145D2010A01E130D2030A55
:1068100001E122D2010A01E10DD2070A01E1FFD113
:10682000010A01E1EAD1030A01E1DCD1010A01E137
:10683000C7D13F0A01E1B9D1010A01E1A4D1030A9C
:1068400001E196D1010A01E181D1070A01E173D189
:10685000010A01E15ED1030A01E150D1010A01E11F
:106860003BD10F0A01E12DD1010A01E118D1030A40
:1068700001E10AD1010A01E1F5D0070A01E1E7D0FF
:10688000010A01E1D2D0030A01E1C4D0010A01E109
:10689000AFD01F0A01E1A1D0010A01E18CD0030AA7
:1068A00001E17ED0010A6BE0070A5EE0010A4DE0DB
:1068B000030A40E00F0A38E0030A2BE0010A23E054
:1068C000070A16E0010A0EE0030A01E011D2F1C442
:1068D000E6FF03DFE5520401E86F0401E839F00B3D
:1068E000E86F07D2F1C4E6FFF8DEE5520401E813D1
:1068F000F1C4E6FFF2DEE5520C01F36F0C01F3394F
:10690000F00BF36FF6D1F1C4E6FFE7DEE5520C01C0
:10691000F313F1C4E6FFE1DEE5520C01F26F0C0166
:10692000F239F00BF26FE5D1F1C4E6FFD6DEE552A5
:106930000C01F213F1C4E6FFD0DEE5520401D66F7C
:106940000401D639F00BD66FD4D1F1C4E6FFC5DE11
:10695000E5520401D613F2CCA2F0F3CCA3F0D6C4D6
:10696000A4F0EDEC16F0C5D1F1C4E6FFB6DEE552B9
:106970000401D76F0401D739F00BD76FBAD1F1C436
:10698000E6FFABDEE5520401D7130C01F22900014A
:10699000A26FF3CCA3F0D7C4A4F0EDEC16F0A9D10C
:1069A000F1C4E6FF9ADEE5520401D86F0401D8393C
:1069B000F00BD86F9ED1F1C4E6FF8FDEE5520401E3
:1069C000D813020E0C01F2250001A26FF3CCA3F044
:1069D000D8C4A4F0EDEC16F08CD1F1C4E6FF7DDE56
:1069E000E5520401D96F0401D939F00BD96F81D177
:1069F000F1C4E6FF72DEE5520401D913030E0C0167
:106A0000F2250001A26FF3CCA3F0D9C4A4F0EDEC01
:106A100016F06FD1F1C4E6FF60DEE5520401DA6FD3
:106A20000401DA39F00BDA6F64D1F1C4E6FF55DE08
:106A3000E5520401DA13040E0C01F2250001A26FE5
:106A4000F3CCA3F0DAC4A4F0EDEC16F052D1F1C40B
:106A5000E6FF43DEE5520401DB6F0401DB39F00B96
:106A6000DB6F47D1F1C4E6FF38DEE5520401DB13EA
:106A7000050E0C01F2250001A26FF3CCA3F0DBC4DC
:106A8000A4F0EDEC16F035D1F1C4E6FF26DEE552B8
:106A90000401DC6F0401DC39F00BDC6F2AD1F1C496
:106AA000E6FF1BDEE5520401DC13060E0C01F225A5
:106AB0000001A26FF3CCA3F0DCC4A4F0EDEC16F05F
:106AC00018D1F1C4E6FF09DEE5520401DD6F0401CF
:106AD000DD39F00BDD6F0DD1F1C4E6FFFEDDE552CF
:106AE0000401DD13070E0C01F2250001A26FF3CCA7
:106AF000A3F0DDC4A4F0EDEC16F0FBD0F1C4E6FF8A
:106B0000ECDDE5520401DE6F0401DE39F00BDE6FCF
:106B1000F0D0F1C4E6FFE1DDE5520401DE13080E1A
:106B20000C01F2250001A26FF3CCA3F0DEC4A4F0A7
:106B3000EDEC16F0DED0F1C4E6FFCFDDE552040146
:106B4000DF6F0401DF39F00BDF6FD3D0F1C4E6FF54
:106B5000C4DDE5520401DF13090E0C01F22500012A
:106B6000A26FF3CCA3F0DFC4A4F0EDEC16F0C1D01B
:106B7000F1C4E6FFB2DDE5520401E06F0401E03943
:106B8000F00BE06FB6D0F1C4E6FFA7DDE5520401DB
:106B9000E0130A0E0C01F2250001A26FF3CCA3F062
:106BA000E0C4A4F0EDEC16F0A4D0F1C4E6FF95DD4E
:106BB000E5520401E16F0401E139F00BE16F99D076
:106BC000F1C4E6FF8ADDE5520401E1130B0E0C016E
:106BD000F2250001A26FF3CCA3F0E1C4A4F0EDEC28
:106BE00016F087D0F1C4E6FF78DDE5520401E26FCC
:106BF0000401E239F00BE26F7CD0F1C4E6FF6DDDF9
:106C0000E5520401E2130C0E0C01F2250001A26F03
:106C1000F3CCA3F0E2C4A4F0EDEC16F06AD0F1C41A
:106C2000E6FF5BDDE5520401E36F0401E339F00B9D
:106C3000E36F5FD0F1C4E6FF50DDE5520401E313DA
:106C40000D0E0C01F2250001A26FF3CCA3F0E3C4FA
:106C5000A4F0EDEC16F04DD0F1C4E6FF3EDDE552B8
:106C60000401E46F0401E439F00BE46F42D0F1C495
:106C7000E6FF33DDE5520401E4130E0E0C01F225AC
:106C80000001A26FF3CCA3F0E4C4A4F0EDEC16F085
:106C900030D0F1C4E6FF21DDE5520401E56F0401C7
:106CA000E539F00BE56F25D0F1C4E6FF16DDE552BE
:106CB0000401E5130F0E0C01F2250001A26FF3CCC5
:106CC000A3F0E5C4A4F0EDEC16F013D0F1C4E6FF98
:106CD00004DDE5520401EB6F0401EB39F00BEB6FBF
:106CE00008D0F1C4E6FFF9DCE5520401EB1301D052
:106CF00000D00D0E0401F15D53E12A0E0401E76E90
:106D0000E919E8AE02D0E73402D0E750E95D48E384
:106D10000401E96B0401F3910401100EEC6F0C0106
:106D2000F3510401EC270C01F2510401EC2704019A
:106D3000EF6BF06B100E0401F0AF02D0D89003D0CF
:106D4000EF5D000EF05910E2D60E0401EF25E96E5A
:106D5000040E0401F021EA6EEF500401EC27040157
:106D6000EF2B000EF023E6D7ECC400F0016A00BE62
:106D70000168000ED8800056010E015600C0ECF4E8
:106D80000401EB510401EC5D05E10401ED2B000E63
:106D9000EE2306D00401EA6BA39AA49A0401F387B8
:106DA000160E0401E95D17E1800E0C01F25D13E19E
:106DB0000C01F35110E1340E0401DB5D04E1310EEE
:106DC0000401DC5D08E00401E96B0401EA6BA39AAD
:106DD000A49A0401F3850C01F3517F0808E2040131
:106DE000E96B0401EA6BA39AA49A0401F3890400F5
:106DF0001200D9CFE6FFE1CFD9FFE6520C01040E15
:106E0000F26F0C01F36B3CEC3EF0F350DF6E0F01C0
:106E100028A10DD08B8A0C01200EF96F22EC0CF00A
:106E20008B9A0C01200EF96F22EC0CF0F3D7110EA7
:106E3000DF5C08E10C01050EF26F3CEC3EF0F3CF95
:106E40002EFF10D00C01110EF66F58EC3EF00C0125
:106E5000050EF26F0F01090E2E6F0C01090EF66F71
:106E600058EC3EF001016F6B0101706B0101716B19
:106E70000101726B0101030EE16F0C01850EF26FCF
:106E80000C01340EF66F58EC3EF00C01F22B0C01A5
:106E9000310EF66F58EC3EF00C01F22BFAC1F6FC05
:106EA00058EC3EF00C01F22BFBC1F6FC58EC3EF026
:106EB0000C01100EF26F0101F26B200E0101F25D68
:106EC00013E23CEC3EF0F350E66E0101F251EA6A47
:106ED000000FE96E0B0EEA22E552E750EF6E0C014F
:106EE000F22B0101F22BE9D70101F26B200E010117
:106EF000F25D0EE20101F251EA6A000FE96E0B0E3B
:106F0000EA22EF50FF0801E004D00101F22BEED796
:106F1000F5D00101F26B080E0101F25D13E23CECC9
:106F20003EF0F350E66E0101F251EA6A200FE96E7D
:106F30000B0EEA22E552E750EF6E0C01F22B010135
:106F4000F22BE9D70101F26B080E0101F25D13E2A9
:106F50003CEC3EF0F350E66E0101F251EA6A280F74
:106F6000E96E0B0EEA22E552E750EF6E0C01F22BB0
:106F70000101F22BE9D70101F26B0F0E0101F25D65
:106F800013E23CEC3EF0F350E66E0101F251EA6A86
:106F9000300FE96E0B0EEA22E552E750EF6E0C015E
:106FA000F22B0101F22BE9D70101F26B0F0E010167
:106FB000F25D13E23CEC3EF0F350E66E0101F2515B
:106FC000EA6A3F0FE96E0B0EEA22E552E750EF6ED8
:106FD0000C01F22B0101F22BE9D70101F26B200E1B
:106FE0000101F25D13E23CEC3EF0F350E66E01016C
:106FF000F251EA6A4E0FE96E0B0EEA22E552E750B3
:10700000EF6E0C01F22B0101F22BE9D70101F26BBB
:10701000040E0101F25D13E23CEC3EF0F350E66E2B
:107020000101F251EA6A6E0FE96E0B0EEA22E55297
:10703000E750EF6E0C01F22B0101F22BE9D70101B1
:10704000F26B030E0101F25D13E23CEC3EF0F350F3
:10705000E66E0101F251EA6A140FE96E0F0EEA22A0
:10706000E552E750EF6E0C01F22B0101F22BE9D74C
:107070000C01890EF26F0101F26B0F0E0101F25D3E
:1070800013E23CEC3EF0F350E66E0101F251EA6A85
:10709000990FE96E0B0EEA22E552E750EF6E0C01F4
:1070A000F22B0101F22BE9D70101F26B040E010171
:1070B000F25D13E23CEC3EF0F350E66E0101F2515A
:1070C000EA6AA80FE96E0B0EEA22E552E750EF6E6E
:1070D0000C01F22B0101F22BE9D7FF0E0B01995D98
:1070E00004E0FF0E0B01A85D02E10F013983FF0EE2
:1070F0000B013F5D02E00F013981B3D10C01820E1B
:10710000F26F3CEC3EF0F3CF14FF0C01F22B3CECA1
:107110003EF0F3CF15FF0C01F22B3CEC3EF0F3CF29
:1071200016FFFF0E0F01145D08E0FF0E0F01155D45
:1071300004E0FF0E0F01165D22E10F01310E146F06
:107140000F01320E156F0F01300E166F0C01820EFB
:10715000F26F0101F26B030E0101F25D10E2010119
:10716000F251EA6A140FE96E0F0EEA22EFCFF6FC35
:1071700058EC3EF00C01F22B0101F22BECD70B0185
:10718000690E006F0B016E0E016F0B01740E026F22
:107190000B01650E036F0B01720E046F0B016E0E77
:1071A000056F0B01650E066F0B01740E076F0B0167
:1071B0002E0E086F0B016C0E096F0B016D0E0A6F1E
:1071C0000B01740E0B6F0B012E0E0C6F0B016C0E6E
:1071D0000D6F0B01760E0E6F01010F0EF26F200E78
:1071E0000101F25D0BE20101F251EA6A000FE96E62
:1071F0000B0EEA22EF680101F22BF1D70C01100E01
:10720000F26F0101F26B200E0101F25D10E201014B
:10721000F251EA6A000FE96E0B0EEA22EFCFF6FC9C
:1072200058EC3EF00C01F22B0101F22BECD70C01D3
:10723000300EF26F400E0C01F25D07E20C01F669B0
:1072400058EC3EF00C01F22BF5D70101F26B080E61
:107250000101F25D0BE20101F251EA6A200FE96ED1
:107260000B0EEA22EF680101F22BF1D70101F26B5C
:10727000080E0101F25D0BE20101F251EA6A280FEA
:10728000E96E0B0EEA22EF680101F22BF1D70B0138
:10729000300E306F0B012E0E316F0B01300E326F3E
:1072A0000B012E0E336F0B01300E346F0B012E0EBF
:1072B000356F0B01300E366F0101070EF26F0F0EA6
:1072C0000101F25D0BE20101F251EA6A300FE96E51
:1072D0000B0EEA22EF680101F22BF1D70C01400EF0
:1072E000F26F0101F26B0F0E0101F25D10E201017C
:1072F000F251EA6A300FE96E0B0EEA22EFCFF6FC8C
:1073000058EC3EF00C01F22B0101F22BECD70101FD
:10731000F26B0F0E0101F25D0BE20101F251EA6A1C
:107320003F0FE96E0B0EEA22EF680101F22BF1D755
:107330000101F26B0F0E0101F25D09E20C01F66929
:1073400058EC3EF00C01F22B0101F22BF3D70101B6
:10735000F26B200E0101F25D0BE20101F251EA6ACB
:107360004E0FE96E0B0EEA22EF680101F22BF1D706
:107370000101F26B200E0101F25D09E20C01F669D8
:1073800058EC3EF00C01F22B0101F22BF3D70F0168
:1073900039910B01390E6E6F0B01330E6F6F0B01BC
:1073A000300E706F0B0171690101F26B040E010167
:1073B000F25D10E20101F251EA6A6E0FE96E0B0E06
:1073C000EA22EFCFF6FC58EC3EF00C01F22B010163
:1073D000F22BECD70101F26B0F0E0101F25D0BE213
:1073E0000101F251EA6A990FE96E0B0EEA22EF6889
:1073F0000101F22BF1D70101F26B040E0101F25DE4
:107400000BE20101F251EA6AA80FE96E0B0EEA22C3
:10741000EF680101F22BF1D70C01890EF26F010127
:10742000F26B0F0E0101F25D09E20C01F66958ECF6
:107430003EF00C01F22B0101F22BF3D70101F26BAC
:10744000040E0101F25D09E20C01F66958EC3EF010
:107450000C01F22B0101F22BF3D70F013983CFEC92
:1074600059F0E552E552E7CFD9FF12000F013CBBBE
:107470006CD00F013CB169D00B01736B0F010F0190
:107480003951010B1FE00F010F013951040B1AE1B3
:107490000C010B0EF96F22EC0CF00F0128939DEC00
:1074A00045F00301FF6BA00E0301FF5D0BE20F012E
:1074B00028B308D0CC6A2EEC0CF02EEC0CF00301B3
:1074C000FF2BF1D70F013D870F013A970B01730E88
:1074D000736FCC6A0C01200EF96F22EC0CF013ECE8
:1074E00048F00F0128930301FF6B700E0301FF5D4D
:1074F00009E20F0128B306D0CC6A2EEC0CF0030190
:10750000FF2BF3D70F013C810F013C970F0128930C
:107510003DEC48F00F013CBF04D00F013B8F0B0145
:10752000766B0301FF6B700E0301FF5D0EE20F012E
:1075300028B30BD00F013DA302D09DD806D0CC6A52
:107540002EEC0CF00301FF2BEED712000F013CA72D
:1075500091D00B01936B0A0E0B01935D16E20B01A8
:107560009351EA6A010FE96E020EEA22EF50E66ECD
:107570000B019351EA6A890FE96E0B0EEA22E5527C
:10758000E750EF6E0B01932BE6D71EEC4AF00B0190
:10759000936B0A0E0B01935D16E20B019351EA6A9D
:1075A000890FE96E0B0EEA22EF50E66E0B01935144
:1075B000EA6A010FE96E020EEA22E552E750EF6E29
:1075C0000B01932BE6D70F012C930F013D910F0177
:1075D0003C990301FF6BFF0E0301FF5D15E2CC6ACE
:1075E0002EEC0CF02EEC0CF00F012CA30AD00F01A6
:1075F0002C93CC6A2EEC0CF073C100F21DEC33F02E
:107600000FD00301FF2BE7D70B01742B030E0B01E7
:10761000745D05E10F013D8F0B01746B2CD82AD0EE
:107620000301FF6BD00E0301FF5D14E2CC6A2EEC68
:107630000CF02EEC0CF00F013CA909D00F013C9985
:107640000F0128930B01746B0F013D8D13D00301C3
:10765000FF2BE8D70B01742B030E0B01745D06E1C1
:107660000F013D8F0B01746B06D804D00F013DB3A1
:1076700002D800D012000F010F013D51010B16E19D
:107680000F010F013D51020B11E10F010F013D519F
:10769000800B0CE10F010F013C51800B01E07ED00B
:1076A0000F010F013A51080B01E178D00B01776B04
:1076B0000F013CBF40D00F010F013D51010B05E10F
:1076C0000F010F013D51020B16E00B01AE2B020E14
:1076D0000B01AE5D10E10B01AE6B0F013AB90BD09F
:1076E0000F013A890F013A9B0F013B9B01010D0EDF
:1076F0003B6F05EC2EF00F010F013C51800B17E1A1
:107700000F010F013A51080B12E00B01AE6B0F0194
:107710003A970F013A990F013ABB09D00F013A8B02
:107720000F013B8B01010E0E3B6F05EC2EF00B01A0
:10773000730E776F1BD00F010F013D51010B0AE152
:107740000F010F013D51020B05E10F010F013D51EA
:10775000800B0CE00B01AE2B020E0B01AE5D06E1BF
:107760000B01AE6B0F013A890F013A9B42EC4AF0D4
:107770000F013C8B0F013C910F013C970F013D9194
:107780000F013D930F013D9F0F013D990F013D9763
:107790000B01786B0F013A830F013B9F12000F0121
:1077A0003CBB43D00F013CB140D00F013D850F01E0
:1077B00039970B01730E736FCC6A0C010B0EF96FC6
:1077C00022EC0CF013EC48F00F0128930301FF6B3F
:1077D000700E0301FF5D09E20F0128B306D0CC6AE9
:1077E0002EEC0CF00301FF2BF3D70F013C810F01AE
:1077F0003C970F013B8F0B01766B0F01289347ECF1
:1078000049F00301FF6B700E0301FF5D0EE20F01F3
:1078100028B30BD00F013DA302D008D806D0CC6A04
:107820002EEC0CF00301FF2BEED712000F010F011D
:107830003D51010B0AE10F010F013D51020B05E122
:107840000F010F013951080B56E00F010F013D5197
:10785000010B05E10F010F013D51020B22E00B016D
:10786000AD2B020E0B01AD5D1CE10B01AD6B0F01E9
:1078700039B912D00F0139890F01399B0F013CBF73
:107880000BD08EEC55F0AAEC31F00F01299B0F01C3
:1078900030A702D0ADEC18F00F013AAB02D00F01C7
:1078A0003C8F0F0139A70ED00B01AD6B0F01399939
:1078B0000F0139BB07D00F01398B01010C0E3B6F53
:1078C00005EC2EF042EC4AF00F013C8B0B01730EDD
:1078D000776F0F013C910F013C970F013D910F0114
:1078E0003D930F0139970F013D950F013A930F0119
:1078F0003A910F013B9F1200D9CFE6FFE1CFD9FFAC
:10790000020EE12601017451050801E389D1530EED
:107910000601055D6AE1540E0601065D66E1140E7E
:107920000601075D62E103014E0E006F0301550E73
:10793000016F0F012EB104D003012D0E026F03D091
:1079400003012B0E026F03012C0E036F0301460E81
:10795000046F0301310E056F0F012EB304D0030134
:107960002D0E066F03D003012B0E066F03012C0EA4
:10797000076F0301490E086F03014E0E096F0F01D7
:107980002EB504D003012D0E0A6F03D003012B0E78
:107990000A6F03012C0E0B6F0301430E0C6F0301E2
:1079A000450E0D6F0F012EB704D003012D0E0E6F83
:1079B00003D003012B0E0E6F03012C0E0F6F03017A
:1079C000570E106F0301540E116F0F012EB904D022
:1079D00003012D0E126F03D003012B0E126F030152
:1079E000130EFC6F0F012D8D28D12ECF2FFF01011B
:1079F000742B010EDB6A050EDF6E01017451DF5C32
:107A000001E30ED1DF50EA6A000FE96E060EEA22AA
:107A1000EF502C080AE0DF50EA6A000FE96E060E0C
:107A2000EA22EF50140801E0F7D0010EDB50030802
:107A300001E0EED0030EDF5CEA6A000FE96E060E8D
:107A4000EA22EF504E0825E1020EDF5CEA6A000FE1
:107A5000E96E060EEA22EF5055081BE1DF04EA6AE0
:107A6000000FE96E060EEA22EF502B0803E10F012A
:107A70002F810FD0DF04EA6A000FE96E060EEA22BA
:107A8000EF502D0803E10F012F9103D00F012D8B33
:107A9000D4D0030EDF5CEA6A000FE96E060EEA221C
:107AA000EF50460825E1020EDF5CEA6A000FE96E3E
:107AB000060EEA22EF5031081BE1DF04EA6A000FEC
:107AC000E96E060EEA22EF502B0803E10F012F8327
:107AD0000FD0DF04EA6A000FE96E060EEA22EF50CB
:107AE0002D0803E10F012F9303D00F012D8BA5D09B
:107AF000030EDF5CEA6A000FE96E060EEA22EF5021
:107B0000490825E1020EDF5CEA6A000FE96E060E05
:107B1000EA22EF504E081BE1DF04EA6A000FE96E2B
:107B2000060EEA22EF502B0803E10F012F850FD03C
:107B3000DF04EA6A000FE96E060EEA22EF502D0814
:107B400003E10F012F9503D00F012D8B76D0030E8B
:107B5000DF5CEA6A000FE96E060EEA22EF50430886
:107B600025E1020EDF5CEA6A000FE96E060EEA22EA
:107B7000EF5045081BE1DF04EA6A000FE96E060ECC
:107B8000EA22EF502B0803E10F012F870FD0DF040B
:107B9000EA6A000FE96E060EEA22EF502D0803E1B3
:107BA0000F012F9703D00F012D8B47D0030EDF5C01
:107BB000EA6A000FE96E060EEA22EF50570825E147
:107BC000020EDF5CEA6A000FE96E060EEA22EF5051
:107BD00054081BE1DF04EA6A000FE96E060EEA2290
:107BE000EF502B0803E10F012F890FD0DF04EA6A61
:107BF000000FE96E060EEA22EF502D0803E10F0197
:107C00002F9903D00F012D8B18D0010EDB6A03D002
:107C10000F012D8B12D002D0010EDB2ADF2AEDD608
:107C20002FCF2EFF0C01A00EF16F0C01050EF26F8D
:107C30000C01F36B2ECFF6FC3BD80101F36BFE0E6B
:107C40000101F35D0BE20101F351EA6A000FE96EF5
:107C5000060EEA22EF6A0101F32BF1D70601FF6B52
:107C60000101746B020EE15C02E2E16AE552E16E31
:107C7000E552E7CFD9FF1200F1CCF4FCA9D8C7D860
:107C8000F3CCF4FCC4D8F2CCF4FCC1D8A1D8F1CC2C
:107C9000F4FC0C01F481BBD8E2D845D90C01F551B4
:107CA000006E016A00C0F3FF01C0F4FF00D01200B3
:107CB000F1CCF4FC8DD8ABD8F3CCF4FCA8D8F2CC42
:107CC000F4FCA5D8F6CCF4FCA2D82DD9CC6A2EECC5
:107CD0000CF01200F1CCF4FC7BD899D8F3CCF4FC76
:107CE00096D8F2CCF4FC93D818CFF4FC90D819CFE6
:107CF000F4FC8DD81ACFF4FC8AD81BCFF4FC87D8BB
:107D00001CCFF4FC84D81DCFF4FC81D81ECFF4FC2A
:107D10007ED81FCFF4FC7BD820CFF4FC78D821CFBD
:107D2000F4FC75D822CFF4FC72D823CFF4FC6FD8C2
:107D300024CFF4FC6CD825CFF4FC69D826CFF4FC12
:107D400066D827CFF4FC63D8EED8CC6A2EEC0CF0C2
:107D50001200F1CCF4FC3CD85AD8F3CCF4FC57D840
:107D6000F2CCF4FC54D879CBF4FC51D87ACBF4FCA7
:107D70004ED87BCBF4FC4BD87CCBF4FC48D87DCBE5
:107D8000F4FC45D87ECBF4FC42D87FCBF4FC3FD842
:107D900080CBF4FC3CD881CBF4FC39D882CBF4FC0A
:107DA00036D883CBF4FC33D884CBF4FC30D885CBE5
:107DB000F4FC2DD886CBF4FC2AD887CBF4FC27D84A
:107DC00088CBF4FC24D8AFD8CC6A2EEC0CF012008F
:107DD00089868984929492960301FE690301FE6963
:107DE0000301FE690301FE690301FE690301FE69E7
:107DF00089960301FE690301FE690301FE6903011F
:107E0000FE690301FE690301FE6989941200010104
:107E1000080EFD6F0101FD5119E00101FD070F0181
:107E2000289D0C01F4AF02D00F01288D58D8F4CC56
:107E3000F7FC0C01F451E8240C01F46F0C01F7AFCE
:107E400004D00C01F4290C01F46FE4D72ED80F01F3
:107E500028910F0128AF02D00F01288112000101E3
:107E6000080EFD6F0C01F56B0101FD511AE00101D7
:107E7000FD07F5CCF7FC0C01F551E8240C01F56F7A
:107E80000C01F7AF04D00C01F5290C01F56F0DD8EA
:107E90000F0128AF05D0010E0C01F5110C01F56F93
:107EA000E3D70F01288D1BD81200928689840F0119
:107EB000289F0301FE690301FE690301FE690301B6
:107EC000FE690301FE690301FE6980A602D00F016D
:107ED000288F0301FE690301FE69899412000F01D6
:107EE00028BD02D0899601D0898692960301FE6949
:107EF0000301FE690301FE690301FE690301FE69D6
:107F00000301FE690301FE6989840301FE6903011F
:107F1000FE690301FE690301FE690301FE690301B5
:107F2000FE6989941200929492968996898403013D
:107F3000FE690301FE690301FE690301FE69030195
:107F4000FE690301FE6989860301FE690301FE697A
:107F50000301FE690301FE690301FE690301FE6975
:107F600092840301FE690301FE69928612000201F8
:107F70000C0E006F0201410E016F0201540E026FE0
:107F800002012B0E036F0201490E046F0201500E15
:107F9000056F0201520E066F02013D0E076F0201CE
:107FA000390E086F0201360E096F0201300E0A6F9A
:107FB0000201300E0B6F02010D0E0C6F1DEC33F041
:107FC000120002010A0E006F0201410E016F020150
:107FD000540E026F02012B0E036F0201430E046F59
:107FE00002014C0E056F0201490E066F0201500E90
:107FF000076F02013D0E086F0201310E096F020189
:108000000D0E0A6F1DEC33F0120002010A0E006F14
:108010000201410E016F0201540E026F02012B0E8C
:10802000036F0201430E046F02014D0E056F020142
:10803000470E066F0201460E076F02013D0E086FE4
:108040000201310E096F02010D0E0A6F0F012A9F06
:108050001DEC33F0120002010A0E006F0201410E06
:10806000016F0201540E026F02012B0E036F020119
:10807000430E046F02014D0E056F0201470E066F9D
:108080000201460E076F02013D0E086F0201300E1D
:10809000096F02010D0E0A6F0F012A8F1DEC33F0DC
:1080A000120002010E0E006F0201410E016F02016B
:1080B000540E026F02012B0E036F0201430E046F78
:1080C00002014D0E056F0201470E066F02014C0EB4
:1080D000076F02013D0E086F0201220E096F0201B7
:1080E000410E0A6F02014C0E0B6F02014C0E0C6F19
:1080F0000201220E0D6F02010D0E0E6F1DEC33F00A
:1081000012000201410E016F0201540E026F0201C2
:108110002B0E036F0201430E046F02014D0E056F1B
:108120000201470E066F0201520E076F02013D0E5B
:10813000086F0F012BB309D07AC109F202010D0EAD
:108140000A6F02010A0E006F0AD07BC109F27AC1E0
:108150000AF202010D0E0B6F02010B0E006F1DECF7
:1081600033F012000201410E016F0201540E026F42
:1081700002012B0E036F0201430E046F02014D0E2C
:10818000056F0201470E066F0201440E076F0201E0
:108190003D0E086F0F012BB309D07AC109F202011D
:1081A0000D0E0A6F02010A0E006F0AD07BC109F2A0
:1081B0007AC10AF202010D0E0B6F02010B0E006F65
:1081C0001DEC33F00F012B910F012B9301017A6B02
:1081D00001017B6B12000201050E006F0201410ECE
:1081E000016F0201540E026F0201450E036F02017E
:1081F000300E046F02010D0E056F1DEC33F01200FE
:108200000201040E006F0201410E016F0201540EC3
:10821000026F0201410E036F02010D0E046F1DEC8F
:1082200033F012000201050E006F0201410E016FD2
:108230000201540E026F0201480E036F0201300E5C
:10824000046F02010D0E056F1DEC33F012000201E8
:108250000D0E006F0201410E016F0201540E026FFC
:1082600002012B0E036F0201430E046F0201500E38
:10827000056F0201490E066F02014E0E076F0201E3
:108280003D0E086F0201300E096F0201300E0A6FB9
:108290000201300E0B6F0201300E0C6F02010D0E49
:1082A0000D6F1DEC33F012000201090E006F020188
:1082B000410E016F0201540E026F02012B0E036F7B
:1082C0000201430E046F0201500E056F0201490EB8
:1082D000066F02014E0E076F02013F0E086F02018A
:1082E0000D0E096F1DEC33F012000201090E006F34
:1082F0000201410E016F0201540E026F02012B0EAA
:10830000036F0201430E046F0201520E056F02015A
:10831000450E066F0201470E076F02013F0E086F00
:1083200002010D0E096F1DEC33F012000201070E61
:10833000006F0201410E016F0201540E026F020133
:108340002B0E036F0201430E046F0201530E056FE3
:108350000201510E066F02010D0E076F1DEC33F086
:10836000120002010C0E006F0201410E016F0201AA
:10837000540E026F02012B0E036F0201510E046FA7
:108380000201490E056F02014E0E066F0201490EF1
:10839000076F0201530E086F0201540E096F0201AC
:1083A000410E0A6F0201540E0B6F02010D0E0C6F8D
:1083B0001DEC33F0120002010C0E006F0201410EA1
:1083C000016F0201540E026F02012B0E036F0201B6
:1083D000430E046F02014E0E056F02014D0E066F33
:1083E0000201490E076F02013D0E086F0201320EB5
:1083F000096F02012C0E0A6F0201300E0B6F020191
:108400000D0E0C6F1DEC33F012000201080E006F10
:108410000201410E016F0201540E026F02012B0E88
:10842000036F0201430E046F0201470E056F020144
:108430004D0E066F0201520E076F02010D0E086FFE
:108440001DEC33F01200D9CFE6FFE1CFD9FF020EC9
:10845000E1260201410E016F0201540E026F02017A
:108460002B0E036F0201430E046F02014D0E056FC8
:108470000201470E066F0201530E076F02013D0E07
:10848000086F0201220E096FDE52110EDD6EDF6AE7
:10849000010EDB50DF5C0EE2DF50EA6A000FE96E8E
:1084A0000D0EEA22EF503A0803E1010EDFCFDBFFA9
:1084B000DF2AEED7DF6A010EDB50DF5C14E2DF500B
:1084C000EA6A000FE96E0D0EEA22EF50E66E090E21
:1084D000DF24EA6A010FE96E020EEA22E552E75054
:1084E000EF6EDF2AE8D7010EDB50090FEA6A010FB1
:1084F000E96E020EEA22220EEF6E010EDB500A0F29
:10850000EA6A010FE96E020EEA220D0EEF6E010E0D
:10851000DB500B0F0201006F1DEC33F0020EE15C2B
:1085200002E2E16AE552E16EE552E7CFD9FF1200BF
:108530000201410E016F0201540E026F02012B0E67
:10854000036F0201430E046F02014D0E056F02011D
:10855000470E066F0201530E076F02013D0E086FB2
:10856000B8CBB7FB0B01B751630823E2640E0B01D4
:10857000B75D0B01B76F0201310E096F0201300EBA
:108580000A6F0B01B751090808E202010A2B0A0E13
:108590000B01B75D0B01B76FF4D7300E0B01B72598
:1085A00002010B6F02010D0E0C6F02010C0E006F29
:1085B0002AD00B01B75109081BE20201300E096FE6
:1085C0000B01B751090808E20201092B0A0E0B0141
:1085D000B75D0B01B76FF4D7300E0B01B725020161
:1085E0000A6F02010D0E0B6F02010B0E006F0BD014
:1085F000300E0B01B7250201096F02010D0E0A6F43
:1086000002010A0E006F1DEC33F01200D9CFE6FF15
:10861000E1CFD9FF040EE126DE52110EDD6EDF6AD6
:10862000010EDB50DF5C10E2DF50EA6A000FE96EFA
:108630000D0EEA22EF503A0805E1DF28E76E010E41
:10864000E7CFDBFFDF2AECD7FE0EF36E020EF3CF8F
:10865000DBFF010EDB50DF6E020EDB50DF5C0EE253
:10866000DF50EA6A000FE96E0D0EEA22EF5014089F
:1086700003E1020EDFCFDBFFDF2AEED7020EDBCFF6
:10868000E6FF010EDB50E552E75CE76E030EE7CF35
:10869000DBFF030EDB5000081AE2DF6A030EDB503B
:1086A000DF5C15E2010EDB50DF24EA6A000FE96EA1
:1086B0000D0EEA22EF50E66EDF50EA6A010FE96E16
:1086C000020EEA22E552E750EF6EDF2AE7D7030EEB
:1086D000DB50EA6A010FE96E020EEA221A0EEF6E13
:1086E000030EDB280201006F1DEC33F0040EE15C89
:1086F00002E2E16AE552E16EE552E7CFD9FF1200EE
:10870000D9CFE6FFE1CFD9FF030EE1260201300EFB
:10871000016F0201300E026F7D0E0B01B85D01E3A7
:1087200084D0DF6A0B01B851DF5C6DE2020EDF021C
:10873000010EF3CFDBFFDF50EA6A000FE96E0D0E8A
:10874000EA22EF380F0BE76E020EE7CFDBFF0A0ECF
:10875000F36E020EDBCFF4FFF350F45C10E2020E76
:10876000DB50300FE66E010EDB50020FEA6A010F9C
:10877000E96E020EEA22E552E750EF6E0FD0020ECC
:10878000DB50370FE66E010EDB50020FEA6A010F75
:10879000E96E020EEA22E552E750EF6EDF50EA6A18
:1087A000000FE96E0D0EEA22EF500F0BE76E020E7E
:1087B000E7CFDBFF0A0EF36E020EDBCFF4FFF350C0
:1087C000F45C10E2020EDB50300FE66E010EDB505F
:1087D000030FEA6A010FE96E020EEA22E552E75042
:1087E000EF6E0FD0020EDB50370FE66E010EDB503E
:1087F000030FEA6A010FE96E020EEA22E552E75022
:10880000EF6EDF2A8FD7010EDB50040FEA6A010FEB
:10881000E96E020EEA221A0EEF6E010EDB50050F12
:108820000201006F1DEC33F0F7D0DF6A7D0EDF5CD4
:108830006DE2020EDF02010EF3CFDBFFDF50EA6ACA
:10884000000FE96E0D0EEA22EF380F0BE76E020EF5
:10885000E7CFDBFF0A0EF36E020EDBCFF4FFF3501F
:10886000F45C10E2020EDB50300FE66E010EDB50BE
:10887000020FEA6A010FE96E020EEA22E552E750A2
:10888000EF6E0FD0020EDB50370FE66E010EDB509D
:10889000020FEA6A010FE96E020EEA22E552E75082
:1088A000EF6EDF50EA6A000FE96E0D0EEA22EF501C
:1088B0000F0BE76E020EE7CFDBFF0A0EF36E020E20
:1088C000DBCFF4FFF350F45C10E2020EDB50300F0C
:1088D000E66E010EDB50030FEA6A010FE96E020E2D
:1088E000EA22E552E750EF6E0FD0020EDB50370F51
:1088F000E66E010EDB50030FEA6A010FE96E020E0D
:10890000EA22E552E750EF6EDF2A90D7010EDB50E6
:10891000040F0201006F1DEC33F0010EDB6A7D0EC7
:10892000DF6E0B01B851DF5C68E2DF50EA6A000FCE
:10893000E96E0D0EEA22EF380F0BE76E020EE7CF5D
:10894000DBFF0A0EF36E020EDBCFF4FFF350F45C94
:108950000FE2020EDB50300FE66E010EDB50EA6ACA
:10896000010FE96E020EEA22E552E750EF6E0ED0DB
:10897000020EDB50370FE66E010EDB50EA6A010F84
:10898000E96E020EEA22E552E750EF6E010EDB2A95
:10899000DF50EA6A000FE96E0D0EEA22EF500F0B6E
:1089A000E76E020EE7CFDBFF0A0EF36E020EDBCF9F
:1089B000F4FFF350F45C0FE2020EDB50300FE66E72
:1089C000010EDB50EA6A010FE96E020EEA22E5525F
:1089D000E750EF6E0ED0020EDB50370FE66E010E41
:1089E000DB50EA6A010FE96E020EEA22E552E75017
:1089F000EF6E010EDB2ADF2A94D7010EDB50EA6A04
:108A0000010FE96E020EEA221A0EEF6E010EDB284C
:108A10000201006F1DEC33F0030EE15C02E2E16A3B
:108A2000E552E16EE552E7CFD9FF12000201010ED7
:108A3000006F02011B0E016F1DEC33F012000201EA
:108A40000D0E006F0201410E016F0201540E026F04
:108A500002012B0E036F0201510E046F0201490E39
:108A6000056F0201460E066F0201470E076F0201F5
:108A7000430E086F02014E0E096F0201540E0A6F79
:108A800002013D0E0B6F0201300E0C6F02010D0E44
:108A90000D6F1DEC33F0120002010B0E006F02018E
:108AA000410E016F0201540E026F02012B0E036F83
:108AB0000201510E046F0201490E056F02014D0EB5
:108AC000066F0201550E076F0201580E086F020172
:108AD0003D0E096F0201300E0A6F02010D0E0B6F81
:108AE0001DEC33F0120002010C0E006F0201410E6A
:108AF000016F0201540E026F02012B0E036F02017F
:108B0000510E046F0201490E056F02014D0E066FF2
:108B100002014F0E076F0201440E086F0201450E5D
:108B2000096F02013D0E0A6F0201300E0B6F020148
:108B30000D0E0C6F1DEC33F0120002010D0E006FD4
:108B40000201410E016F0201540E026F02012B0E51
:108B5000036F0201510E046F0201490E056F0201FD
:108B6000440E066F02014E0E076F0201530E086F8E
:108B70000201490E096F0201500E0A6F02013D0EFB
:108B80000B6F0F0139B106D00201300E0C6F0F01CF
:108B9000399505D00201310E0C6F0F0139850201A4
:108BA0000D0E0D6F1DEC33F0120002010C0E006F64
:108BB0000201410E016F0201540E026F02012B0EE1
:108BC000036F0201510E046F0201490E056F02018D
:108BD000480E066F0201450E076F0201410E086F35
:108BE0000201440E096F02013D0E0A6F0201310EAF
:108BF0000B6F02010D0E0C6F1DEC33F01200D9CF7C
:108C0000E6FFE1CFD9FF040EE1260201410E016F1C
:108C10000201540E026F02012B0E036F0201510E6E
:108C2000046F0201490E056F0201430E066F020137
:108C3000530E076F0201470E086F0201500E096FB5
:108C400002013D0E0A6F0201310E0B6F02012C0E64
:108C50000C6F0201220E0D6FDE52200EDD6EDF6AF8
:108C6000010EDB50DF5C0EE2DF50EA6A000FE96EB6
:108C70000B0EEA22EF50FF0803E1010EDFCFDBFF0E
:108C8000DF2AEED7DF6A010EDB50DF5C14E2DF5033
:108C9000EA6A000FE96E0B0EEA22EF50E66E0D0E47
:108CA000DF24EA6A010FE96E020EEA22E552E7507C
:108CB000EF6EDF2AE8D7010EDB500D0FEA6A010FD5
:108CC000E96E020EEA22220EEF6E010EDB500E0F4D
:108CD000EA6A010FE96E020EEA222C0EEF6EFF0E19
:108CE0000B01205D67E0010EDB500F0FEA6A010FF8
:108CF000E96E020EEA22220EEF6E080EF36E020EED
:108D0000F3CFDBFFDF6A020EDB50DF5C0EE2DF50E9
:108D1000EA6A200FE96E0B0EEA22EF50FF0803E12A
:108D2000020EDFCFDBFFDF2AEED7010EDB50100F84
:108D3000E76E030EE7CFDBFFDF6A020EDB50DF5C7E
:108D400015E2DF50EA6A200FE96E0B0EEA22EF50BF
:108D5000E66E030EDB50DF24EA6A010FE96E020EB5
:108D6000EA22E552E750EF6EDF2AE7D7020EDBCFAB
:108D7000E6FF030EDB50E552E724E76E030EE7CF74
:108D8000DBFF030EDB50EA6A010FE96E020EEA22F6
:108D9000220EEF6E030EDB28EA6A010FE96E020E67
:108DA000EA222C0EEF6E030EDB28E76E030EE7CFF0
:108DB000DBFF11D0010EDB500F0FEA6A010FE96EE5
:108DC000020EEA222C0EEF6E010EDB500F0FE76E43
:108DD000030EE7CFDBFFFF0E0B01285D55E0030E0E
:108DE000DB28EA6A010FE96E020EEA22220EEF6E1C
:108DF000080EF36E020EF3CFDBFFDF6A020EDB50CC
:108E0000DF5C0EE2DF50EA6A280FE96E0B0EEA2201
:108E1000EF50FF0803E1020EDFCFDBFFDF2AEED7C2
:108E2000030EDB28E76E030EE7CFDBFFDF6A020EDF
:108E3000DB50DF5C15E2DF50EA6A280FE96E0B0EAB
:108E4000EA22EF50E66E030EDB50DF24EA6A010FE0
:108E5000E96E020EEA22E552E750EF6EDF2AE7D70D
:108E6000020EDBCFE6FF030EDB50E552E724E76E90
:108E7000030EE7CFDBFF030EDB50EA6A010FE96E5A
:108E8000020EEA22220EEF6E030EDB28EA6A010FC1
:108E9000E96E020EEA220D0EEF6E030EDB50020F9A
:108EA0000201006F1DEC33F0040EE15C02E2E16AA6
:108EB000E552E16EE552E7CFD9FF1200D9CFE6FFC8
:108EC000E1CFD9FF020EE1260201410E016F02013E
:108ED000540E026F02012B0E036F0201510E046F3C
:108EE0000201490E056F0201440E066F02014E0E8B
:108EF000076F0201530E086F0201430E096F020152
:108F0000460E0A6F0201470E0B6F02013D0E0C6FF9
:108F10000201220E0D6F010EDB6ADF50EA6A3F0F7D
:108F2000E96E0B0EEA22EF50FF082FE0DE520F0E23
:108F3000DD6EDF6A010EDB50DF5C0EE2DF50EA6AB5
:108F40003F0FE96E0B0EEA22EF50FF0803E1010E1E
:108F5000DFCFDBFFDF2AEED7DF6A010EDB50DF5CFD
:108F600014E2DF50EA6A3F0FE96E0B0EEA22EF507F
:108F7000E66E0D0EDF24EA6A010FE96E020EEA22A8
:108F8000E552E750EF6EDF2AE8D7010EDB500D0FF8
:108F9000EA6A010FE96E020EEA22220EEF6E010E5E
:108FA000DB500E0FE76E010EE7CFDBFF010EDB504B
:108FB000EA6A010FE96E020EEA220D0EEF6E010E53
:108FC000DB280201006F1DEC33F0020EE15C02E2CF
:108FD000E16AE552E16EE552E7CFD9FF12000201E6
:108FE0000A0E006F0201410E016F0201540E026F62
:108FF00002012B0E036F0201430E046F0201470EA4
:10900000056F0201410E066F0201540E076F020147
:10901000540E086F02013F0E096F02010D0E0A6F18
:109020001DEC33F0120002010C0E006F0201410E24
:10903000016F0201540E026F02012B0E036F020139
:10904000510E046F0201490E056F0201530E066FA7
:109050000201520E076F0201560E086F0201430E05
:10906000096F02013D0E0A6F0201310E0B6F020102
:109070000D0E0C6F1DEC33F01200D9CFE6FFE1CFDF
:10908000D9FF020EE1260401010EF26F0201410E2A
:10909000016F0201540E026F02012B0E036F0201D9
:1090A000510E046F0201490E056F02014F0E066F4B
:1090B0000201500E076F0201450E086F02014E0EAD
:1090C000096F02013D0E0A6F0201220E0B6F0201B1
:1090D000540E0C6F0201430E0D6F0201500E0E6F05
:1090E0000201220E0F6F02012C0E106F0201220EE0
:1090F000116F010EDB6A0F0139B134D0FF0E0B0185
:10910000305D2FE0DE520F0EDD6EDF6A010EDB50A8
:10911000DF5C0EE2DF50EA6A300FE96E0B0EEA22E6
:10912000EF50FF0803E1010EDFCFDBFFDF2AEED7B0
:10913000DF6A010EDB50DF5C14E2DF50EA6A300FB9
:10914000E96E0B0EEA22EF50E66E110EDF24EA6A9A
:10915000010FE96E020EEA22E552E750EF6EDF2AB8
:10916000E8D72FD0DE52200EDD6EDF6A010EDB5015
:10917000DF5C0EE2DF50EA6A4E0FE96E0B0EEA2268
:10918000EF50FF0803E1010EDFCFDBFFDF2AEED750
:10919000DF6A010EDB50DF5C14E2DF50EA6A4E0F3B
:1091A000E96E0B0EEA22EF50E66E110EDF24EA6A3A
:1091B000010FE96E020EEA22E552E750EF6EDF2A58
:1091C000E8D7010EDB50110FEA6A010FE96E020EBB
:1091D000EA22220EEF6E010EDB50120FEA6A010F37
:1091E000E96E020EEA222C0EEF6E010EDB50130F19
:1091F000E76E010EE7CFDBFFFF0E0B016E5D25E092
:10920000DF6A040EDF5C20E2DF50EA6A6E0FE96E6F
:109210000B0EEA22EF50FF0801E120D0DF50EA6A8E
:109220006E0FE96E0B0EEA22EF50E66E010EDB5078
:10923000EA6A010FE96E020EEA22E552E750EF6E8C
:10924000010EDB2ADF2ADDD709D0010EDB50EA6AE6
:10925000010FE96E020EEA22300EEF6E010EDB50B6
:10926000EA6A010FE96E020EEA220D0EEF6E010EA0
:10927000DB280201006F1DEC33F0020EE15C02E21C
:10928000E16AE552E16EE552E7CFD9FF1200D9CF8E
:10929000E6FFE1CFD9FF020EE1260401010EF26FD5
:1092A0000201410E016F0201540E026F02012B0EEA
:1092B000036F0201510E046F0201490E056F020196
:1092C0004F0E066F0201500E076F0201450E086F28
:1092D00002014E0E096F02013D0E0A6F0201220EBD
:1092E0000B6F0201540E0C6F0201430E0D6F020151
:1092F000500E0E6F0201220E0F6F02012C0E106F26
:109300000201220E116F010EDB6AFF0E0B01995D47
:109310002FE0DE520F0EDD6EDF6A010EDB50DF5CE8
:109320000EE2DF50EA6A990FE96E0B0EEA22EF5067
:10933000FF0803E1010EDFCFDBFFDF2AEED7DF6A94
:10934000010EDB50DF5C14E2DF50EA6A990FE96E30
:109350000B0EEA22EF50E66E110EDF24EA6A010FCF
:10936000E96E020EEA22E552E750EF6EDF2AE8D7F7
:10937000010EDB50110FEA6A010FE96E020EEA22BC
:10938000220EEF6E010EDB50120FEA6A010FE96E3A
:10939000020EEA222C0EEF6E010EDB50130FE76E69
:1093A000010EE7CFDBFFFF0E0B01A85D25E0DF6AB2
:1093B000040EDF5C20E2DF50EA6AA80FE96E0B0EB4
:1093C000EA22EF50FF0801E120D0DF50EA6AA80F3F
:1093D000E96E0B0EEA22EF50E66E010EDB50EA6AF0
:1093E000010FE96E020EEA22E552E750EF6E010E20
:1093F000DB2ADF2ADDD709D0010EDB50EA6A010F34
:10940000E96E020EEA22300EEF6E010EDB50EA6AC0
:10941000010FE96E020EEA220D0EEF6E010EDB283F
:109420000201006F1DEC33F0020EE15C02E2E16A22
:10943000E552E16EE552E7CFD9FF120002010A0EB4
:10944000006F0201410E016F0201540E026F020112
:109450002B0E036F0201510E046F0201490E056FBE
:109460000201530E066F0201450E076F02014E0EF8
:10947000086F0201440E096F02010D0E0A6F1DEC08
:1094800033F0120002010B0E006F0201410E016F5A
:109490000201540E026F02012B0E036F0201510EE6
:1094A000046F0201490E056F0201440E066F0201AE
:1094B000450E076F0201410E086F0201430E096F4E
:1094C0000201540E0A6F02010D0E0B6F1DEC33F0FA
:1094D0000401F26B12000201570E016F0201610ECE
:1094E000026F0201690E036F0201740E046F020124
:1094F000200E056F0201660E066F02016F0E076FE8
:109500000201720E086F0201200E096F0201680E3F
:109510000A6F0201650E0B6F0201780E0C6F0201DB
:109520002E0E0D6F02012E0E0E6F0201140E0F6F24
:1095300001010F0E736F0F0130BF03D0D7EC32F073
:109540000FD042EC7AF000090BE173C1E6FF010E87
:10955000E66E020EE66E4AEC7AF0E552E552E5520E
:1095600012000201430E016F0201530E026F02014D
:10957000200E036F0201450E046F0201520E056FAB
:109580000201520E066F0201140E076F0101070E51
:10959000736F0F0130BF03D0D7EC32F00FD042EC25
:1095A0007AF000090BE173C1E6FF010EE66E020ED0
:1095B000E66E4AEC7AF0E552E552E55212000201FD
:1095C000480E016F0201450E026F0201580E036F33
:1095D0000201200E046F0201530E056F0201490EB5
:1095E000066F02015A0E076F0201450E086F020155
:1095F000200E096F0201450E0A6F0201520E0B6F19
:109600000201520E0C6F0201140E0D6F01010D0EBE
:10961000736F0F0130BF03D0D7EC32F00FD042ECA4
:109620007AF000090BE173C1E6FF010EE66E020E4F
:10963000E66E4AEC7AF0E552E552E552120002017C
:10964000480E016F0201450E026F0201580E036FB2
:109650000201200E046F0201450E056F0201520E39
:10966000066F0201520E076F0201140E086F01010E
:10967000080E736F0F0130BF03D0D7EC32F00FD05C
:1096800042EC7AF000090BE173C1E6FF010EE66ED1
:10969000020EE66E4AEC7AF0E552E552E55212000F
:1096A0000201460E016F02016C0E026F0201610E93
:1096B000036F0201730E046F0201680E056F020151
:1096C000690E066F02016E0E076F0201670E086FCA
:1096D0000201210E096F0201440E0A6F02016F0E92
:1096E0000B6F02016E0E0C6F0201270E0D6F02014F
:1096F000740E0E6F0201200E0F6F0201700E106FBC
:1097000002016F0E116F0201770E126F0201650EDA
:10971000136F0201720E146F0201200E156F020109
:109720006F0E166F0201660E176F0201660E186F3C
:109730000201210E196F0201140E1A6F01011A0E97
:10974000736F0F0130BF03D0D7EC32F00FD042EC73
:109750007AF000090BE173C1E6FF010EE66E020E1E
:10976000E66E4AEC7AF0E552E552E552120002014B
:10977000430E016F02012F0E026F0F0130BF03D0A5
:10978000D7EC32F00FD042EC7AF000090BE173C154
:10979000E6FF010EE66E020EE66E4AEC7AF0E55246
:1097A000E552E55212000201760E016F02012E0E03
:1097B000026F0201340E036F0201310E046FFAC111
:1097C00005F2FBC106F202015F0E076F02016D0E8A
:1097D000086F02016F0E096F0201640E0A6F020129
:1097E000650E0B6F0201300E0C6F0201140E0D6F2F
:1097F00001010D0E736F0F0130BF03D0D7EC32F0B3
:109800000FD042EC7AF000090BE173C1E6FF010EC4
:10981000E66E020EE66E4AEC7AF0E552E552E5524B
:1098200012000201450E016F0201450E026F020196
:10983000200E036F0201450E046F0201520E056FE8
:109840000201520E066F0201140E076F0101070E8E
:10985000736F0F0130BF03D0D7EC32F00FD042EC62
:109860007AF000090BE173C1E6FF010EE66E020E0D
:10987000E66E4AEC7AF0E552E552E552120002013A
:10988000310E016F0201300E026F0201310E036FC3
:109890000201310E046F0201200E056F0201200E3D
:1098A000066F0201200E076F0201200E086F0201F1
:1098B000200E096F0201200E0A6F0201200E0B6FAD
:1098C0000201200E0C6F0201200E0D6F0201200E0E
:1098D0000E6F0201200E0F6F0201400E106F020189
:1098E000200E116F0201200E126F0201200E136F65
:1098F0000201200E146F0201140E156F0101150EE6
:10990000736F0F0130BF03D0D7EC32F00FD042ECB1
:109910007AF000090BE173C1E6FF010EE66E020E5C
:10992000E66E4AEC7AF0E552E552E5521200020189
:10993000310E016F0201300E026F0201310E036F12
:109940000201310E046F0201200E056F0201200E8C
:10995000066F0201200E076F0201200E086F020140
:10996000200E096F0201200E0A6F0201200E0B6FFC
:109970000201200E0C6F0201200E0D6F0201200E5D
:109980000E6F0201200E0F6F0201400E106F0201D8
:10999000200E116F0201200E126F0201200E136FB4
:1099A0000201200E146F0201140E156F02011A0E2F
:1099B000166F0101160E736FA6EC3AF01200020149
:1099C000430E016F0201550E026F02012D0E036F4F
:1099D0000201470E046F0201530E056F02014D0E86
:1099E000066F02012D0E076F0201320E086F020191
:1099F000200E096F0201760E0A6FFAC10BF2020106
:109A00002E0E0C6FFBC10DF20201140E0E6F010140
:109A10000E0E736F0F013CBF16D00F0130BF03D085
:109A2000D7EC32F00FD042EC7AF000090BE173C1B1
:109A3000E6FF010EE66E020EE66E4AEC7AF0E552A3
:109A4000E552E55207D002011A0E0F6F0101732B88
:109A5000A6EC3AF012000201430E016F0201530E10
:109A6000026F0201510E036F02013A0E046F0201F0
:109A7000200E056F0A0E0B01B45D0DE1B1CB06F2AD
:109A8000B2CB07F2B3CB08F20201140E096F010149
:109A9000090E736F37D00A0E0B01B55D0FE1B1CB24
:109AA00006F2B2CB07F2B3CB08F2B4CB09F2020153
:109AB000140E0A6F01010A0E736F24D00A0E0B01F7
:109AC000B65D11E1B1CB06F2B2CB07F2B3CB08F22F
:109AD000B4CB09F2B5CB0AF20201140E0B6F0101EF
:109AE0000B0E736F0FD00201300E066F02012C0EA9
:109AF000076F0201300E086F0201140E096F010199
:109B0000090E736F0F013CBF16D00F0130BF03D099
:109B1000D7EC32F00FD042EC7AF000090BE173C1C0
:109B2000E6FF010EE66E020EE66E4AEC7AF0E552B2
:109B3000E552E5520DD001017351EA6A010FE96E59
:109B4000020EEA221A0EEF6E0101732BA6EC3AF018
:109B500012000201730E016F0201650E026F020115
:109B6000740E036F0201200E046F02016F0E056F69
:109B700002016B0E066F0201140E076F0101070E42
:109B8000736F0F013CBF16D00F0130BF03D0D7EC6D
:109B900032F00FD042EC7AF000090BE173C1E6FF1E
:109BA000010EE66E020EE66E4AEC7AF0E552E552E0
:109BB000E55207D002011A0E086F0101732BA6ECC3
:109BC0003AF012000201630E016F02016C0E026F87
:109BD0000201650E036F0201610E046F0201720E35
:109BE000056F0201200E066F02016F0E076F020162
:109BF0006B0E086F0201140E096F0101090E736FDD
:109C00000F013CBF16D00F0130BF03D0D7EC32F0AC
:109C10000FD042EC7AF000090BE173C1E6FF010EB0
:109C2000E66E020EE66E4AEC7AF0E552E552E55237
:109C300007D002011A0E0A6F0101732BA6EC3AF04D
:109C400012000201730E016F0201790E026F020110
:109C50006E0E036F0201740E046F0201610E056F38
:109C60000201780E066F0201200E076F0201650ED9
:109C7000086F0201720E096F0201720E0A6F020173
:109C80006F0E0B6F0201720E0C6F0201140E0D6F3E
:109C900001010D0E736F0F013CBF16D00F0130BFD5
:109CA00003D0D7EC32F00FD042EC7AF000090BE190
:109CB00073C1E6FF010EE66E020EE66E4AEC7AF024
:109CC000E552E552E55207D002011A0E0E6F01016E
:109CD000732BA6EC3AF012000201740E016F020120
:109CE000650E026F02016C0E036F0201650E046FB8
:109CF0000201700E056F0201680E066F02016F0E01
:109D0000076F02016E0E086F0201650E096F0201F6
:109D1000200E0A6F02016E0E0B6F0201750E0C6FA2
:109D200002016D0E0D6F0201620E0E6F0201650ED3
:109D30000F6F0201720E106F0201200E116F0201EF
:109D4000650E126F0201720E136F0201720E146F14
:109D500002016F0E156F0201720E166F0201140ED2
:109D6000176F0101170E736F0F013CBF16D00F0163
:109D700030BF03D0D7EC32F00FD042EC7AF00009BC
:109D80000BE173C1E6FF010EE66E020EE66E4AECD1
:109D90007AF0E552E552E55207D002011A0E186F2B
:109DA0000101732BA6EC3AF0120002016D0E016F57
:109DB0000201650E026F02016D0E036F02016F0E4C
:109DC000046F0201720E056F0201790E066F020127
:109DD000200E076F0201660E086F0201750E096FF3
:109DE00002016C0E0A6F02016C0E0B6F0201140E61
:109DF0000C6F01010C0E736F0F013CBF16D00F01E9
:109E000030BF03D0D7EC32F00FD042EC7AF000092B
:109E10000BE173C1E6FF010EE66E020EE66E4AEC40
:109E20007AF0E552E552E55207D002011A0E0D6FA5
:109E30000101732BA6EC3AF012000201310E016F02
:109E40000201300E026F0201310E036F0201310E6A
:109E5000046F0201200E056F0201200E066F020141
:109E6000200E076F0201200E086F0201200E096FFD
:109E70000201200E0A6F0201300E0B6F0201300E3C
:109E80000C6F0201300E0D6F0201300E0E6F0201D9
:109E9000200E0F6F0201540E106F0201200E116F81
:109EA0000201200E126F0201350E136F0201300EF7
:109EB000146F0201140E156F0101150E736F0F015F
:109EC0003CBF16D00F0130BF03D0D7EC32F00FD01B
:109ED00042EC7AF000090BE173C1E6FF010EE66E79
:109EE000020EE66E4AEC7AF0E552E552E55207D0F2
:109EF00002011A0E166F0101732BA6EC3AF0120044
:109F00000201310E016F0201300E026F0201310EAB
:109F1000036F0201310E046F0201200E056F020172
:109F2000200E066F0201200E076F0201200E086F3F
:109F30000201200E096F0201200E0A6F0201300E8D
:109F40000B6F0201300E0C6F0201300E0D6F02011B
:109F5000300E0E6F0201200E0F6F0201410E106FC6
:109F60000201200E116F0201200E126F0201310E4C
:109F7000136F0201330E146F0201140E156F0101ED
:109F8000150E736F0F0130BF03D0D7EC32F00FD036
:109F900042EC7AF000090BE173C1E6FF010EE66EB8
:109FA000020EE66E4AEC7AF0E552E552E5521200F6
:109FB0000201310E016F0201300E026F0201310EFB
:109FC000036F0201310E046F0201200E056F0201C2
:109FD000200E066F0201200E076F0201200E086F8F
:109FE0000201200E096F0201200E0A6F0201300EDD
:109FF0000B6F0201300E0C6F0201300E0D6F02016B
:10A00000300E0E6F0201200E0F6F0201520E106F04
:10A010000201200E116F0201200E126F0201310E9B
:10A02000136F0201340E146F0201140E156F01013B
:10A03000150E736F0F0130BF03D0D7EC32F00FD085
:10A0400042EC7AF000090BE173C1E6FF010EE66E07
:10A05000020EE66E4AEC7AF0E552E552E552120045
:10A060000201310E016F0201300E026F0201310E4A
:10A07000036F0201310E046F0201200E056F020111
:10A08000200E066F0201200E076F0201200E086FDE
:10A090000201200E096F0201200E0A6F0201300E2C
:10A0A0000B6F0201300E0C6F0201300E0D6F0201BA
:10A0B000300E0E6F0201200E0F6F0201520E106F54
:10A0C0000201200E116F0201200E126F0201350EE7
:10A0D000136F0201300E146F0201140E156F01018F
:10A0E000150E736F0F013CBF16D00F0130BF03D0A8
:10A0F000D7EC32F00FD042EC7AF000090BE173C1DB
:10A10000E6FF010EE66E020EE66E4AEC7AF0E552CC
:10A11000E552E55207D002011A0E166F0101732BAA
:10A12000A6EC3AF012000201310E016F0201300E6E
:10A13000026F0201310E036F0201310E046F020142
:10A14000200E056F0201200E066F0201200E076F20
:10A150000201200E086F0201200E096F0201200E7D
:10A160000A6F0201300E0B6F0201300E0C6F0201FC
:10A17000300E0D6F0201300E0E6F0201200E0F6FB8
:10A180000201410E106F0201200E116F0201200E1C
:10A19000126F0201320E136F0201300E146F0201B2
:10A1A000140E156F0101150E736F0F013CBF16D011
:10A1B0000F0130BF03D0D7EC32F00FD042EC7AF071
:10A1C00000090BE173C1E6FF010EE66E020EE66EBA
:10A1D0004AEC7AF0E552E552E55207D002011A0E38
:10A1E000166F0101732BA6EC3AF012000201310E3A
:10A1F000016F0201300E026F0201310E036F020186
:10A20000310E046F0201200E056F0201200E066F51
:10A210000201200E076F0201200E086F0201200EBE
:10A22000096F0201200E0A6F0201300E0B6F02014E
:10A23000300E0C6F0201300E0D6F0201300E0E6FEA
:10A240000201200E0F6F0201520E106F0201200E4C
:10A25000116F0201200E126F0201330E136F020103
:10A26000300E146F0201140E156F0101150E736F7D
:10A270000F013CBF16D00F0130BF03D0D7EC32F036
:10A280000FD042EC7AF000090BE173C1E6FF010E3A
:10A29000E66E020EE66E4AEC7AF0E552E552E552C1
:10A2A00007D002011A0E166F0101732BA6EC3AF0CB
:10A2B00012000201310E016F0201300E026F020125
:10A2C000310E036F0201310E046F0201200E056F83
:10A2D0000201200E066F0201200E076F0201200E00
:10A2E000086F0201200E096F0201200E0A6F0201A1
:10A2F000300E0B6F0201300E0C6F0201300E0D6F2D
:10A300000201300E0E6F0201200E0F6F0201540E7B
:10A31000106F0201200E116F0201200E126F020158
:10A32000340E136F0201300E146F0201140E156FFC
:10A330000101150E736F0F013CBF16D00F0130BF26
:10A3400003D0D7EC32F00FD042EC7AF000090BE1E9
:10A3500073C1E6FF010EE66E020EE66E4AEC7AF07D
:10A36000E552E552E55207D002011A0E166F0101BF
:10A37000732BA6EC3AF012000201310E016F0201BC
:10A38000300E026F0201310E036F0201310E046FB5
:10A390000201200E056F0201200E066F0201200E41
:10A3A000076F0201200E086F0201200E096F0201E3
:10A3B000200E0A6F0201300E0B6F0201300E0C6F7F
:10A3C0000201300E0D6F0201300E0E6F0201200EE1
:10A3D0000F6F0201540E106F0201200E116F020167
:10A3E000200E126F0201380E136F0201370E146F28
:10A3F0000201140E156F0101150E736F0F013CBFA2
:10A4000016D00F0130BF03D0D7EC32F00FD042ECA2
:10A410007AF000090BE173C1E6FF010EE66E020E51
:10A42000E66E4AEC7AF0E552E552E55207D00201B9
:10A430001A0E166F0101732BA6EC3AF012000301FD
:10A44000FC5100081DE20301FD6B0301FC510301F7
:10A45000FD5D16E20301FD51EA6A000FE96E030E8D
:10A46000EA22EF50E66E0301FD51EA6A010FE96E40
:10A47000020EEA22E552E750EF6E0301FD2BE5D70D
:10A480000F012D830301FC51EA6A010FE96E020EF0
:10A49000EA22140EEF6E0301FC290101736F0F0114
:10A4A0003CBF16D00F0130BF03D0D7EC32F00FD035
:10A4B00042EC7AF000090BE173C1E6FF010EE66E93
:10A4C000020EE66E4AEC7AF0E552E552E5520DD006
:10A4D00001017351EA6A010FE96E020EEA221A0EB7
:10A4E000EF6E0101732BA6EC3AF012000201310E5F
:10A4F000016F0201300E026F0201310E036F020183
:10A50000310E046F0201200E056F0201200E066F4E
:10A510000201200E076F0201200E086F0201200EBB
:10A52000096F0201200E0A6F0201300E0B6F02014B
:10A53000300E0C6F0201300E0D6F0201300E0E6FE7
:10A540000201200E0F6F0201540E106F0201200E47
:10A55000116F0201200E126F0201360E136F0201FD
:10A56000300E146F0201140E156F0101150E736F7A
:10A570000F013CBF16D00F0130BF03D0D7EC32F033
:10A580000FD042EC7AF000090BE173C1E6FF010E37
:10A59000E66E020EE66E4AEC7AF0E552E552E552BE
:10A5A00007D002011A0E166F0101732BA6EC3AF0C8
:10A5B00012000201310E016F0201300E026F020122
:10A5C000310E036F0201310E046F0201200E056F80
:10A5D0000201200E066F0201200E076F0201200EFD
:10A5E000086F0201200E096F0201200E0A6F02019E
:10A5F000300E0B6F0201300E0C6F0201300E0D6F2A
:10A600000201300E0E6F0201200E0F6F0201520E7A
:10A61000106F0201200E116F0201200E126F020155
:10A62000370E136F0201300E146F0201140E156FF6
:10A630000101150E736F0F013CBF16D00F0130BF23
:10A6400003D0D7EC32F00FD042EC7AF000090BE1E6
:10A6500073C1E6FF010EE66E020EE66E4AEC7AF07A
:10A66000E552E552E55207D002011A0E166F0101BC
:10A67000732BA6EC3AF012000201310E016F0201B9
:10A68000300E026F0201310E036F0201310E046FB2
:10A690000201200E056F0201200E066F0201200E3E
:10A6A000076F0201200E086F0201200E096F0201E0
:10A6B000200E0A6F0201300E0B6F0201300E0C6F7C
:10A6C0000201300E0D6F0201300E0E6F0201200EDE
:10A6D0000F6F0201540E106F0201200E116F020164
:10A6E000200E126F0201370E136F0201300E146F2D
:10A6F0000201140E156F0101150E736F0F013CBF9F
:10A7000016D00F0130BF03D0D7EC32F00FD042EC9F
:10A710007AF000090BE173C1E6FF010EE66E020E4E
:10A72000E66E4AEC7AF0E552E552E55207D00201B6
:10A730001A0E166F0101732BA6EC3AF012000201FB
:10A74000310E016F0201300E026F0201310E036FF4
:10A750000201310E046F0201200E056F0201200E6E
:10A76000066F0201200E076F0201200E086F020122
:10A77000200E096F0201200E0A6F0201300E0B6FCE
:10A780000201300E0C6F0201300E0D6F0201300E0F
:10A790000E6F0201200E0F6F0201540E106F0201A6
:10A7A000200E116F0201200E126F0201380E136F7E
:10A7B0000201300E146F0201140E156F0101150E07
:10A7C000736F0F013CBF16D00F0130BF03D0D7EC21
:10A7D00032F00FD042EC7AF000090BE173C1E6FFD2
:10A7E000010EE66E020EE66E4AEC7AF0E552E55294
:10A7F000E55207D002011A0E166F0101732BA6EC69
:10A800003AF012000201310E016F0201300E026FA8
:10A810000201310E036F0201310E046F0201200E9E
:10A82000056F0201200E066F0201200E076F020164
:10A83000200E086F0201200E096F0201200E0A6F20
:10A840000201300E0B6F0201300E0C6F0201300E50
:10A850000D6F0201300E0E6F0201200E0F6F02010C
:10A86000540E106F0201200E116F0201200E126FA4
:10A870000201380E136F0201310E146F0201140E23
:10A88000156F0101150E736F0F013CBF16D00F013C
:10A8900030BF03D0D7EC32F00FD042EC7AF0000991
:10A8A0000BE173C1E6FF010EE66E020EE66E4AECA6
:10A8B0007AF0E552E552E55207D002011A0E166F02
:10A8C0000101732BA6EC3AF012000201310E016F68
:10A8D0000201300E026F0201310E036F0201310ED0
:10A8E000046F0201200E056F0201200E066F0201A7
:10A8F000200E076F0201200E086F0201200E096F63
:10A900000201200E0A6F0201300E0B6F0201300EA1
:10A910000C6F0201300E0D6F0201300E0E6F02013E
:10A92000200E0F6F0201520E106F0201200E116FE8
:10A930000201200E126F0201380E136F0201320E57
:10A94000146F0201140E156F0101150E736F0F01C4
:10A950003CBF16D00F0130BF03D0D7EC32F00FD080
:10A9600042EC7AF000090BE173C1E6FF010EE66EDE
:10A97000020EE66E4AEC7AF0E552E552E55207D057
:10A9800002011A0E166F0101732BA6EC3AF01200A9
:10A990000201310E016F0201300E026F0201310E11
:10A9A000036F0201310E046F0201200E056F0201D8
:10A9B000200E066F0201200E076F0201200E086FA5
:10A9C0000201200E096F0201200E0A6F0201300EF3
:10A9D0000B6F0201300E0C6F0201300E0D6F020181
:10A9E000300E0E6F0201200E0F6F0201540E106F19
:10A9F0000201200E116F0201200E126F0201380EAB
:10AA0000136F0201330E146F0201140E156F010152
:10AA1000150E736F0F013CBF16D00F0130BF03D06E
:10AA2000D7EC32F00FD042EC7AF000090BE173C1A1
:10AA3000E6FF010EE66E020EE66E4AEC7AF0E55293
:10AA4000E552E55207D002011A0E166F0101732B71
:10AA5000A6EC3AF012000201310E016F0201300E35
:10AA6000026F0201310E036F0201310E046F020109
:10AA7000200E056F0201200E066F0201200E076FE7
:10AA80000201200E086F0201200E096F0201200E44
:10AA90000A6F0201300E0B6F0201300E0C6F0201C3
:10AAA000300E0D6F0201300E0E6F0201200E0F6F7F
:10AAB0000201520E106F0201200E116F0201200ED2
:10AAC000126F0201380E136F0201340E146F02016F
:10AAD000140E156F0101150E736F0F013CBF16D0D8
:10AAE0000F0130BF03D0D7EC32F00FD042EC7AF038
:10AAF00000090BE173C1E6FF010EE66E020EE66E81
:10AB00004AEC7AF0E552E552E55207D002011A0EFE
:10AB1000166F0101732BA6EC3AF012000201310E00
:10AB2000016F0201300E026F0201310E036F02014C
:10AB3000310E046F0201200E056F0201200E066F18
:10AB40000201200E076F0201200E086F0201200E85
:10AB5000096F0201200E0A6F0201300E0B6F020115
:10AB6000300E0C6F0201300E0D6F0201300E0E6FB1
:10AB70000201200E0F6F0201540E106F0201200E11
:10AB8000116F0201200E126F0201380E136F0201C5
:10AB9000350E146F0201140E156F0101150E736F3F
:10ABA0000F013CBF16D00F0130BF03D0D7EC32F0FD
:10ABB0000FD042EC7AF000090BE173C1E6FF010E01
:10ABC000E66E020EE66E4AEC7AF0E552E552E55288
:10ABD00007D002011A0E166F0101732BA6EC3AF092
:10ABE00012000201310E016F0201300E026F0201EC
:10ABF000310E036F0201310E046F0201200E056F4A
:10AC00000201200E066F0201200E076F0201200EC6
:10AC1000086F0201200E096F0201200E0A6F020167
:10AC2000300E0B6F0201300E0C6F0201300E0D6FF3
:10AC30000201300E0E6F0201200E0F6F0201520E44
:10AC4000106F0201200E116F0201200E126F02011F
:10AC5000380E136F0201360E146F0201140E156FB9
:10AC60000101150E736F0F013CBF16D00F0130BFED
:10AC700003D0D7EC32F00FD042EC7AF000090BE1B0
:10AC800073C1E6FF010EE66E020EE66E4AEC7AF044
:10AC9000E552E552E55207D002011A0E166F010186
:10ACA000732BA6EC3AF012000201060E016F0201AE
:10ACB000140E026F0101020E736F0F013CBF16D01C
:10ACC0000F0130BF03D0D7EC32F00FD042EC7AF056
:10ACD00000090BE173C1E6FF010EE66E020EE66E9F
:10ACE0004AEC7AF0E552E552E55207D002011A0E1D
:10ACF000036F0101732BA6EC3AF00F013D9D2EEC82
:10AD00000CF02EEC0CF012000201150E016F020186
:10AD1000140E026F0101020E736F0F013CBF16D0BB
:10AD20000F0130BF03D0D7EC32F00FD042EC7AF0F5
:10AD300000090BE173C1E6FF010EE66E020EE66E3E
:10AD40004AEC7AF0E552E552E55207D002011A0EBC
:10AD5000036F0101732BA6EC3AF00F013D9D2EEC21
:10AD60000CF02EEC0CF012000C01FE6B0B0E0C0123
:10AD7000FE5D0BE20C01FE51EA6A200FE96E010E46
:10AD8000EA22EF680C01FE2BF1D70101DF050C016F
:10AD9000FD6F0101DF0507E12B0E0F01025D02E0EF
:10ADA00002CF20F132D00C01FF6BFDCCFEFC0C0178
:10ADB000FE5100081DE20C01FE51EA6A020FE96E25
:10ADC0000F0EEA22EF50E66E0C01FF51EA6A200FE7
:10ADD000E96E010EEA22E552E750EF6E0C01FF2BFF
:10ADE0000B0E0C01FF5D01E110D00C01FE07DFD757
:10ADF0002B0E0F01025D09E00C01FF51EA6A200FE2
:10AE0000E96E010EEA2202CFEFFF0C01A00EF16FF6
:10AE10000C01B00EF26F0C01F36BF2CC12FF3CECA4
:10AE20003EF0F3CF13FF010120510F01135D07E046
:10AE3000240E0F01135D02E1DBD001D0C3D00C0161
:10AE4000F22B3CEC3EF0F3CF13FF010121510F0137
:10AE5000135D01E0B7D00C01F22B3CEC3EF0F3CFD8
:10AE600013FF010122510F01135D01E0ABD00C0172
:10AE7000F22B3CEC3EF0F3CF13FF010123510F0105
:10AE8000135D01E09FD00C01F22B3CEC3EF0F3CFC0
:10AE900013FF010124510F01135D01E093D00C0158
:10AEA000F22B3CEC3EF0F3CF13FF010125510F01D3
:10AEB000135D01E087D00C01F22B3CEC3EF0F3CFA8
:10AEC00013FF010126510F01135D01E07BD00C013E
:10AED000F22B3CEC3EF0F3CF13FF010127510F01A1
:10AEE000135D01E06FD00C01F22B3CEC3EF0F3CF90
:10AEF00013FF010128510F01135D01E063D00C0124
:10AF0000F22B3CEC3EF0F3CF13FF010129510F016E
:10AF1000135D01E057D00C01F22B3CEC3EF0F3CF77
:10AF200013FF01012A510F01135D01E04BD00C0109
:10AF3000F22B3CEC3EF0F3CF00F10C01F22B3CEC99
:10AF40003EF0F3CF01F10C01F22B3CEC3EF0F3CFDD
:10AF500002F10C01F22B3CEC3EF0F3CF03F1FF0EBB
:10AF60000101035D28E1FF0E0101025D1BE1FF0EFF
:10AF70000101015D0CE100C103F10101300E026F1E
:10AF80000101300E016F0101300E006F0AD001C1C6
:10AF900003F100C102F10101300E016F0101300E19
:10AFA000006F09D002C103F101C102F100C101F13A
:10AFB0000101300E006F0C01F22B3CEC3EF0F3CFA0
:10AFC00017FFE5D01F0E0C01F35D05E1E00E0F0148
:10AFD000125D01E10DD0100E0F0112250C01F26F70
:10AFE000F2CC12FF0C01F25102E10C01F32B17D746
:10AFF0000F012EA19DD00201550E016F0201300EEE
:10B00000026F0201310E036F0201310E046F020163
:10B01000200E056F0201200E066F0201300E076F31
:10B020000201300E086F0201300E096F0201300E6E
:10B030000A6F0C010A0EFF6F2B0E0F01025D04E177
:10B040000C01010EFD6F02D00C01FD6B0101DF51FF
:10B0500022E00101DF051FE0FDCCFEFC0101DF5114
:10B060000C01FE5D18E20C01FE51EA6A020FE96E66
:10B070000F0EEA22EF50E66E0C01FF51EA6A010F53
:10B08000E96E020EEA22E552E750EF6E0C01FF2B4B
:10B090000C01FE2BE3D7FFCCFEFC1C0E0C01FE5D69
:10B0A0000CE20C01FE51EA6A010FE96E020EEA227F
:10B0B000460EEF6E0C01FE2BF0D70201140E1D6F31
:10B0C00001011D0E736F0F013CBF16D00F0130BF81
:10B0D00003D0D7EC32F00FD042EC7AF000090BE14C
:10B0E00073C1E6FF010EE66E020EE66E4AEC7AF0E0
:10B0F000E552E552E55207D002011A0E1E6F01011A
:10B10000732BA6EC3AF00F010F013C51800B05E0C8
:10B110000F010F013D51400B0BE0AAEC31F00F0184
:10B12000299B0F0130A702D0ADEC18F00F013D9D17
:10B130000C01FF6B0C01FF6B0101DF6B0C01FE6B5F
:10B14000100E0C01FE5D0BE20C01FE51EA6A020FCB
:10B15000E96E0F0EEA22EF6A0C01FE2BF1D759ECD3
:10B1600051F00F010F013C51800B05E00F010F0161
:10B170003D51400B0BE0AAEC31F00F01299B0F0170
:10B1800030A702D0ADEC18F00F013D9D07D10F01A3
:10B190002EA1BDD000C110F101C111F102C112F107
:10B1A00003C113F1DFC114F10101550E156F010147
:10B1B000145101E195D00101140501E191D00C0178
:10B1C000060EFD6F2B0E0F01025D45E10C01010E15
:10B1D000FE6F0101DF510C01FE5D3CE2010E0C012E
:10B1E000FE150C01FF6F0C01FE51EA6A020FE96EB9
:10B1F0000F0EEA22EF50D00F0C01FC6F0C01FF5133
:10B200000FE00C01FC39F00BE66E0C01FD51EA6A0F
:10B21000100FE96E010EEA22E552E750EF6E17D0EB
:10B220000C01FD51EA6A100FE96E010EEA22EF509F
:10B230000C01FC25E66E0C01FD51EA6A100FE96E67
:10B24000010EEA22E552E750EF6E0C01FD2B0C01D6
:10B25000FE2BBFD745D00101142B0C01FE6B010161
:10B26000DF510C01FE5D3CE2010E0C01FE150C01EC
:10B27000FF6F0C01FE51EA6A020FE96E0F0EEA221F
:10B28000EF50D00F0C01FC6F0C01FF510FE10C01CE
:10B29000FC39F00BE66E0C01FD51EA6A100FE96E05
:10B2A000010EEA22E552E750EF6E17D00C01FD5176
:10B2B000EA6A100FE96E010EEA22EF500C01FC253C
:10B2C000E66E0C01FD51EA6A100FE96E010EEA22EA
:10B2D000E552E750EF6E0C01FD2B0C01FE2BBFD7A2
:10B2E0003AEC30F00101E62B400E0101E65D02E18F
:10B2F0000101E66B0101E8510101E65D08E1010190
:10B30000E82B400E0101E85D02E10101E86B01015B
:10B31000DF6B0C01FE6B100E0C01FE5D0BE20C01ED
:10B32000FE51EA6A020FE96E0F0EEA22EF6A0C0183
:10B33000FE2BF1D70101310E046F0101380E056FAC
:10B340000101310E066F14CF07F115CF08F116CFAA
:10B3500009F10101300E0A6F0101300E0B6F01017E
:10B36000300E0C6F0101300E0D6F17CF0EF17DEC1A
:10B370002FF00101E62B400E0101E65D02E1010123
:10B38000E66B0101E8510101E65D08E10101E82BEE
:10B39000400E0101E85D02E10101E86B12000C01C1
:10B3A000A00EF16F0C01B00EF26F0C01F36B0F01E8
:10B3B00018690F0119690F011A690F011B690F0143
:10B3C0001C690F011D690F011E690F011F690F0123
:10B3D00020690F0121690F0122690F0123690F0103
:10B3E00024690F0125690F0126690F0127696AEC9D
:10B3F0003EF01F0E0C01F35D0FE1E00E0C01F25D5B
:10B400000BE10C01B00EF26F0C01F36B0C01240E7A
:10B41000F66F58EC3EF00BD0100E0C01F2250C012B
:10B42000F26F0C01F25102E10C01F32BE0D7120094
:10B430000C01A00EF16F0C01B00EF26F0C01F36B5A
:10B44000F2CC12FF3CEC3EF0F3CF13FF0F0118518A
:10B450000F01135D07E0240E0F01135D02E1B7D069
:10B4600001D07BD00C01F22B3CEC3EF0F3CF13FF6C
:10B470000F0119510F01135D01E06FD00C01F22B88
:10B480003CEC3EF0F3CF13FF0F011A510F01135D97
:10B4900001E063D00C01F22B3CEC3EF0F3CF13FF44
:10B4A0000F011B510F01135D01E057D00C01F22B6E
:10B4B0003CEC3EF0F3CF13FF0F011C510F01135D65
:10B4C00001E04BD00C01F22B3CEC3EF0F3CF13FF2C
:10B4D0000F011D510F01135D01E03FD00C01F22B54
:10B4E0003CEC3EF0F3CF13FF0F011E510F01135D33
:10B4F00001E033D00C01F22B3CEC3EF0F3CF13FF14
:10B500000F011F510F01135D01E027D00C01F22B39
:10B510003CEC3EF0F3CF13FF0F0120510F01135D00
:10B5200001E01BD00C01F22B3CEC3EF0F3CF13FFFB
:10B530000F0121510F01135D01E00FD00C01F22B1F
:10B540003CEC3EF0F3CF13FF0F0122510F01135DCE
:10B5500001E003D00F01388D4FD01F0E0C01F35DB9
:10B5600005E1E00E0F01125D01E10DD0100E0F019B
:10B5700012250C01F26FF2CC12FF0C01F25102E124
:10B580000C01F32B5FD70C01B00EF26F0C01F36BC3
:10B590003CEC3EF0F3CF13FFFF0E0F01135D01E112
:10B5A00016D01F0E0C01F35D07E1E00E0C01F25DF9
:10B5B00003E10F01388B20D0100E0C01F2250C0195
:10B5C000F26F0C01F25102E10C01F32BE1D76AECAE
:10B5D0003EF0100E0C01F2250C01F26F0C01F2513D
:10B5E00002E10C01F32B0C01240EF66F58EC3EF037
:10B5F0000C01F26B0C01F36B1200D9CFE6FFE1CF27
:10B60000D9FF090EE126BB0E0101055D01E0D8D08E
:10B610000201550E016F0201300E026F0201310E60
:10B62000036F0201310E046F00C105F201C106F281
:10B6300002C107F203C108F20EC109F20FC10AF2FA
:10B64000060EF36E060EF3CFDBFF0A0EF36E070E47
:10B65000F3CFDBFF0101045172E0010104056FE04B
:10B6600001010405E76E040EE7CFDBFF030EDB6A82
:10B67000040EDB50F36E030EDBCFF4FFF350F45CEB
:10B680005EE2030EDB50010BE76E050EE7CFDBFF3A
:10B69000050EDB5032E1060EDB50EA6A000FE96E60
:10B6A000010EEA22EF50F00BE76E080EE7CFDBFF4A
:10B6B000080EDB380F0BE66E070EDB50EA6A010F4F
:10B6C000E96E020EEA22E552E750EF6E070EDB50FC
:10B6D000EA6A010FE96E020EEA22EF50300FE66EC1
:10B6E000070EDB50EA6A010FE96E020EEA22E5520C
:10B6F000E750EF6E070EDB2A1FD0060EDB50EA6A1A
:10B70000000FE96E010EEA22EF500F0BE76E080EF4
:10B71000E7CFDBFF080EDB50300FE66E070EDB5085
:10B72000EA6A010FE96E020EEA22E552E750EF6E77
:10B73000070EDB2A060EDB2A030EDB2A99D7070E3B
:10B74000DB50E76E030EE7CFDBFF1C0EF36E030E3C
:10B75000DBCFF4FFF350F45C0CE2030EDB50EA6A3B
:10B76000010FE96E020EEA22460EEF6E030EDB2A8F
:10B77000ECD70201140E1D6F01011D0E736F0F0136
:10B780003CBF16D00F0130BF03D0D7EC32F00FD042
:10B7900042EC7AF000090BE173C1E6FF010EE66EA0
:10B7A000020EE66E4AEC7AF0E552E552E55207D019
:10B7B00002011A0E1E6F0101732BA6EC3AF006D39C
:10B7C000550E0101055D01E0DAD00201550E016F51
:10B7D0000201300E026F0201310E036F0201310EC1
:10B7E000046F0201200E056F0201200E066F00C1DA
:10B7F00007F201C108F202C109F203C10AF2060E02
:10B80000F36E060EF3CFDBFF0A0EF36E070EF3CFD7
:10B81000DBFF0101045172E0010104056FE0010149
:10B820000405E76E040EE7CFDBFF030EDB6A040EB0
:10B83000DB50F36E030EDBCFF4FFF350F45C5EE2FB
:10B84000030EDB50010BE76E050EE7CFDBFF050EA5
:10B85000DB5032E1060EDB50EA6A000FE96E010EA2
:10B86000EA22EF50F00BE76E080EE7CFDBFF080E81
:10B87000DB380F0BE66E070EDB50EA6A010FE96E4C
:10B88000020EEA22E552E750EF6E070EDB50EA6A3D
:10B89000010FE96E020EEA22EF50300FE66E070E3E
:10B8A000DB50EA6A010FE96E020EEA22E552E75028
:10B8B000EF6E070EDB2A1FD0060EDB50EA6A000F80
:10B8C000E96E010EEA22EF500F0BE76E080EE7CF8C
:10B8D000DBFF080EDB50300FE66E070EDB50EA6A26
:10B8E000010FE96E020EEA22E552E750EF6E070EF5
:10B8F000DB2A060EDB2A030EDB2A99D7070EDB5064
:10B90000E76E030EE7CFDBFF1C0EF36E030EDBCFFB
:10B91000F4FFF350F45C0CE2030EDB50EA6A010F13
:10B92000E96E020EEA22460EEF6E030EDB2AECD71A
:10B930000201140E1D6F01011D0E736F0F013CBF3C
:10B9400016D00F0130BF03D0D7EC32F00FD042EC4D
:10B950007AF000090BE173C1E6FF010EE66E020EFC
:10B96000E66E4AEC7AF0E552E552E55207D0020164
:10B970001A0E1E6F0101732BA6EC3AF027D2380E77
:10B980000101055D47E10201350E016F0201300E34
:10B99000026F0201310E036F0201310E046F0201CA
:10B9A000200E056F0201310E066F0201380E076F7F
:10B9B00000C108F201C109F202C10AF203C10BF28F
:10B9C000310E0101065D04E10201450E0C6F03D04A
:10B9D0000201520E0C6F07C10DF208C10EF209C12F
:10B9E0000FF20AC110F20BC111F20CC112F20DC11B
:10B9F00013F20EC114F20201140E156F0101150E9F
:10BA0000736F0F013CAF05D002011A0E166F0101D2
:10BA1000732BC1D10F0E01010515DF6E090EDF5C1E
:10BA200070E10201350E016F0201300E026F02015A
:10BA3000310E036F0201310E046F0201200E056FFB
:10BA40000201310E066F0201380E076F00C108F2C5
:10BA500001C109F202C10AF203C10BF2310E010168
:10BA6000065D04E10201450E0C6F03D00201520E87
:10BA70000C6F07C10DF208C10EF209C10FF20AC125
:10BA800010F20BC111F20CC112F2F00E01010D15F2
:10BA9000E76E010EE7CFDBFF010EDB380F0BE76E21
:10BAA000020EE7CFDBFF0A0EF36E020EDBCFF4FFD0
:10BAB000F350F45C06E2020EDB50300F0201136F0C
:10BAC00005D0020EDB50370F0201136F0F0E01017C
:10BAD0000D15E76E010EE7CFDBFF0A0EF36E010EC8
:10BAE000DBCFF4FFF350F45C06E2010EDB50300FC5
:10BAF0000201146F05D0010EDB50370F0201146FE5
:10BB000067D00A0EDF5C31E10201330E016F0201E2
:10BB1000300E026F0201310E036F0201310E046F0D
:10BB20000201200E056F0201200E066F0201200E99
:10BB3000076F0201200E086F00C109F201C10AF26D
:10BB400002C10BF203C10CF206C10DF207C10EF2E5
:10BB500008C10FF209C110F20AC111F20BC112F2B1
:10BB60000CC113F20DC114F233D00201310E016F7A
:10BB70000201300E026F0201310E036F0201310E1D
:10BB8000046F0201200E056F0201200E066F0201F4
:10BB9000200E076F0201200E086F0201200E096FB0
:10BBA0000201200E0A6F00C10BF201C10CF202C1AA
:10BBB0000DF203C10EF20201200E0F6F06C110F24A
:10BBC00007C111F208C112F209C113F20AC114F23D
:10BBD0000F012EA90FD00201140E156F0101150ED1
:10BBE000736F0F013CAF05D002011A0E166F0101F1
:10BBF000732BD1D07C0E01010415E76E020EE7CF46
:10BC0000DBFF020EDB40E8403F0BDF6E010EDB6A1C
:10BC1000DF50090806E20A0EDF5CDF6E010EDB2A48
:10BC2000F7D7010EDB50300F0201156F300EDF2405
:10BC30000201166F02013A0E176FF00E0101051591
:10BC4000E76E020EE7CFDBFF020EDB380F0BDF6E75
:10BC5000030E01010415E76E020EE7CFDBFF020EB3
:10BC6000DB50100D010EF3CFDBFF010EDB50DF24A4
:10BC7000DF6E010EDB6ADF50090806E20A0EDF5CA8
:10BC8000DF6E010EDB2AF7D7010EDB50300F020109
:10BC9000186F300EDF240201196F02013A0E1A6F7D
:10BCA0007E0E01010E15E76E020EE7CFDBFF020EDE
:10BCB000DB407F0BDF6E010EDB6ADF50090806E216
:10BCC0000A0EDF5CDF6E010EDB2AF7D7010EDB50B8
:10BCD000300F02011B6F300EDF2402011C6F0201C6
:10BCE0002D0E1D6FF00E01010F15E76E020EE7CF4E
:10BCF000DBFF020EDB380F0BDF6E010E01010E15AC
:10BD0000E76E020EE7CFDBFF020EDB50100D010ED7
:10BD1000F3CFDBFF010EDB50DF24DF6E010EDB6AA9
:10BD2000DF50090806E20A0EDF5CDF6E010EDB2A37
:10BD3000F7D7010EDB50300F02011E6F300EDF24EB
:10BD400002011F6F02012F0E206F0F0E01010F1550
:10BD5000DF6E010EDB6ADF50090806E20A0EDF5CC7
:10BD6000DF6E010EDB2AF7D7010EDB50300F020128
:10BD7000216F300EDF240201226F0201140E236FA7
:10BD80000101230E736F0F013CAF05D002011A0EA3
:10BD9000246F0101732B0F013CBF16D00F0130BF80
:10BDA00003D0D7EC32F00FD042EC7AF000090BE16F
:10BDB00073C1E6FF010EE66E020EE66E4AEC7AF003
:10BDC000E552E552E55202D0A6EC3AF0090EE15CEC
:10BDD00002E2E16AE552E16EE552E7CFD9FF1200D7
:10BDE000D9CFE6FFE1CFD9FF0D0EE1260F012EA539
:10BDF00012EF65F00101CC51EA6A000FE96E050E01
:10BE0000EA22EF50230802E012EF65F0010ECCC1E8
:10BE1000DBFF020EDB6ADF6A010EDB50DF5C0DE246
:10BE2000DF50EA6A000FE96E050EEA22EF502308A0
:10BE300002E1020EDB2ADF2AEFD7020EDB5004E01C
:10BE4000020EDB50280802E212EF65F0DF6A010EF5
:10BE5000DB50DF5C10E2DF50EA6A000FE96E050E8E
:10BE6000EA22EF50230805E1DF28E76E010EE7CF55
:10BE7000DBFFDF2AECD7010EDB06010EDB5004E00E
:10BE8000010EDB50080802E212EF65F0DF6A010ED6
:10BE9000DB50DF5C46E2DF50EA6A000FE96E050E18
:10BEA000EA22EFCF00F0300E005C02E212EF65F004
:10BEB000DF50EA6A000FE96E050EEA22EF503908FA
:10BEC0000DE2DF50EA6A000FE96E050EEA22EFCFBD
:10BED00000F0410E005C02E212EF65F0DF50EA6A0A
:10BEE000000FE96E050EEA22EF5046080DE2DF5022
:10BEF000EA6A000FE96E050EEA22EFCF00F0610E4C
:10BF0000005C02E212EF65F0DF50EA6A000FE96EB2
:10BF1000050EEA22EF50660802E212EF65F0DF2A12
:10BF2000B6D7010EDB041CE10101200E006F0101F8
:10BF3000200E016F0101200E026F0101200E036F20
:10BF40000101200E066F470E0501005D03E200C5EA
:10BF500007F105D0200E0501005D0101076FC0D17A
:10BF6000010EDB50020825E10101200E006F0101E6
:10BF7000200E016F0101200E026F0101200E036FE0
:10BF8000470E0501005D03E200C506F105D0200E55
:10BF90000501005D0101066F470E0501015D03E229
:10BFA00001C507F105D0200E0501015D0101076FF4
:10BFB00097D1010EDB5003082EE10101200E006F26
:10BFC0000101200E016F0101200E026F470E0501D5
:10BFD000005D03E200C503F105D0200E0501005D00
:10BFE0000101036F470E0501015D03E201C506F182
:10BFF00005D0200E0501015D0101066F470E050108
:10C00000025D03E202C507F105D0200E0501025DC5
:10C010000101076F65D1010EDB50040837E1010112
:10C02000200E006F0101200E016F470E0501005D1B
:10C0300003E200C502F105D0200E0501005D0101FB
:10C04000026F470E0501015D03E201C503F105D052
:10C05000200E0501015D0101036F470E0501025D20
:10C0600003E202C506F105D0200E0501025D0101C3
:10C07000066F470E0501035D03E203C507F105D016
:10C08000200E0501035D0101076F2AD1010EDB506F
:10C09000050840E10101200E006F470E0501005D1B
:10C0A00003E200C501F105D0200E0501005D01018C
:10C0B000016F470E0501015D03E201C502F105D0E4
:10C0C000200E0501015D0101026F470E0501025DB1
:10C0D00003E202C503F105D0200E0501025D010156
:10C0E000036F470E0501035D03E203C506F105D0AA
:10C0F000200E0501035D0101066F470E0501045D79
:10C1000003E204C507F105D0200E0501045D01011D
:10C11000076FE6D0010EDB50060849E1470E050126
:10C12000005D03E200C500F105D0200E0501005DB1
:10C130000101006F470E0501015D03E201C501F138
:10C1400005D0200E0501015D0101016F470E0501BB
:10C15000025D03E202C502F105D0200E0501025D79
:10C160000101026F470E0501035D03E203C503F100
:10C1700005D0200E0501035D0101036F470E050187
:10C18000045D03E204C506F105D0200E0501045D3F
:10C190000101066F470E0501055D03E205C507F1C4
:10C1A00005D0200E0501055D0101076F99D0010E34
:10C1B000DB50070849E1470E0501015D03E201C5B7
:10C1C00000F105D0200E0501015D0101006F470E51
:10C1D0000501025D03E202C501F105D0200E050153
:10C1E000025D0101016F470E0501035D03E203C516
:10C1F00002F105D0200E0501035D0101026F470E1B
:10C200000501045D03E204C503F105D0200E05011C
:10C21000045D0101036F470E0501055D03E205C5DD
:10C2200006F105D0200E0501055D0101066F470EE0
:10C230000501065D03E206C507F105D0200E0501E4
:10C24000065D0101076F4CD0010EDB50080848E184
:10C25000470E0501025D03E202C500F105D0200E84
:10C260000501025D0101006F470E0501035D03E258
:10C2700003C501F105D0200E0501035D0101016F29
:10C28000470E0501045D03E204C502F105D0200E4E
:10C290000501045D0101026F470E0501055D03E222
:10C2A00005C503F105D0200E0501055D0101036FF1
:10C2B000470E0501065D03E206C506F105D0200E16
:10C2C0000501065D0101066F470E0501075D03E2EA
:10C2D00007C507F105D0200E0501075D0101076FB5
:10C2E000010EDB2A010EDB50EA6A000FE96E050E33
:10C2F000EA22EF504E0801E095D3010EDB28EA6AEE
:10C30000000FE96E050EEA22EFCF08F1010EDB50B7
:10C31000020FEA6A000FE96E050EEA22EFCF09F17B
:10C32000010EDB50030FE76E010EE7CFDBFF010EBE
:10C33000DB50EA6A000FE96E050EEA22EF5023088F
:10C340000DE10101200E0A6F0101200E0B6F0101AA
:10C35000300E0C6F0101300E0D6FA7D0010EDB2ADD
:10C36000010EDB50EA6A000FE96E050EEA22EF507B
:10C37000230813E10101200E0A6F0101200E0B6F4B
:10C380000101300E0C6F010EDB04EA6A000FE96E4A
:10C39000050EEA22EFCF0DF188D0010EDB2A010E47
:10C3A000DB50EA6A000FE96E050EEA22EF5023081F
:10C3B0001AE10101200E0A6F0101200E0B6F010E20
:10C3C000DB50FE0FEA6A000FE96E050EEA22EFCF9E
:10C3D0000CF1010EDB04EA6A000FE96E050EEA2299
:10C3E000EFCF0DF162D0010EDB2A010EDB50EA6ABD
:10C3F000000FE96E050EEA22EF50230821E101014A
:10C40000200E0A6F010EDB50FD0FEA6A000FE96E85
:10C41000050EEA22EFCF0BF1010EDB50FE0FEA6AA8
:10C42000000FE96E050EEA22EFCF0CF1010EDB04DE
:10C43000EA6A000FE96E050EEA22EFCF0DF135D062
:10C44000010EDB2A010EDB50EA6A000FE96E050ED1
:10C45000EA22EF50230828E1010EDB50FC0FEA6AC4
:10C46000000FE96E050EEA22EFCF0AF1010EDB5054
:10C47000FD0FEA6A000FE96E050EEA22EFCF0BF11D
:10C48000010EDB50FE0FEA6A000FE96E050EEA228C
:10C49000EFCF0CF1010EDB04EA6A000FE96E050E26
:10C4A000EA22EFCF0DF101D0BDD2020EDB06020E63
:10C4B000DB5001E1C0D1060EDB6A020EDB50000842
:10C4C00001E3B9D10C01F02B010EDB2A010EDB5088
:10C4D000EA6A000FE96E050EEA22EF504E0801E00D
:10C4E00088D2010EDB28EA6A000FE96E050EEA2207
:10C4F000EF50E66E060EDB50EA6A000FE96E0C0E96
:10C50000EA22E552E750EF6E010EDB50020FEA6AB5
:10C51000000FE96E050EEA22EF50E66E060EDB28EC
:10C52000EA6A000FE96E0C0EEA22E552E750EF6E60
:10C53000010EDB50030FE76E010EE7CFDBFF010EAC
:10C54000DB50EA6A000FE96E050EEA22EF5023087D
:10C5500029E1060EDB50020FEA6A000FE96E0C0EAD
:10C56000EA22200EEF6E060EDB50030FEA6A000F80
:10C57000E96E0C0EEA22200EEF6E060EDB50040F61
:10C58000EA6A000FE96E0C0EEA22300EEF6E060E1C
:10C59000DB50050FEA6A000FE96E0C0EEA22300E3E
:10C5A000EF6E3FD1010EDB2A010EDB50EA6A000F6D
:10C5B000E96E050EEA22EF50230833E1060EDB5048
:10C5C000020FEA6A000FE96E0C0EEA22200EEF6EEF
:10C5D000060EDB50030FEA6A000FE96E0C0EEA222A
:10C5E000200EEF6E060EDB50040FEA6A000FE96EB4
:10C5F0000C0EEA22300EEF6E010EDB04EA6A000F29
:10C60000E96E050EEA22EF50E66E060EDB50050FCE
:10C61000EA6A000FE96E0C0EEA22E552E750EF6E6F
:10C6200000D1010EDB2A010EDB50EA6A000FE96E31
:10C63000050EEA22EF5023083EE1060EDB50020F02
:10C64000EA6A000FE96E0C0EEA22200EEF6E060E6B
:10C65000DB50030FEA6A000FE96E0C0EEA22200E8F
:10C66000EF6E010EDB50FE0FEA6A000FE96E050E59
:10C67000EA22EF50E66E060EDB50040FEA6A000F66
:10C68000E96E0C0EEA22E552E750EF6E010EDB0474
:10C69000EA6A000FE96E050EEA22EF50E66E060E1A
:10C6A000DB50050FEA6A000FE96E0C0EEA22E55234
:10C6B000E750EF6EB6D0010EDB2A010EDB50EA6ABE
:10C6C000000FE96E050EEA22EF50230849E1060E3D
:10C6D000DB50020FEA6A000FE96E0C0EEA22200E10
:10C6E000EF6E010EDB50FD0FEA6A000FE96E050EDA
:10C6F000EA22EF50E66E060EDB50030FEA6A000FE7
:10C70000E96E0C0EEA22E552E750EF6E010EDB50A7
:10C71000FE0FEA6A000FE96E050EEA22EF50E66EA0
:10C72000060EDB50040FEA6A000FE96E0C0EEA22D7
:10C73000E552E750EF6E010EDB04EA6A000FE96E86
:10C74000050EEA22EF50E66E060EDB50050FEA6A90
:10C75000000FE96E0C0EEA22E552E750EF6E61D051
:10C76000010EDB2A010EDB50EA6A000FE96E050EAE
:10C77000EA22EF50230854E1010EDB50FC0FEA6A75
:10C78000000FE96E050EEA22EF50E66E060EDB5052
:10C79000020FEA6A000FE96E0C0EEA22E552E7503A
:10C7A000EF6E010EDB50FD0FEA6A000FE96E050E19
:10C7B000EA22EF50E66E060EDB50030FEA6A000F26
:10C7C000E96E0C0EEA22E552E750EF6E010EDB50E7
:10C7D000FE0FEA6A000FE96E050EEA22EF50E66EE0
:10C7E000060EDB50040FEA6A000FE96E0C0EEA2217
:10C7F000E552E750EF6E010EDB04EA6A000FE96EC6
:10C80000050EEA22EF50E66E060EDB50050FEA6ACF
:10C81000000FE96E0C0EEA22E552E750EF6E01D0F0
:10C82000E8D0060EDB50060FE76E060EE7CFDBFF03
:10C83000020EDB0642D601010A0E056F0F012B899D
:10C8400000C110F101C111F102C112F103C113F1D4
:10C85000DEC114F10101BB0E156F0101145101E19C
:10C86000AFD00101140501E1ABD0060EF36E0C0E42
:10C87000F3CFDBFF2B0E0101CE5D52E1010EF36E13
:10C88000080EF3CFDBFF0101DE51F36E080EDBCFA4
:10C89000F4FFF350F45C43E2080EDB50010BE76E4B
:10C8A000090EE7CFDBFF080EDB50EA6ACE0FE96E18
:10C8B000010EEA22EF50D00FE76E0A0EE7CFDBFF42
:10C8C000090EDB500FE00A0EDB38F00BE66E0C0EA3
:10C8D000DB50EA6A100FE96E010EEA22E552E750DA
:10C8E000EF6E1AD00A0EDBCFE6FF0C0EDB50EA6AC1
:10C8F000100FE96E010EEA22EF50E552E724E66ED2
:10C900000C0EDB50EA6A100FE96E010EEA22E552C6
:10C91000E750EF6E0C0EDB2A080EDB2AB4D750D09E
:10C920000101142B080EDB6A0101DE51F36E080EC3
:10C93000DBCFF4FFF350F45C43E2080EDB50010B55
:10C94000E76E090EE7CFDBFF080EDB50EA6ACE0F79
:10C95000E96E010EEA22EF50D00FE76E0A0EE7CF24
:10C96000DBFF090EDB500FE10A0EDB38F00BE66E41
:10C970000C0EDB50EA6A100FE96E010EEA22E55256
:10C98000E750EF6E1AD00A0EDBCFE6FF0C0EDB503D
:10C99000EA6A100FE96E010EEA22EF50E552E72431
:10C9A000E66E0C0EDB50EA6A100FE96E010EEA2209
:10C9B000E552E750EF6E0C0EDB2A080EDB2AB4D7E7
:10C9C00006C11EF107C11FF10101DE6B0101F86B09
:10C9D000100E0101F85D0BE20101F851EA6ACE0F79
:10C9E000E96E010EEA22EF6A0101F82BF1D75FEF41
:10C9F0006DF00C01F06B060EDB6AF00EF36E060EA6
:10CA0000DBCFF4FFF350F45C0BE2060EDB50EA6A76
:10CA1000000FE96E0C0EEA22EF6A060EDB2AEDD754
:10CA200018EF6EF02C0E0501025D02E018EF6EF0BB
:10CA30002C0E0501075D02E018EF6EF0020E0101F9
:10CA4000CC5DE76E010EE7CFDBFF010EDB50EA6A3B
:10CA5000000FE96E050EEA22EF502A0802E018EFF7
:10CA60006EF0020EDB6ADF6A010EDB50DF5C12E261
:10CA7000020EDBCFE6FFDF50EA6A000FE96E050E1B
:10CA8000EA22EF50E552E718E76E020EE7CFDBFF30
:10CA9000DF2AEAD70101CC05E76E010EE7CFDBFF05
:10CAA000020EDB50F00BE76E030EE7CFDBFF030E49
:10CAB000DB380F0BE76E030EE7CFDBFF0A0EF36EDA
:10CAC000030EDBCFF4FFF350F45C08E2030EDB50FF
:10CAD000300FE76E040EE7CFDBFF07D0030EDB500D
:10CAE000370FE76E040EE7CFDBFF010EDB50EA6A7B
:10CAF000000FE96E050EEA22EF50500814E2010E15
:10CB0000DB50EA6A000FE96E050EEA22EF50E00FF3
:10CB1000E66E010EDB50EA6A000FE96E050EEA22AE
:10CB2000E552E750EF6E010EDB50EA6A000FE96E46
:10CB3000050EEA22EF50F36E040EDB50F35C02E0C8
:10CB400018EF6EF0020EDB500F0BE76E030EE7CF0F
:10CB5000DBFF0A0EF36E030EDBCFF4FFF350F45C41
:10CB600008E2030EDB50300FE76E040EE7CFDBFF69
:10CB700007D0030EDB50370FE76E040EE7CFDBFF65
:10CB80000101CC51EA6A000FE96E050EEA22EF506E
:10CB9000500814E20101CC51EA6A000FE96E050E5B
:10CBA000EA22EF50E00FE66E0101CC51EA6A000F75
:10CBB000E96E050EEA22E552E750EF6E0101CC5115
:10CBC000EA6A000FE96E050EEA22EF50F36E040EDA
:10CBD000DB50F35C02E018EF6EF0460E0501005DDD
:10CBE00005E0660E0501005D01E0D7D1460E0501A6
:10CBF000015D05E0660E0501015D01E0CED1470E45
:10CC00000501035D03E203C500F105D0200E050117
:10CC1000035D0101006F470E0501045D03E204C5D9
:10CC200001F105D0200E0501045D0101016F470EE1
:10CC30000501055D03E205C502F105D0200E0501E1
:10CC4000055D0101026F470E0501065D03E206C5A1
:10CC500003F105D0200E0501065D0101036F0101FE
:10CC60000F0E056F470E0501085D03E208C506F1CA
:10CC700005D0200E0501085D0101066F0101200E9F
:10CC8000076F0101300E086F0101300E096F470E6A
:10CC90000501095D03E209C50AF105D0200E050171
:10CCA000095D01010A6F0F012EA305D006C109F12C
:10CCB0000101410E066F0F012B890A0EF36E070E5C
:10CCC000F3CFDBFF01016E6B060EDB6A280EF36EFD
:10CCD000060EDBCFF4FFF350F45C01E38BD0070EBC
:10CCE000DB50EA6A000FE96E050EEA22EF502A08CF
:10CCF00001E180D0070EDB50EA6A000FE96E050EF5
:10CD0000EA22EF502C0801E075D001016E2B070ECE
:10CD1000DB2A070EDB50EA6A000FE96E050EEA22F5
:10CD2000EFCF00F0470E005C14E2070EDB50EA6A1A
:10CD3000000FE96E050EEA22EF50E66E060EDB509C
:10CD4000EA6A460FE96E010EEA22E552E750EF6EFD
:10CD500014D0070EDB50EA6A000FE96E050EEA22D6
:10CD6000EF50E00FE66E060EDB50EA6A460FE96E02
:10CD7000010EEA22E552E750EF6E060EDB2A070E9F
:10CD8000DB2A070EDB50EA6A000FE96E050EEA2285
:10CD9000EFCF00F0470E005C14E2070EDB50EA6AAA
:10CDA000000FE96E050EEA22EF50E66E060EDB502C
:10CDB000EA6A460FE96E010EEA22E552E750EF6E8D
:10CDC00014D0070EDB50EA6A000FE96E050EEA2266
:10CDD000EF50E00FE66E060EDB50EA6A460FE96E92
:10CDE000010EEA22E552E750EF6E070EDB2A060E2F
:10CDF000DB2A6CD700C110F101C111F102C112F19F
:10CE000003C113F1DEC114F10101550E156F0101CB
:10CE1000145101E1AFD00101140501E1ABD0060EC0
:10CE2000F36E0C0EF3CFDBFF2B0E0101CE5D52E152
:10CE3000010EF36E080EF3CFDBFF0101DE51F36E3E
:10CE4000080EDBCFF4FFF350F45C43E2080EDB5036
:10CE5000010BE76E090EE7CFDBFF080EDB50EA6A35
:10CE6000CE0FE96E010EEA22EF50D00FE76E0A0EE8
:10CE7000E7CFDBFF090EDB500FE00A0EDB38F00BCB
:10CE8000E66E0C0EDB50EA6A100FE96E010EEA2224
:10CE9000E552E750EF6E1AD00A0EDBCFE6FF0C0E1C
:10CEA000DB50EA6A100FE96E010EEA22EF50E552FC
:10CEB000E724E66E0C0EDB50EA6A100FE96E010EF5
:10CEC000EA22E552E750EF6E0C0EDB2A080EDB2A51
:10CED000B4D750D00101142B080EDB6A0101DE51DA
:10CEE000F36E080EDBCFF4FFF350F45C43E2080E60
:10CEF000DB50010BE76E090EE7CFDBFF080EDB50BE
:10CF0000EA6ACE0FE96E010EEA22EF50D00FE76E0B
:10CF10000A0EE7CFDBFF090EDB500FE10A0EDB380C
:10CF2000F00BE66E0C0EDB50EA6A100FE96E010E94
:10CF3000EA22E552E750EF6E1AD00A0EDBCFE6FF89
:10CF40000C0EDB50EA6A100FE96E010EEA22EF5078
:10CF5000E552E724E66E0C0EDB50EA6A100FE96E2C
:10CF6000010EEA22E552E750EF6E0C0EDB2A080EA6
:10CF7000DB2AB4D70101DE6B0101F86B100E010151
:10CF8000F85D0BE20101F851EA6ACE0FE96E010E7D
:10CF9000EA22EF6A0101F82BF1D7300E0501005D9E
:10CFA00002E05FEF6DF0360E0501015D05E0370E22
:10CFB0000501015D01E091D1470E0501035D03E22A
:10CFC00003C500F105D0200E0501035D0101006FCE
:10CFD000470E0501045D03E204C501F105D0200EF2
:10CFE0000501045D0101016F470E0501055D03E2C6
:10CFF00005C502F105D0200E0501055D0101026F96
:10D00000470E0501065D03E206C503F105D0200EBB
:10D010000501065D0101036F0101090E056F360E62
:10D020000501015D04E10101310E066F03D001012C
:10D03000330E066F470E0501085D03E208C507F1D0
:10D0400005D0200E0501085D0101076F470E05019F
:10D05000095D03E209C508F105D0200E0501095D4F
:10D060000101086F470E05010A5D03E20AC509F1D7
:10D0700005D0200E05010A5D0101096F470E05016B
:10D080000B5D03E20BC50AF105D0200E05010B5D17
:10D0900001010A6F470E05010C5D03E20CC50BF19F
:10D0A00005D0200E05010C5D01010B6F470E050137
:10D0B0000D5D03E20DC50CF105D0200E05010D5DDF
:10D0C00001010C6F3A0E05010E5D05E2300E0501FF
:10D0D0000E5DDF6E0DD0470E05010E5D05E2370EC9
:10D0E00005010E5DDF6E04D0570E05010E5DDF6E8B
:10D0F000DF50100D030EF3CFDBFF3A0E05010F5D7D
:10D1000005E2300E05010F5DDF6E0DD0470E050103
:10D110000F5D05E2370E05010F5DDF6E04D0570E7F
:10D1200005010F5DDF6E030EDB50DF2401010D6F83
:10D130000F012B8900C110F101C111F102C112F1DF
:10D1400003C113F1DEC114F10101550E156F010188
:10D15000145101E1AFD00101140501E1ABD0060E7D
:10D16000F36E0C0EF3CFDBFF2B0E0101CE5D52E10F
:10D17000010EF36E080EF3CFDBFF0101DE51F36EFB
:10D18000080EDBCFF4FFF350F45C43E2080EDB50F3
:10D19000010BE76E090EE7CFDBFF080EDB50EA6AF2
:10D1A000CE0FE96E010EEA22EF50D00FE76E0A0EA5
:10D1B000E7CFDBFF090EDB500FE00A0EDB38F00B88
:10D1C000E66E0C0EDB50EA6A100FE96E010EEA22E1
:10D1D000E552E750EF6E1AD00A0EDBCFE6FF0C0ED9
:10D1E000DB50EA6A100FE96E010EEA22EF50E552B9
:10D1F000E724E66E0C0EDB50EA6A100FE96E010EB2
:10D20000EA22E552E750EF6E0C0EDB2A080EDB2A0D
:10D21000B4D750D00101142B080EDB6A0101DE5196
:10D22000F36E080EDBCFF4FFF350F45C43E2080E1C
:10D23000DB50010BE76E090EE7CFDBFF080EDB507A
:10D24000EA6ACE0FE96E010EEA22EF50D00FE76EC8
:10D250000A0EE7CFDBFF090EDB500FE10A0EDB38C9
:10D26000F00BE66E0C0EDB50EA6A100FE96E010E51
:10D27000EA22E552E750EF6E1AD00A0EDBCFE6FF46
:10D280000C0EDB50EA6A100FE96E010EEA22EF5035
:10D29000E552E724E66E0C0EDB50EA6A100FE96EE9
:10D2A000010EEA22E552E750EF6E0C0EDB2A080E63
:10D2B000DB2AB4D70101DE6B0101F86B100E01010E
:10D2C000F85D0BE20101F851EA6ACE0FE96E010E3A
:10D2D000EA22EF6A0101F82BF1D7310E0501015D59
:10D2E00001E031D1470E0501035D03E203C500F102
:10D2F00005D0200E0501035D0101006F470E0501F9
:10D30000045D03E204C501F105D0200E0501045DB2
:10D310000101016F470E0501055D03E205C502F13C
:10D3200005D0200E0501055D0101026F470E0501C4
:10D33000065D03E206C503F105D0200E0501065D7A
:10D340000101036F0101010E056F470E0501085D24
:10D3500003E208C506F105D0200E0501085D0101B4
:10D36000066F0101200E076F0101300E086F0101E9
:10D37000300E096F470E0501095D03E209C50AF188
:10D3800005D0200E0501095D01010A6F0F012EA3D2
:10D3900005D006C109F10101410E066F0F012B896D
:10D3A00000C110F101C111F102C112F103C113F169
:10D3B000DEC114F10101550E156F0101145101E197
:10D3C000AFD00101140501E1ABD0060EF36E0C0ED7
:10D3D000F3CFDBFF2B0E0101CE5D52E1010EF36EA8
:10D3E000080EF3CFDBFF0101DE51F36E080EDBCF39
:10D3F000F4FFF350F45C43E2080EDB50010BE76EE0
:10D40000090EE7CFDBFF080EDB50EA6ACE0FE96EAC
:10D41000010EEA22EF50D00FE76E0A0EE7CFDBFFD6
:10D42000090EDB500FE00A0EDB38F00BE66E0C0E37
:10D43000DB50EA6A100FE96E010EEA22E552E7506E
:10D44000EF6E1AD00A0EDBCFE6FF0C0EDB50EA6A55
:10D45000100FE96E010EEA22EF50E552E724E66E66
:10D460000C0EDB50EA6A100FE96E010EEA22E5525B
:10D47000E750EF6E0C0EDB2A080EDB2AB4D750D033
:10D480000101142B080EDB6A0101DE51F36E080E58
:10D49000DBCFF4FFF350F45C43E2080EDB50010BEA
:10D4A000E76E090EE7CFDBFF080EDB50EA6ACE0F0E
:10D4B000E96E010EEA22EF50D00FE76E0A0EE7CFB9
:10D4C000DBFF090EDB500FE10A0EDB38F00BE66ED6
:10D4D0000C0EDB50EA6A100FE96E010EEA22E552EB
:10D4E000E750EF6E1AD00A0EDBCFE6FF0C0EDB50D2
:10D4F000EA6A100FE96E010EEA22EF50E552E724C6
:10D50000E66E0C0EDB50EA6A100FE96E010EEA229D
:10D51000E552E750EF6E0C0EDB2A080EDB2AB4D77B
:10D520000101DE6B0101F86B100E0101F85D0BE2E9
:10D530000101F851EA6ACE0FE96E010EEA22EF6AA4
:10D540000101F82BF1D7320E0501015D01E03BD15D
:10D550000F012B89470E0501035D03E203C500F1AE
:10D5600005D0200E0501035D0101006F470E050186
:10D57000045D03E204C501F105D0200E0501045D40
:10D580000101016F470E0501055D03E205C502F1CA
:10D5900005D0200E0501055D0101026F470E050152
:10D5A000065D03E206C503F105D0200E0501065D08
:10D5B0000101036F0101020E056F470E0501085DB1
:10D5C00003E208C506F105D0200E0501085D010142
:10D5D000066F0101200E076F470E0501095D03E28A
:10D5E00009C508F105D0200E0501095D0101086F8C
:10D5F000470E05010A5D03E20AC509F105D0200EB8
:10D6000005010A5D0101096F470E05010B5D03E28B
:10D610000BC50AF105D0200E05010B5D01010A6F53
:10D6200000C110F101C111F102C112F103C113F1E6
:10D63000DEC114F10101550E156F0101145101E114
:10D64000AFD00101140501E1ABD0060EF36E0C0E54
:10D65000F3CFDBFF2B0E0101CE5D52E1010EF36E25
:10D66000080EF3CFDBFF0101DE51F36E080EDBCFB6
:10D67000F4FFF350F45C43E2080EDB50010BE76E5D
:10D68000090EE7CFDBFF080EDB50EA6ACE0FE96E2A
:10D69000010EEA22EF50D00FE76E0A0EE7CFDBFF54
:10D6A000090EDB500FE00A0EDB38F00BE66E0C0EB5
:10D6B000DB50EA6A100FE96E010EEA22E552E750EC
:10D6C000EF6E1AD00A0EDBCFE6FF0C0EDB50EA6AD3
:10D6D000100FE96E010EEA22EF50E552E724E66EE4
:10D6E0000C0EDB50EA6A100FE96E010EEA22E552D9
:10D6F000E750EF6E0C0EDB2A080EDB2AB4D750D0B1
:10D700000101142B080EDB6A0101DE51F36E080ED5
:10D71000DBCFF4FFF350F45C43E2080EDB50010B67
:10D72000E76E090EE7CFDBFF080EDB50EA6ACE0F8B
:10D73000E96E010EEA22EF50D00FE76E0A0EE7CF36
:10D74000DBFF090EDB500FE10A0EDB38F00BE66E53
:10D750000C0EDB50EA6A100FE96E010EEA22E55268
:10D76000E750EF6E1AD00A0EDBCFE6FF0C0EDB504F
:10D77000EA6A100FE96E010EEA22EF50E552E72443
:10D78000E66E0C0EDB50EA6A100FE96E010EEA221B
:10D79000E552E750EF6E0C0EDB2A080EDB2AB4D7F9
:10D7A0000101DE6B0101F86B100E0101F85D0BE267
:10D7B0000101F851EA6ACE0FE96E010EEA22EF6A22
:10D7C0000101F82BF1D7330E0501015D01E077D19E
:10D7D000470E0501035D03E203C500F105D0200EED
:10D7E0000501035D0101006F470E0501045D03E2C1
:10D7F00004C501F105D0200E0501045D0101016F92
:10D80000470E0501055D03E205C502F105D0200EB6
:10D810000501055D0101026F470E0501065D03E28A
:10D8200006C503F105D0200E0501065D0101036F59
:10D830000101090E056F0101310E066F0101300E65
:10D84000076F470E0501085D03E208C508F105D022
:10D85000200E0501085D0101086F470E0501095DF5
:10D8600003E209C509F105D0200E0501095D01019A
:10D87000096F470E05010C5D03E20CC50AF105D0E6
:10D88000200E05010C5D01010A6F470E05010D5DBB
:10D8900003E20DC50BF105D0200E05010D5D010160
:10D8A0000B6F0101300E0C6F3A0E05010A5D05E2A7
:10D8B000300E05010A5DDF6E0DD0470E05010A5DD1
:10D8C00005E2370E05010A5DDF6E04D0570E050133
:10D8D0000A5DDF6EDF50100D030EF3CFDBFF3A0E53
:10D8E00005010B5D05E2300E05010B5DDF6E0DD00D
:10D8F000470E05010B5D05E2370E05010B5DDF6E7E
:10D9000004D0570E05010B5DDF6E030EDB50DF24E4
:10D9100001010D6F0F012B8900C110F101C111F13F
:10D9200002C112F103C113F1DEC114F10101550E60
:10D93000156F0101145101E1AFD00101140501E19E
:10D94000ABD0060EF36E0C0EF3CFDBFF2B0E0101F6
:10D95000CE5D52E1010EF36E080EF3CFDBFF010145
:10D96000DE51F36E080EDBCFF4FFF350F45C43E2BC
:10D97000080EDB50010BE76E090EE7CFDBFF080E48
:10D98000DB50EA6ACE0FE96E010EEA22EF50D00FAB
:10D99000E76E0A0EE7CFDBFF090EDB500FE00A0E41
:10D9A000DB38F00BE66E0C0EDB50EA6A100FE96E06
:10D9B000010EEA22E552E750EF6E1AD00A0EDBCFD5
:10D9C000E6FF0C0EDB50EA6A100FE96E010EEA2248
:10D9D000EF50E552E724E66E0C0EDB50EA6A100FBA
:10D9E000E96E010EEA22E552E750EF6E0C0EDB2ADB
:10D9F000080EDB2AB4D750D00101142B080EDB6AC5
:10DA00000101DE51F36E080EDBCFF4FFF350F45C3E
:10DA100043E2080EDB50010BE76E090EE7CFDBFF98
:10DA2000080EDB50EA6ACE0FE96E010EEA22EF50D3
:10DA3000D00FE76E0A0EE7CFDBFF090EDB500FE1D8
:10DA40000A0EDB38F00BE66E0C0EDB50EA6A100FA4
:10DA5000E96E010EEA22E552E750EF6E1AD00A0E87
:10DA6000DBCFE6FF0C0EDB50EA6A100FE96E010E09
:10DA7000EA22EF50E552E724E66E0C0EDB50EA6A2C
:10DA8000100FE96E010EEA22E552E750EF6E0C0E20
:10DA9000DB2A080EDB2AB4D70101DE6B0101F86B2B
:10DAA000100E0101F85D0BE20101F851EA6ACE0F98
:10DAB000E96E010EEA22EF6A0101F82BF1D7300E70
:10DAC00001013C5DDF6E300E01013D5DE76E030E2E
:10DAD000E7CFDBFFDF5009E0030EDB500A0FE76EF4
:10DAE000030EE7CFDBFFDF06F5D7030EDB50040D97
:10DAF000F3CF04F1300E01013E5DDF6E300E010107
:10DB00003F5DE76E030EE7CFDBFFDF5009E0030E5A
:10DB1000DB500A0FE76E030EE7CFDBFFDF06F5D71A
:10DB2000030EDB50300BDF6EDF380F0BE76E050E98
:10DB3000E7CFDBFF050EDB50010104250101046F77
:10DB4000030EDB500F0BDF6EDF50100D050EF3CF11
:10DB5000DBFF050EDB50010105250101056F300ECD
:10DB60000101405DDF6E300E0101415DE76E030E85
:10DB7000E7CFDBFFDF5009E0030EDB500A0FE76E53
:10DB8000030EE7CFDBFFDF06F5D7030EDB50E824FB
:10DB900001010E6F300E0101425DDF6E300E01019A
:10DBA000435DE76E030EE7CFDBFFDF5009E0030EB6
:10DBB000DB500A0FE76E030EE7CFDBFFDF06F5D77A
:10DBC000030EDB50100BDF6EDF380F0BE76E050E18
:10DBD000E7CFDBFF050EDB5001010E2501010E6FC3
:10DBE000030EDB500F0BDF6EDF50100D050EF3CF71
:10DBF000DBFF300E0101445DDF6E300E0101455D3B
:10DC0000E76E030EE7CFDBFFDF5009E0030EDB50CA
:10DC10000A0FE76E030EE7CFDBFFDF06F5D7050E31
:10DC2000DBCFE6FF030EDB50E552E72401010F6F67
:10DC30000D0EE15C02E2E16AE552E16EE552E7CFEA
:10DC4000D9FF1200D9CFE6FFE1CFD9FF060EE126BA
:10DC50000F012BB549EF74F00F012BAD06D00F016A
:10DC60002B9D6EEC75F064EF75F00D0E0501005DF7
:10DC700007E10101020EED6F92EC75F064EF75F0B3
:10DC80004F0E0501005D11E14B0E0501015D0DE137
:10DC90000D0E0501025D09E10101040EED6F92EC2C
:10DCA00075F00F01288364EF75F02B0E0501005D00
:10DCB00002E08AEF73F0510E0501015D16E1490E95
:10DCC0000501025D12E14E0E0501035D0EE1490EF4
:10DCD0000501045D0AE1330E05010B5D02E10F0150
:10DCE00029836EEC75F064EF75F0430E0501015D5C
:10DCF0002CE1500E0501025D28E1490E0501035D8E
:10DD000024E14E0E0501045D20E1520E0501075D80
:10DD100006E1450E0501085D02E10F012885500E60
:10DD200005010B5D0EE1490E05010C5D0AE14E0E89
:10DD300005010D5D06E10D0E05010E5D02E10F010D
:10DD400028876EEC75F064EF75F0430E0501015DF8
:10DD50000DE14D0E0501025D09E1450E0501035D72
:10DD600005E1DF6A6EEC75F064EF75F0430E0501B6
:10DD7000015D0EE14D0E0501025D0AE1530E050144
:10DD8000035D06E10F01308B6EEC75F064EF75F00A
:10DD9000430E0501015D25E1520E0501025D21E101
:10DDA000450E0501035D1DE1470E0501045D19E106
:10DDB0003A0E0501055D15E1200E0501065D11E134
:10DDC000310E0501095D04E0350E0501095D03E131
:10DDD0000F012A8302D00F012A816EEC75F064EFE7
:10DDE00075F0430E0501015D01E087D1530E050179
:10DDF000025D01E082D1510E0501035D01E07DD19C
:10DE00000101FE0EED6F0101EC6B0101ED5101010D
:10DE1000EC5D11E20101EC51EA6A000FE96E050EBA
:10DE2000EA22EF50200804E10101EC290101ED6F25
:10DE30000101EC2BEAD70101ED290101EC6F010191
:10DE4000EC51EA6A000FE96E050EEA22EF502C0849
:10DE50006BE10101ED51EA6A000FE96E050EEA225D
:10DE6000EF502F0860E20101ED51EA6A000FE96E00
:10DE7000050EEA22EFCF00F03A0E005C54E20F01EB
:10DE800031910F0131830F0131950F01319701015C
:10DE9000ED51EA6A000FE96E050EEA22EFCFB1FB01
:10DEA0000B012C0EB26F0101EC2B0101EC51EA6A5F
:10DEB000000FE96E050EEA22EFCFB3FB0101EC2B58
:10DEC0000101EC51EA6A000FE96E050EEA22EF50FB
:10DED0000A0804E10B010A0EB46F0BD10101EC51E9
:10DEE000EA6A000FE96E050EEA22EFCFB4FB0101EA
:10DEF000EC2B0101EC51EA6A000FE96E050EEA22F3
:10DF0000EF500A0804E10B010A0EB56FF2D00B01C5
:10DF1000300EB16F0B012C0EB26F0B01300EB36FD0
:10DF20000B010A0EB46FE5D00101EC2B0101EC519D
:10DF3000EA6A000FE96E050EEA22EF502C0801E0B4
:10DF4000D8D00101ED51EA6A000FE96E050EEA2210
:10DF5000EF502F0801E3CDD00101ED51EA6A000F27
:10DF6000E96E050EEA22EFCF00F03A0E005C01E305
:10DF7000C0D00101ED51EA6A000FE96E050EEA22F8
:10DF8000EF50D00F0101E96F0A0E0101E903F3CF51
:10DF9000EAF10101ED2B0101ED51EA6A000FE96E92
:10DFA000050EEA22EF502F0801E3A3D00101ED5145
:10DFB000EA6A000FE96E050EEA22EFCF00F03A0E92
:10DFC000005C01E396D00101ED51EA6A000FE96EB1
:10DFD000050EEA22EF50D00F0101E96F0101EA516D
:10DFE0000101E9250101EA6F0101ED05EA6A000F6F
:10DFF000E96E050EEA22EFCFB1FB0101ED51EA6AAD
:10E00000000FE96E050EEA22EFCFB2FB0B012C0EDA
:10E01000B36F630E0101EA5D09E10F0131810F0168
:10E0200031930F0131950F01319722D00B0E010171
:10E03000EA5D09E20F0131910F0131830F01319542
:10E040000F01319715D0100E0101EA5D09E20F01B1
:10E0500031910F0131930F0131850F01319708D0B4
:10E060000F0131910F0131930F0131950F0131876C
:10E070000101EC2B0101EC51EA6A000FE96E050E7B
:10E08000EA22EFCFB4FB0101EC2B0101EC51EA6A6B
:10E09000000FE96E050EEA22EF500A0804E10B01B9
:10E0A0000A0EB56F26D00101EC51EA6A000FE96E45
:10E0B000050EEA22EFCFB5FB0101EC2B0101EC517B
:10E0C000EA6A000FE96E050EEA22EF500A0804E141
:10E0D0000B010A0EB66F0DD00B01300EB16F0B01A4
:10E0E0002C0EB26F0B01300EB36F0B010A0EB46F22
:10E0F00000D06EEC75F064EF75F0430E0501015D24
:10E100001DE1470E0501025D19E1410E0501035DA8
:10E1100015E1540E0501045D11E1540E0501055D84
:10E120000DE1310E0501085D03E10F013C8502D0D0
:10E130000F013C956EEC75F064EF75F0430E050130
:10E14000015D74E14C0E0501025D70E1490E0501AF
:10E15000035D6CE1500E0501045D68E10F01399F1C
:10E160000F01399D220E0501075D53E10F01398F23
:10E17000040EDB6A110EF36E040EDBCFF4FFF350D6
:10E18000F45C47E2040EDB50080FE76E050EE7CFA4
:10E19000DBFF050EDB50EA6A000FE96E050EEA228E
:10E1A000EF50220804E1040EDBCFDFF134D0050E7E
:10E1B000DB50EA6A000FE96E050EEA22EF50E66EC8
:10E1C000040EDB50EA6A020FE96E0F0EEA22E552F6
:10E1D000E750EF6E040EDB50000818E2040EDB502F
:10E1E000EA6A020FE96E0F0EEA22EFCF00F0300E5E
:10E1F000005C0AE3040EDB50EA6A020FE96E0F0EC0
:10E20000EA22EF50390802E20F01399F040EDB2A9F
:10E21000B1D70F01399F0101DF5102E10F01398DA3
:10E220006EEC75F0040EDB6A64EF75F0430E0501C9
:10E23000015D12E14D0E0501025D0EE1470E050183
:10E24000035D0AE1530E0501045D06E10F012C8711
:10E250006EEC75F064EF75F0430E0501015D72E13F
:10E260004D0E0501025D6EE1470E0501035D6AE199
:10E270004C0E0501045D66E10501FF6B0101FE0E18
:10E28000ED6F0101EC6B0101ED510101EC5D11E25B
:10E290000101EC51EA6A000FE96E050EEA22EF5027
:10E2A0002C0804E10101EC290101ED6F0101EC2BC7
:10E2B000EAD7020E0101ED5D0101EC6F0101EC51A5
:10E2C000EA6A000FE96E050EEA22EF502F0838E2E5
:10E2D0000101EC51EA6A000FE96E050EEA22EFCF68
:10E2E00000F03A0E005C2CE20101EC51EA6A000FEA
:10E2F000E96E050EEA22EFCF7AF10F012B810101C1
:10E30000EC070101EC51EA6A000FE96E050EEA2202
:10E31000EF502F0815E20101EC51EA6A000FE96E97
:10E32000050EEA22EFCF00F03A0E005C09E201018F
:10E33000EC51EA6A000FE96E050EEA22EFCF7BF19D
:10E34000CDDBC2D3430E0501015D01E0E3D14D0EEB
:10E350000501025D01E0DED1470E0501035D01E02C
:10E36000D9D1520E0501045D01E0D4D10101FE0EA8
:10E37000ED6F0F012B870201FF6B0101EC6B0101B7
:10E38000ED510101EC5D2CE20101EC51EA6A000F54
:10E39000E96E050EEA22EF500A0804E10101EC29BA
:10E3A0000101ED6F0101EC51EA6A000FE96E050E03
:10E3B000EA22EF502C0811E10201FF2B0F012CB1D2
:10E3C00006D0020EECC1DBFF0F012C8106D0030E3C
:10E3D0000201FF5D02E1ECC1DFFF0101EC2BCFD7B1
:10E3E0000F012C910101DE6B020EDB28E76E030E9C
:10E3F000E7CFDBFF030EDB28E76E020EE7CFDBFF84
:10E40000030EDB50EA6A000FE96E050EEA22EF50B8
:10E41000220855E1040EDB6A110EF36E040EDBCF09
:10E42000F4FFF350F45C4BE2040EDBCFE6FF020E88
:10E43000DB50E552E724E76E050EE7CFDBFF050E64
:10E44000DB50EA6A000FE96E050EEA22EF5022085F
:10E4500004E1040EDBCFDEF134D0050EDB50EA6AB6
:10E46000000FE96E050EEA22EF50E66E040EDB5057
:10E47000EA6ACE0FE96E010EEA22E552E750EF6E2E
:10E48000040EDB50000818E2040EDB50EA6ACE0FDF
:10E49000E96E010EEA22EFCF00F0300E005C0AE3D5
:10E4A000040EDB50EA6ACE0FE96E010EEA22EF504D
:10E4B000390802E20F012B97040EDB2AADD70F01BA
:10E4C0002B970101DE5102E10F012B97DF28E76E48
:10E4D000010EE7CFDBFF010EDB50EA6A000FE96EA9
:10E4E000050EEA22EF50220802E00F012B97060EDC
:10E4F000DF24E76E010EE7CFDBFF010EDB50EA6A97
:10E50000000FE96E050EEA22EF502F0802E00F011E
:10E510002B97090EDF24E76E010EE7CFDBFF010E1C
:10E52000DB50EA6A000FE96E050EEA22EF502F0871
:10E5300002E00F012B970F0EDF24E76E010EE7CFED
:10E54000DBFF010EDB50EA6A000FE96E050EEA22DE
:10E55000EF503A0802E00F012B97120EDF24E76E0E
:10E56000010EE7CFDBFF010EDB50EA6A000FE96E18
:10E57000050EEA22EF503A0802E00F012B970F0137
:10E580002BA7B7D0070EDF24E76E010EE7CFDBFF26
:10E59000010EDB50EA6A000FE96E050EEA22EFCFAA
:10E5A00044F1080EDF24E76E010EE7CFDBFF010E1A
:10E5B000DB50EA6A000FE96E050EEA22EFCF45F163
:10E5C0000A0EDF24E76E010EE7CFDBFF010EDB5002
:10E5D000EA6A000FE96E050EEA22EFCF42F10B0E58
:10E5E000DF24E76E010EE7CFDBFF010EDB50EA6AA6
:10E5F000000FE96E050EEA22EFCF43F10D0EDF2486
:10E60000E76E010EE7CFDBFF010EDB50EA6A000F79
:10E61000E96E050EEA22EFCF3CF10E0EDF24E76E25
:10E62000010EE7CFDBFF010EDB50EA6A000FE96E57
:10E63000050EEA22EFCF3DF1100EDF24E76E010E4A
:10E64000E7CFDBFF010EDB50EA6A000FE96E050E33
:10E65000EA22EFCF3EF1110EDF24E76E010EE7CF85
:10E66000DBFF010EDB50EA6A000FE96E050EEA22BD
:10E67000EFCF3FF1130EDF24E76E010EE7CFDBFF94
:10E68000010EDB50EA6A000FE96E050EEA22EFCFB9
:10E6900040F1140EDF24E76E010EE7CFDBFF010E21
:10E6A000DB50EA6A000FE96E050EEA22EFCF41F176
:10E6B0000101EC6B0A0E0101EC5D1BE20101EC5162
:10E6C000EA6A3C0FE96E010EEA22EFCF00F0300E4D
:10E6D000005C0AE30101EC51EA6A3C0FE96E010EAD
:10E6E000EA22EF50390802E20F012B970101EC2BCF
:10E6F000E1D70F012BA703D00F012B8502D00F010B
:10E700002B8D9EAA05D0AFCFFEF59E9AB9EC2DF0C9
:10E7100009DADAD1430E0501005D12E14F0E050161
:10E72000015D0EE14E0E0501025D0AE1460E050196
:10E73000085D06E10F013D830F013C97CFD9C4D19D
:10E74000430E0501005D10E14F0E0501015D0CE176
:10E750004E0E0501025D08E14F0E0501085D04E162
:10E760000F013C87BBD9B0D1530E0501005D14E108
:10E77000450E0501015D10E14E0E0501025D0CE143
:10E78000440E0501035D08E14F0E0501055D02E140
:10E790000F013C89A3D998D1440E0501005D14E115
:10E7A000450E0501015D10E1410E0501025D0CE120
:10E7B0004F0E0501065D08E10F013C9B0B01776BD5
:10E7C0000F013C978BD980D10F013CA112D0450E8F
:10E7D0000501005D0EE1520E0501015D0AE1520ED8
:10E7E0000501025D06E10F013D830F013C9776D9DB
:10E7F0006BD10F013CA74BD0430E0501005D0CE12E
:10E800004C0E0501015D08E14F0E0501025D04E1BA
:10E810000F013D8363D958D1470E0501005D18E112
:10E82000730E0501015D14E16D0E0501025D10E13D
:10E83000540E0501035D0CE1730E0501045D08E152
:10E84000630E0501055D04E10F01398747D93CD10D
:10E850000F013CBF1CD0520E0501005D18E1500EA7
:10E860000501015D14E1340E0501025D10E1300E79
:10E870000501035D0CE1300E0501045D08E1300E79
:10E880000501055D04E10F013A8728D91DD126D97C
:10E890001BD10F012B950101FE0EED6F0101EC6BF9
:10E8A0000101ED510101EC5D11E20101EC51EA6A57
:10E8B000000FE96E050EEA22EF500A0804E101019B
:10E8C000EC290101ED6F0101EC2BEAD70101ED51BB
:10E8D00002080BE2030E0101ED5D0101CC6FA10EF8
:10E8E0000101ED5D02E2F0EC5EF00F012BB9E4D026
:10E8F0000101300E006F0101300E016F0101300E79
:10E90000026F0101300E036FDEC104F10101550EEB
:10E91000056F0101DE5101E195D00101DE0501E144
:10E9200091D00C01060EFD6F2B0E0101CE5D45E16D
:10E930000C01010EFE6F0101DE510C01FE5D3CE297
:10E94000010E0C01FE150C01FF6F0C01FE51EA6A6D
:10E95000CE0FE96E010EEA22EF50D00F0C01FC6FD2
:10E960000C01FF510FE00C01FC39F00BE66E0C01BD
:10E97000FD51EA6A000FE96E010EEA22E552E75006
:10E98000EF6E17D00C01FD51EA6A000FE96E010E1F
:10E99000EA22EF500C01FC25E66E0C01FD51EA6AFB
:10E9A000000FE96E010EEA22E552E750EF6E0C010E
:10E9B000FD2B0C01FE2BBFD745D00101042B0C0110
:10E9C000FE6B0101DE510C01FE5D3CE2010E0C010B
:10E9D000FE150C01FF6F0C01FE51EA6ACE0FE96EC5
:10E9E000010EEA22EF50D00F0C01FC6F0C01FF5119
:10E9F0000FE10C01FC39F00BE66E0C01FD51EA6AE7
:10EA0000000FE96E010EEA22E552E750EF6E17D0D3
:10EA10000C01FD51EA6A000FE96E010EEA22EF5087
:10EA20000C01FC25E66E0C01FD51EA6A000FE96E4F
:10EA3000010EEA22E552E750EF6E0C01FD2B0C01AE
:10EA4000FE2BBFD70101DE6B0101F86B100E010137
:10EA5000F85D0BE20101F851EA6ACE0FE96E010E92
:10EA6000EA22EF6A0101F82BF1D7020E0101ED5DF8
:10EA70000101EE6F0101EE511DE00101EC6B01019E
:10EA8000EE510101EC5D16E20101EC51EA6A000F62
:10EA9000E96E050EEA22EF50E66E0101EC51EA6ADA
:10EAA000000FE96E030EEA22E552E750EF6E010116
:10EAB000EC2BE5D7EEC1FCF39EAA05D0AFCFFEF557
:10EAC0009E9AB9EC2DF02ED8060EE15C02E2E16AC6
:10EAD000E552E16EE552E7CFD9FF12000101FE0ECB
:10EAE000ED6F0101EC6B0101ED510101EC5D11E2F3
:10EAF0000101EC51EA6A000FE96E050EEA22EF50BF
:10EB00000A0804E10101EC290101ED6F0101EC2B80
:10EB1000EAD79EAA05D0AFCFFEF59E9AB9EC2DF0AC
:10EB200001D81200FE0E0101D880ED550101EE6FF3
:10EB30000101EE5123E00101EC6B0101EE510101F5
:10EB4000EC5D1CE20101EC510101ED250101F76FC3
:10EB50000101F751EA6A000FE96E050EEA22EF5053
:10EB6000E66E0101EC51EA6A000FE96E050EEA2239
:10EB7000E552E750EF6E0101EC2BDFD7EEC1ECF16F
:10EB8000FE0E0101EC5D0BE20101EC51EA6A000F9F
:10EB9000E96E050EEA22EF6A0101EC2BF1D71200B3
:10EBA0000401CB51CB07000916E00401C7C4E9FFFB
:10EBB000C8C4EAFFC72B000EC823EF50E66E04015D
:10EBC000C9C4E9FFCAC4EAFFC92B000ECA23E55233
:10EBD000E750EF6EE5D71200040120511F0B01082A
:10EBE00001E04AD004012051600BE842E842E842CB
:10EBF000E842E842010801E03FD00401245104E06A
:10EC00000401240501E038D004012151220A2EE03C
:10EC1000030A20E0010A1AE0210A10E0010A01E0DB
:10EC20002BD00401B50EC26F040EC36F0401080E91
:10EC3000C56F0401C4810401C48F1ED00401B50E48
:10EC4000C26F040EC36F0401C48F16D00401010EFD
:10EC5000C16F12D00401CE0EC26F040EC36F040147
:10EC6000070EC56F0401810EC46F06D022C4CCF418
:10EC70000401CC8F0401C48F120004011C7D400EDE
:10EC800004011C17880E04011C1312000401187DD6
:10EC90000401300E1A6F040E1B6F0401400E196F31
:10ECA000400E04011817880E040118131200636A3D
:10ECB000626A0F019F0E5D6F0F015E6B0F014D6B5E
:10ECC0000F014E6B0F01FB0E5C6F658C0401C46B72
:10ECD0000401C16B0401BD6B0401CD6B659C0F0188
:10ECE000160E4C6F62A603D062960400FBD765989F
:10ECF0001200800E0401205D01E020D00401800E8E
:10ED0000C46F04012351030A17E0010A0CE0030A4F
:10ED100001E014D00401BC0EC26F000EC36F0401E9
:10ED2000120EC56F0BD00401CE0EC26F000EC36F62
:10ED30000401430EC56F02D00401C46B120004012C
:10ED4000C48F0F014D6B0F014E6B0401BE6B22C4CB
:10ED5000BDF40401225104E10401100ECD6F2ED048
:10ED60000401200ECD6F0401CE6B4B0ECF6FD06B24
:10ED7000D16B0401D26B0401D36B0401080ED46F74
:10ED80000401010ED56F0401CC6B0401CC8F04018A
:10ED9000B16B0401B06B0F011A0E4E6F0401148D9C
:10EDA0000401149F0F011E0E4F6F04011C8D0401FE
:10EDB0001C9F0401188D0401189F68DF12000401D4
:10EDC00024510F0B080DF3CFE9FFF4CFEAFF000E3B
:10EDD000E926040EEA22E9CFC7F4EACFC8F4040119
:10EDE00024AF05D00401040EC727000EC82312006B
:10EDF0000401286B0401296B040120511F0B020A36
:10EE000012E0030A0DE0010A01E01AD00401C48FE8
:10EE1000040128810401C65102E00401288310D0B6
:10EE20000401C48F0DD00401C48FC9DFC7C4E9FF3A
:10EE3000C8C4EAFFEF50040B03E00401010E286F81
:10EE40000401C4AF0AD00401280EC26F040EC36FC0
:10EE50000401C4810401020EC56F120004012205E1
:10EE600010E1040120511F0B00090BE10401C48FC4
:10EE70000401C66B030E0401215D03E10401010ED0
:10EE8000C66F0401225130E1040120511F0B02081A
:10EE90002BE1040124510F0B000926E00401C48F6B
:10EEA0008EDFC7C4E9FFC8C4EAFF840EEF6E030E0D
:10EEB0000401215D19E0040124510F0BEA6A4C0F93
:10EEC000E96E0F0EEA22EE90ED6AC7C4E9FFC8C4EE
:10EED000EAFFC80EEF6E040124AF06D0C7C4E9FFF5
:10EEE000C8C4EAFF400EEF6E120004012051600B0F
:10EEF000E842E842E842E842E842000901E047D03F
:10EF0000040121510B0A3FE0010A2AE00B0A26E026
:10EF1000020A24E0030A20E0080A11E0010A0DE0D9
:10EF20000F0A09E0030A01E032D00401C48F040192
:10EF3000080ECD6F2CD0DDDE2AD001DF28D00401F1
:10EF4000BD0EC26F040EC36F0401C4810401010E23
:10EF5000C56F0401C48F1BD04BDF19D07FDF17D0E2
:10EF6000040124510401C26FC36BBE0E0401C22709
:10EF7000040E0401C3230401C4810401010EC56F02
:10EF80000401C48F04D00401C48F22C4BEF4120053
:10EF90000401080ECB6F080E0401C55D0EE2C5C466
:10EFA000CBF40401BF0503E10401020EBF6F0401AD
:10EFB000BF5103E10401010EBF6F0401049304017A
:10EFC0000491CBC405F40401CB510401C55D0401D7
:10EFD000C56F0401280EC96F040ECA6F0401C4B1C5
:10EFE0001DD00401CB51CB07000917E00401C2C4B6
:10EFF000F6FFC3C4F7FFC22B000EC3230800F55071
:10F00000E66E0401C9C4E9FFCAC4EAFFC92B000EB9
:10F01000CA23E552E750EF6EE4D709D0C2C4C7F463
:10F02000C3C4C8F4BDDDC7C4C2F4C8C4C3F412006D
:10F0300065980401080E016F0401C4BF20D00401CB
:10F04000C15111E00401020EC06F0401056B0401FF
:10F05000C80E046F0401280E026F040E036F040132
:10F06000C80E006F4FD00401200E026F040E036F14
:10F0700004018C0E006F0401840E046F43D0040160
:10F08000C15101E03FD0040120AF2CD00401C55193
:10F09000006E016A04010050265D0150275902E20A
:10F0A00026C4C5F475DF0401010EC06F0401200EF3
:10F0B000026F040E036F0401800E006F0401080E3E
:10F0C000016F0401200E026F040E036F0401800E15
:10F0D000006F0401280E066F040E076F0401C80EAE
:10F0E000046F10D00401020EC06F0401056B04010F
:10F0F000C80E046F0401280E026F040E036F040192
:10F10000C80E006F1200645001E034D004010051B9
:10F110003C0BE842E8420D0811E1040104AF02D0C3
:10F120000401046B0401BF6B0401C06B0401C56BD7
:10F130000401C46BDADE50DD7BDF8CD0020E0401EB
:10F14000C05D17E10401070ECB6F0401280EC76FE5
:10F15000040EC86F0401CE0EC96F040ECA6F20DD05
:10F160000401010ED56F0401200E026F040E036F1F
:10F1700071D02FD0040E645C01E06CD0080E040145
:10F18000CD5D0BE122C45EFF0401040ECD6F0F01C3
:10F190005E5103E00401100ECD6F0401C00519E1BA
:10F1A0000401280E066F040E076FF2DE020E040142
:10F1B000BF5D04E10401840E046F4CD0040104BD62
:10F1C00004D00401C80E046F45D00401880E046FFA
:10F1D00041D00401C16B020E0401C05D01E02BD0DF
:10F1E00065A829D004010151006E016A080E0018BB
:10F1F00001E1015001E01FD0040100513C0BE84245
:10F20000E8420D0801E017D0040100BF14D004014A
:10F21000200E026F040E036F0401280EC76F040E48
:10F22000C86F0401200EC96F040ECA6F0401080ED6
:10F23000CB6FB6DC0FD00401C06B0401080E016F68
:10F240000401200E026F040E036F04018C0E006F88
:10F250000401046B12000401CD511BE1656A0F012A
:10F260005C6B65B603D065860400FBD70401010E14
:10F27000CD6F0F01140E5F6F65BAFED7626A0F0182
:10F280005C6B0F015C810F015C890401020ECD6F84
:10F29000A0880401CD050CE165BA0AD0626A0F01AD
:10F2A0005C6B0F015C810F015C890401020ECD6F64
:10F2B0006250040B0CE00F010F015C51040B07E0DE
:10F2C00065920F015C9562A402D06294FCD765B28E
:10F2D000A9D06250010B15E00F010F015C51010B29
:10F2E00010E0E5DC0401040ECD6F0401200E026F76
:10F2F000040E036F0401080E016F04018C0E006FF1
:10F3000062906250100B0AE00F010F015C51100B6C
:10F3100005E00F015C856298658262986250400B3F
:10F3200006E00F010F015C51400B01E0629C62504E
:10F33000200B16E00F010F015C51200B11E00F01B3
:10F340004CA10DD0800E0401005D07E1840E040184
:10F35000045D03E104018C0E006F0F014C91629A71
:10F36000636A040E0401CD5D01E25CD00F010F0160
:10F370005C51080B08E06250080B05E062A603D060
:10F38000C2DE6296FBD704011CBF4CD0030E040101
:10F39000B15D02E10401B16B0401B15101E142D060
:10F3A000020E0401B15D09E104011E6B1F6B040133
:10F3B0001D6B63DC0401030EB16F0401B10501E0B4
:10F3C00031D0B2C4CBF40401B251400803E20401CD
:10F3D000400ECB6F0401CB510401B25F0401B25166
:10F3E0000AE10401030EB16F400E0401CB5D03E19D
:10F3F0000401020EB16FCBC41DF40401700E1E6F28
:10F40000040E1F6F0401700EC96F040ECA6FB3C4DF
:10F41000C7F4B4C4C8F4D0EC75F0C7C4B3F4C8C41E
:10F42000B4F42BDC12000401D56B0401CC9FA2883C
:10F430003EDC11DF1200A098656A1200A050100B8C
:10F4400006E0A150100B03E006DF02D8A1981200DD
:10F45000040118AF02D0000E14D0200E0401CD5DBF
:10F4600002E2000E0ED0A0B802D0000E0AD00401B5
:10F47000195104E146EC76F0000E03D00401195155
:10F4800000D01200A0B802D0010E03D00401B15187
:10F4900000D01200D9CFE6FFE1CFD9FFFD0EDBCFC0
:10F4A000B3F4FE0EDBCFB4F4FC0EDBCFB2F40401F8
:10F4B000010EB16FE552E7CFD9FF1200D9CFE6FFB9
:10F4C000E1CFD9FFE652C4DFDF6EDF5013E0A09832
:10F4D0000401300EC76F040EC86FFD0EDBCFC9F4F8
:10F4E000FE0EDBCFCAF4DFCFCBF4D0EC75F0A088F2
:10F4F00046EC76F0DF5000D0E552E552E7CFD9FF79
:10F500001200FFFFFFFFFFFFFFFFFFFFFFFFFFFFF7
:00000001FF
